:0600000076EF06F012008D
:0600080004EF08F01200F5
:100018000CEF08F012001DEE00F02DEE00F0F86A6B
:0600280092EF06F0120049
:1000300000003E0E006E016AFC0E026E036A046A46
:10004000076808680968066A1200D9CFE6FFE1CFA1
:10005000D9FFE65204501EE1040108BF1AD0400E39
:10006000E66E600EE66E000EE66E38EC06F0E552C7
:10007000E552E552010E046EDF6A400EDF5C09E2D4
:10008000DF50EA6AA00FE96E000EEA22EF6ADF2A6B
:10009000F4D717D100016051080A01E10DD10F0A10
:1000A00001E1D3D0010A01E1CAD0030A67E0010AE5
:1000B00058E0070A44E0010A01E003D10001020E02
:1000C000A06F00013A0EA16F0001010EA26F0001A6
:1000D000010EA36F0001A46B100EA56FA66BA76B9A
:1000E00001C0A8F002C0A9F003C0AAF0100E0001E0
:1000F000A95F000E0001AA5B0001AB6B0001030EBB
:10010000AC6F0001F80EAD6FAE69AF6BB06B000164
:10011000080EB16FB26BB36BB46B0001B56904012B
:100120000CBF0CD0400EE66EA00EE66E000EE66E22
:1001300008EC06F0E552E552E552046AC2D000012F
:10014000615107E13F0E006EF80E016E0268036A0E
:1001500006D03E0E006E016AFC0E026E036A046A4F
:10016000B0D0040E056E0028055C06E20400AED88F
:100170009DEC04F0052AF7D7046AA3D0E8680718B5
:1001800005E1E868081802E1E868091806E161C0BD
:1001900007F062C008F063C009F007500001611960
:1001A00008E108500001621904E1095000016319D7
:1001B00000E143E1DF6A00016551DF5C3EE2000ED1
:1001C000075C100E0858000E09582CE300285B6EDF
:1001D0005C6A0A0ED8905B365C36E806FBE15D6A25
:1001E0005CBE5D685B50075C5C5008585D50095808
:1001F00019E23A0E0001D8806555DF24EA6A660FDD
:10020000E96E000EEA22EF50E66E0650E96EEA6AE9
:10021000E9BEEA680A0EE926000EEA22E552E75036
:10022000EF6E062A072A000E0822000E09223A0E57
:10023000065C01E15ED8DF2ABED7046A42D059D8F5
:10024000076808680968046A3CD00001070EA06FBF
:1002500061C0A1F062C0A2F063C0A3F064C0A4F0CA
:1002600065C0A5F061C0F6FF62C0F7FF63C0F8FF8C
:10027000DF6A00016551DF5C0FE209003A0E000100
:10028000D8806555DF24EA6AA60FE96E000EEA22DF
:10029000F5CFEFFFDF2AEDD704010CBF0CD0400EE5
:1002A000E66EA00EE66E000EE66E08EC06F0E55275
:1002B000E552E552046A05D06592656A68D8FF0088
:1002C00000D0E552E552E7CFD9FF1200F66A05509B
:1002D000F76EF86AD890F736F836F736F836140E17
:1002E000A66EF29E550EA76EAA0EA76EA682A694C3
:1002F0001200D9CFE6FFE1CFD9FFE652DF6A000E48
:10030000E76E0618E8AE02D0063403D0E750D88076
:10031000065436E206505B6E5C6A5D6A5BAE02D0E4
:100320005C685D685B50075CF66E5C500858F76E61
:100330005D500958F86EDF50EA6A0A0FE96E000E48
:10034000EA22EF50F56E0D00DF2A0606065009E09E
:10035000DF50EA6A0A0FE96E000EEA22EF50F56EEE
:1003600001D0F5680C00DF2A240EA66EF29E550E11
:10037000A76EAA0EA76EA682065001E00606BFD79A
:10038000A694066AE552E552E7CFD9FF1200D9CF0D
:10039000E6FFE1CFD9FFE652DF6AFF0EDF5C0AE23B
:1003A000E868E85005E0E80600D000D000D0F9D7B2
:1003B000DF2AF3D7E552E552E7CFD9FF12005FD924
:1003C000E652645032E16296040100513C0BE8426F
:1003D000E8420D0828E1180E021923E1040E031962
:1003E00020E1100E026F040E036FDF6ADF505B6EB8
:1003F0005C6A080E5B5C000E5C5813E2DF50EA6A30
:10040000180FE96E040EEA22EF50E66EDF50EA6A3A
:10041000100FE96E040EEA22E552E750EF6EDF2A74
:10042000E5D70ED80AD03DD808D0040E645C03E1AD
:1004300062964DD802D0000E01D0010EE55224D1B3
:100440001ED9E652040104BF046B556A516A526A10
:10045000536A546A4FEC03F0DF6ADF505B6E5C6AEC
:10046000010E5B5C000E5C5819E2525017E1F76A0E
:10047000DF34FE0BF736F66EA40EF6260E0EF722CC
:100480000900F5CF5BF00800F5CF5CF004D05CC04C
:10049000FAFF5B50F96EFBDFDF2ADFD79ED8E5520B
:1004A000F3D0020E515C0EE176D80401180E026FF3
:1004B000040E036F080E016F00BD02D0C80E05D0F8
:1004C000880E03D0BCD8CCD88C0E006F1200040E5E
:1004D000575C0AE112C438FF0F013851000802E2EC
:1004E000050E01D0030E576E51040FE110D8020E15
:1004F000555C03E10401840E06D0040104BD02D062
:10050000C80E01D0880E046F12001FEF03F0B7D899
:10051000020EE126080E535C000E54580DE253C043
:10052000DEFF54C0DDFF555002E1010E03D055043B
:1005300006E1020E556E03D0080EDE6EDD6A040180
:1005400004930491010EDB500413DFCF05F4DE5059
:10055000535EDD50545A0001180EE26F040EE36F33
:1005600058A20CD085D810E0E0C0F6FFE1C0F7FF3C
:100570000800F55068D8F6E2DB06F4D779D804E035
:1005800087D8FCE2DB06FAD7020EE15C02E2E16A00
:10059000E552E16E79D073D8020EE126030E040114
:1005A0000015E76E010EE7CFDBFF01C4DFFFDE5071
:1005B0005326DD5054220001180EE06F040EE16F47
:1005C00057D804E065D8FCE2DB06FAD7020EE15CFE
:1005D00002E2E16AE552E16E57D06598525005E1BA
:1005E0003FD8840E006F040118D0040110AF17D05B
:1005F0005350165D5450175904E216C453F017C4F3
:1006000054F085DF010E516E2BD8800E006F04016F
:10061000180E066F040E076FC80E046F1200020E4C
:10062000516E0401056BC80E046F0401080E016FC2
:10063000180E026F040E036FC80E006F1200516A8D
:100640000401046B1200E2C0E9FFE3C0EAFFEF6EB1
:10065000E22B000EE323E02BE123DF06010E120064
:100660000401080E016F100E026F040E036F1200DA
:10067000D9CFE9FFDACFEAFFEE50ED101200D9CF63
:10068000E6FFE1CFD9FF1200E552E7CFD9FF120014
:10069000E0C0E9FFE1C0EAFFEF5023EF03F00401FF
:1006A0001051600BE842E842E842E842E8420009A3
:1006B00001E012001151070A43E00B0A41E0070A6A
:1006C00034E0010A24E00B0A20E0020A1EE0030ADB
:1006D0001AE0080A10E0010A0CE00F0A08E0030A19
:1006E00001E01200010E526E040E576E1200A1EFCF
:1006F00003F0D7EF03F0010E526E0001590EE06FC8
:10070000000EE16F0ED0F1EF03F01FEF04F0010EC9
:10071000526E14510001E06FE16B5A0EE027000E9B
:10072000E1235892010E536E1200010E526E1451C5
:10073000EA6A5A0FE96E000EEA2212C4EFFF1200B5
:100740001200800E0401105D31E11351030A20E014
:10075000010A0BE0030A29E1010E526E0001E40ECA
:10076000E06F0D0EE16F120E1ED0AAD89A0EF6267B
:100770000E0EB8D8020E0001F76AE025F66EE151C0
:10078000F7220900F5CF53F00A00F5CF54F00DD051
:1007900097D89E0EF6260E0EA5D8E0C0F6FFE1C053
:1007A000F7FF0800F550536E546A58821200010E8C
:1007B000526E0F0EE66E270EE66E0F0E9BD8010EE0
:1007C000E66E5A0EE66E000E95D812C459F004017A
:1007D000125103E1050E576E1200060E576EF3EF2D
:1007E00005F00401186B196B040110511F0B020A6C
:1007F0000EE0030A09E0010A17E1010E526E58A04B
:1008000013D00401188310D0010E526E0DD04AD8B7
:1008100001E0010E5ED8E2C0E9FFEA6EEF50040B82
:1008200003E00401010E186F520408E10001180EE4
:10083000E06F040EE16F5892020E536E1200040135
:1008400012050CE110511F0B000908E1010E526E58
:10085000030E115D02E1588001D05890125121E140
:1008600010511F0B02081DE114510F0B000919E074
:1008700019D801E0010E2DD8030E0401115D02E12B
:10088000840E03D014AF07D0400EE2C0E9FFE3C0EE
:10089000EAFFEF6E1200880EE2C0E9FFE3C0EAFF54
:1008A000EF6E1200010E526E14510F0B080DF35033
:1008B0005C6A000F5B6E040E5C221451800B120008
:1008C000010E526E1251F66EF76AD890F636F73670
:1008D0001200040DF35000015B24E26F000E5C2057
:1008E000E36F1200F7220900F5CFE0F00A00F5CF20
:1008F000E1F01200E66E76EC05F0E552E552E552C5
:10090000120065A60CD8570409E165BA07D0626ADF
:100910000F01366B36813689020E576E1200656AFA
:100920000F01366B6586010E576E1200656A0F0166
:10093000366B576A120096EF04F0575001E112002F
:100940006250040B05E00F013651040B01E083D81F
:1009500065B212006250010B05E00F013651010B28
:1009600001E093D86250100B05E00F013651100BD7
:1009700001E01FD86250200B05E00F013651200B1B
:1009800001E071D8030E575C01E21200566A040EB2
:10099000565C0EE26250080B0BE00F013651080B5B
:1009A00007E0DFEC01F0000901E16296562AEFD77B
:1009B0001200D9CFE6FFE1CFD9FF020EE12636CFF4
:1009C000DFFF0F01040E366F629865828C50040BB6
:1009D00001E0010E5B6E8C50080B01E0010E5B1014
:1009E000E76E010EE7CFDBFF8C968C94A198A08870
:1009F0000300A150100B05E1D050080B02E10300E9
:100A0000F8D7A098DF500F013613010EDB50E8B085
:100A10008C86E8A08C96010EDB50E8B08C84E8A0B0
:100A20008C94D50E4F6E020E506E4FC05BF050C0CE
:100A30005CF04F06000E505A5B505C1002E0040060
:100A4000F4D7020EE15C02E2E16AE552E16EE552A2
:100A5000E7CFD9FF120065920F01369562A402D04C
:100A60006294FCD712000F0126A10DD0800E040164
:100A7000005D07E1840E0401045D03E104018C0EB6
:100A8000006F0F012691629A1200636A626A0F0179
:100A90009F0E376F0F017B0E366F0F01386B0F0EF5
:100AA000E66E270EE66E0F0EE66E20D8E552E55292
:100AB000E5520F01160E266F62A605D0629600D091
:100AC00000D00000F9D765981FEC03F00401080E70
:100AD000016F0401100E026F040E036F04018C0EEF
:100AE000006F5890596A030E576E1200D9CFE6FF77
:100AF000E1CFD9FFFD0EDBCFE9FFFE0EDBCFEAFF32
:100B0000FC0EDB5004E0EE6AFC0EDB06F9D7E55282
:100B1000E7CFD9FF1200040110511F0B010801E0BB
:100B20001200145101E01200060E115D21E1135173
:100B3000230A1DE0010A0DE0030A19E1020E526EBC
:100B4000590405E10001080EE06F0E0EE16F090E79
:100B50000CD0020E526E590405E100017D0EE06FCB
:100B60000E0EE16F590403E11D0E536E546A588254
:100B700004011051600BE842E842E842E842E842D2
:100B8000010801E0120011510B0A26E0080A19E0E1
:100B9000090A12E0080A09E00B0A05E0080A01E068
:100BA0001200F1EF05F0F2EF05F0020E526E0001B7
:100BB0004A0EE06F000E0BD0020E526E13C44AF0C4
:100BC0001200020E526E00014B0EE06F000EE16F3C
:100BD0005892010E536E1200020E526E12C44BF068
:100BE0001200120012004C6A0F011E0E276F040142
:100BF000400E096F200E0A6F040E0B6F880E086FEF
:100C00000401600E0E6F040E0F6F400E0C6F120089
:100C1000D9CFE6FFE1CFD9FFE652FC0EDB5040080A
:100C200005E2400EF36EFC0EF3CFDBFFDF6AFC0E35
:100C3000DB50DF5C0FE2DF504DD8EF50E66EDF5047
:100C4000EA6A600FE96E040EEA22E552E750EF6EA1
:100C5000DF2AEDD7FC0EDBCF0DF4400E04010C179C
:100C60000C7D880E0C13E552E552E7CFD9FF120038
:100C7000D9CFE6FFE1CFD9FF4C6A040108BF25D0E8
:100C8000FC0EDBCF5BF00951D8805B5403E2FC0E15
:100C900009C4DBFF4C6AFC0EDB504C5C0FE24C508D
:100CA000EA6A200FE96E040EEA22EF50E66E4C501D
:100CB00011D8E552E750EF6E4C2AEDD70401400EF3
:100CC000096F0817087D880E08134C50E552E7CFCE
:100CD000D9FF1200E76EFD0EDBCFE9FFFE0EDBCF82
:100CE000EAFFE750E926000EEA2212001DEE00F0AE
:100CF0002DEE00F0F86AF66A100EF76E0800F55057
:100D0000FF0808E1010EF66E100EF76E0800F550B0
:100D1000FF0806E080AE02D000EF08F080AEFED7FC
:100D200001D812000DD8040034D837D8060E575C0D
:100D300005E16550020B02E125EC00F0F4D712004A
:100D4000600ED36E9B8C580E4F6E020E506E4FC0CD
:100D50005BF050C05CF04F06000E505A5B505C10C8
:100D6000F6E165A604D06592656AC7EC01F00F0153
:100D7000140E396F576A586A596A19EC00F04D6AB7
:100D80004E6A8C968C94959695940F01486B496B9E
:100D9000120081EC04F09DEF04F04D504E1004E180
:100DA000100E4D6E270E4E6E4D06000E4E5A060E5C
:100DB000575C02E28C868C94060E575C12E14D5013
:100DC0004E100FE10001E65102E18C868C94030E77
:100DD000E65D02E18C968C84E62BE651030801E285
:100DE000E66B12001201000200000008D8043C006B
:100DF00002000102000109022900010100C03209BC
:100E00000400000203000000092111010001221D5D
:100E100000070581034000010705010340000104AC
:100E200003090434034D006900630072006F00631E
:100E300000680069007000200054006500630068CD
:100E4000006E006F006C006F0067007900200049A1
:100E5000006E0063002E0026034800490044002075
:100E600000550053004200200042006F006F0074E4
:100E7000006C006F0061006400650072000600FFF6
:100E80000901A10119012940150026FF00750895E7
:100E9000408100190129409100C0F60DF60D1F0E8A
:100EA000230E570E160BC00EF36E00EE00F00E0E62
:100EB00001D81200EA6002D0EE6AFCD7F350E96074
:060EC0001200EE6AFCD7EF
:061000000AEF65F012008A
:061008006EEF24F012005F
:061018002CEF37F012007E
:10102A00030081CA000000050000E100000078CA40
:10103A000000B70E00000900000076CA0000F3079E
:10104A00000002000000020100000000000132005E
:10105A00000000000180004D0000000200000000B6
:10106A0000000132000000000001A700FBFFDFFFC3
:10107A00015700EFFF0400014E00F2FF0700014C88
:10108A0000F3FF0800014A00F5FF0A00014400F8D6
:10109A00FF0B00014800FAFF0D00014E00FCFF0F94
:1010AA0000015000FFFF100001320000000A000199
:1010BA002E000200090001330002000A00012D007F
:1010CA0004000800012D0004000800012F0005009B
:1010DA00080001310007000700012E000700060082
:1010EA00013200080006000133000900050001363C
:1010FA00000A0004000134000A0003000139000B51
:10110A00000300013D000C0002000141000D000136
:10111A00000146000E0001000146000E00FFFF011B
:10112A0041000D00FFFF013D000C00FEFF013E00E3
:10113A000C00FDFF0139000B00FDFF0136000A001B
:10114A00FCFF0133000900FBFF0132000800FAFF2F
:10115A000135000800F9FF012E000600F9FF012EF3
:10116A00000600F9FF012D000400F8FF012D00041C
:10117A0000F8FF012E000200F7FF012E000200F71F
:10118A00FF0132000000F6FF012D000000F7FF0109
:10119A002E00FEFFF7FF012900FEFFF8FF012B00DA
:1011AA00FDFFF8FF012F00FBFFF8FF012B00FBFFFB
:1011BA00F9FF013100F9FFF9FF012E00F9FFFAFFEB
:1011CA00013200F8FFFAFF013300F7FFFBFF013697
:1011DA0000F6FFFCFF013900F5FFFDFF013900F5BC
:1011EA00FFFDFF013D00F4FFFEFF014100F3FFFF99
:1011FA00FF014600F2FFFFFF013200F6FF01000186
:10120A00C60200008E00015B00EEFFFEFF015100E6
:10121A00F0FFFDFF014800F3FFFAFF014100F5FF6F
:10122A00F9FF013C00F7FFF8FF013A00FAFFF6FF69
:10123A00013600FCFFF6FF013C00FFFFF4FF012826
:10124A00000100F8FF0129000200F8FF012600034F
:10125A0000F9FF012B000500F9FF012E000700FA33
:10126A00FF012F000800FBFF0133000900FBFF010B
:10127A003F000C00FCFF010000000000000201001A
:10128A00000000000132000000000001CE003F0013
:10129A006A000200000000000001320000000000A5
:1012AA00011202000096FF0141000D000100013EFB
:1012BA00000C0003000134000A000300012F00089B
:1012CA000005000140000A000800013D0007000A6D
:1012DA0000011B0002000500011B000200050001BD
:1012EA003C0001000C00013700FFFF0B00012F003A
:1012FA00FDFF0900013600FAFF0900013500F9FF78
:10130A000800013D00F6FF0700013C00F5FF05005B
:10131A00014400F3FF0400014600F2FF010001004E
:10132A00000000000002010000000000013200007D
:10133A0000000001900164FF4AFF02000000000063
:10134A00000132000000000001A200FBFFE0FF01E3
:10135A002D00F7FFFFFF012600F9FFFDFF011D0029
:10136A00FBFFFDFF012000FBFFFCFF012700FBFF45
:10137A00FAFF012B00FDFFF8FF012E00FEFFF7FF29
:10138A00013200FFFFF6FF0132000100F6FF0133D0
:10139A00000200F6FF012B000300F8FF01270005F9
:1013AA0000FAFF012A000600FAFF012B000700FBE2
:1013BA00FF012B000800FDFF012F000900FDFF01BE
:1013CA0060001300FEFF019B001F000000012B00BC
:1013DA00F9FF0500012A00FAFF0600012700FBFFBA
:1013EA000600012800FCFF0700012400FCFF06009C
:1013FA00012400FEFF0700012800FFFF0800012862
:10140A0000FFFF0800012D0001000900012D000165
:10141A00000900012F0003000900012D0004000843
:10142A000001280004000700012E00060007000141
:10143A002E000700060001320008000600013300F2
:10144A0009000500013100090004000136000A0004
:10145A0004000134000A000300016B0015000400B7
:10146A000173001700010001500010000000015133
:10147A00001000FEFF0148000E00FDFF014A000EA9
:10148A0000FBFF014A000E00FBFF0141000B00F9BF
:10149A00FF0140000A00F8FF0139000800F8FF01C7
:1014AA003D000700F6FF013C000500F5FF0138008A
:1014BA000200F5FF0141000100F3FF0128000000CE
:1014CA00F8FF012900FEFFF8FF012400FEFFF9FFE3
:1014DA00012800FCFFF9FF012800FCFFF9FF012E9B
:1014EA0000FAFFF9FF012E00F9FFFAFF012B00F9BC
:1014FA00FFFBFF0187001B0000000196000000E2CD
:10150A00FF01DE033AFF0000017D00E7FF00000152
:10151A006900EBFF0200015600EFFF0300014400DF
:10152A00F3FF0400013800F6FF0500013D00F6FF55
:10153A000700013500F8FF0700013D00F9FF0A0026
:10154A00013A00FAFF0A00013F00FCFF0C00013DCE
:10155A0000FEFF0C00014600FFFF0E0001500001D3
:10156A00001000014E0004000F0001480006000DA3
:10157A000001440008000B000120000400050001DE
:10158A0027000600050001220006000300012600CC
:10159A0007000300012400070002000129000800D7
:1015AA0002000155001100010001000000000000C6
:1015BA00020100000000000132000000000001EA00
:1015CA00008A00E5FF02000000000000013200006E
:1015DA00000000016900EBFFFFFF015B00EEFFFD69
:1015EA00FF014F00F1FFFBFF012200FAFFFDFF019F
:1015FA002200FAFFFDFF013C00F7FFF8FF01390066
:10160A00F9FFF7FF013400FDFFF6FF013300FEFF8B
:10161A00F6FF0138000200F5FF0134000300F6FF6F
:10162A000139000700F7FF013C000900F8FF011D1E
:10163A00000500FDFF0126000700FDFF014A000E1C
:10164A0000FBFF015B001200FDFF0164001400FFB4
:10165A00FF0164001400010001560011000300019B
:10166A004F000F0005000145000C000700013C0077
:10167A0009000800013900070009000131000400CF
:10168A00090001370001000B00013200FFFF0A00C8
:10169A00013600FCFF0A00013900F9FF0900013C8C
:1016AA0000F7FF0800014300F4FF0600014A00F2B8
:1016BA00FF0500015600EFFF0300015F00EDFF0187
:1016CA00000100000000000002010000000000010B
:1016DA0032000000000001770176FF4EFF02000091
:1016EA00000000000132000000000001A200FBFF20
:1016FA00E0FF012D00F7FFFFFF012600F9FFFDFFC4
:10170A00011D00FBFFFDFF012000FBFFFCFF01277D
:10171A0000FBFFFAFF012B00FDFFF8FF012E00FE80
:10172A00FFF7FF013200FFFFF6FF0132000100F66A
:10173A00FF0133000200F6FF012B000300F8FF014E
:10174A0027000500FAFF012A000600FAFF012B0014
:10175A000700FBFF012B000800FDFF012F00090015
:10176A00FDFF0160001300FEFF019B001F00000047
:10177A00012B00F9FF0500012A00FAFF06000127E4
:10178A0000FBFF0600012400FCFF0600012800FC04
:10179A00FF0700012400FEFF0700012800FFFF08E1
:1017AA0000012800FFFF0800012D000100090001C7
:1017BA002D0001000900012F000300090001280083
:1017CA0004000700012D0004000800012E00060095
:1017DA000700012E0007000600013200080006007B
:1017EA000133000900050001310009000400013637
:1017FA00000A0004000134000A000300016B00150E
:10180A00000400017300170001000150001000FFDE
:10181A00FF0150001000FFFF0148000E00FDFF010C
:10182A004A000E00FBFF014A000E00FBFF014100C7
:10183A000B00F9FF0140000A00F8FF013900080017
:10184A00F8FF013D000700F6FF013C000500F5FF27
:10185A000138000200F5FF0141000100F3FF0128F1
:10186A00000000F8FF012900FEFFF8FF012400FE36
:10187A00FFF9FF012800FCFFF9FF012800FCFFF92E
:10188A00FF012E00FAFFF9FF012E00F9FFFAFF010E
:10189A002B00F9FFFBFF0187001B000000019600E7
:1018AA000000E2FF01DE033AFF0000017D00E7FFCE
:1018BA000000016900EBFF0200015600EFFF030080
:1018CA00014400F3FF0400013800F6FF0500013D62
:1018DA0000F6FF0700013500F8FF0700013D00F997
:1018EA00FF0A00013A00FAFF0A00013F00FCFF0C60
:1018FA0000013D00FEFF0C00014600FFFF0E000143
:10190A00500001001000014E0004000F00014800C1
:10191A0006000D0001440008000B0001200004002D
:10192A00050001240006000400012400060004004A
:10193A000126000700030001240007000200012914
:10194A00000800020001550011000100010000001A
:10195A000000000201000000000001320000000047
:10196A000001EA008A00E5FF020000000000000111
:10197A00320000000000016900EBFFFFFF015B007D
:10198A00EEFFFDFF014F00F1FFFBFF012200FAFF0E
:10199A00FDFF012200FAFFFDFF013C00F7FFF8FFFF
:1019AA00013900F9FFF7FF013400FDFFF6FF0138A6
:1019BA0000FEFFF5FF0133000200F6FF01340003C9
:1019CA0000F6FF0139000700F7FF013C000900F8A3
:1019DA00FF011D000500FDFF0128000700FCFF01B3
:1019EA0049000E00FCFF015B001200FDFF016400CC
:1019FA001400FFFF016400140001000156001100E9
:101A0A000300014F000F0005000145000C0007000C
:101A1A00013C0009000800013900070009000131F2
:101A2A00000400090001370001000B00013200FF29
:101A3A00FF0A00013600FCFF0A00013900F9FF091C
:101A4A0000013C00F7FF0800014300F4FF06000113
:101A5A004A00F2FF0500015600EFFF0300015F0094
:101A6A00EDFF01000100000000000002010000007B
:101A7A00000001320000000000018D0189FF32FFE1
:101A8A000200000000000001320000000000019680
:101A9A000000001E00012C063C01000001A5000008
:101AAA0000DFFF01300290FF0000012B000700FB5E
:101ABA00FF012A000600FAFF0127000500FAFF01CC
:101ACA0027000500FAFF0126000300F9FF012400A0
:101ADA000200F9FF0124000200F9FF0128000000BA
:101AEA00F8FF012D000000F7FF012900FEFFF8FFB3
:101AFA00012900FEFFF8FF012D00FCFFF8FF012F6E
:101B0A0000FBFFF8FF012B00FBFFF9FF012E00F994
:101B1A00FFFAFF012B00F9FFFBFF012F00F8FFFB83
:101B2A00FF013100F7FFFCFF013600F6FFFCFF0161
:101B3A003400F6FFFDFF013900F5FFFDFF013C000F
:101B4A00F4FFFFFF017800E8FFFEFF014600F2FF05
:101B5A000000014700F2FF0200013D00F4FF02000D
:101B6A00013D00F4FF0200013B00F5FF04000136CD
:101B7A0000F6FF0400013300F7FF0500013300F708
:101B8A00FF0500013100F9FF0700012E00F9FF06E9
:101B9A0000012B00FBFF0700012B00FBFF070001E0
:101BAA002D00FCFF0800012400FEFF0700012900A8
:101BBA00FEFF0800012D00000009000128000000B6
:101BCA00080001290002000800012600030007009E
:101BDA000126000300070001270005000600012A6C
:101BEA000006000600012E0007000600012F00086B
:101BFA00000500019100E3FF00000201000000005F
:101C0A00000132000000000001C10074000000025F
:101C1A0000000000000001320000000000015F0027
:101C2A00EDFFFFFF015000F0FFFFFF014800F2FF48
:101C3A00FDFF013600F6FFFCFF012800F9FFFCFF5B
:101C4A00012700FAFFFBFF012000FBFFFCFF012335
:101C5A0000FBFFFBFF012200FDFFFAFF011B00FE54
:101C6A00FFFBFF012000FEFFFAFF0123000000F93D
:101C7A00FF0132000100F6FF0131000400F7FF0105
:101C8A0039000700F7FF0140000A00F8FF0145008C
:101C9A000C00F9FF0154001000FBFF01560011006F
:101CAA00FDFF0169001500FFFF0169001500010031
:101CBA00015B0012000300014F000F000500012222
:101CCA00000600030001220006000300013C00098F
:101CDA000008000135000700080001360004000A68
:101CEA000001320001000A00013200FFFF0A000170
:101CFA003600FCFF0A00013900F9FF090001400023
:101D0A00F6FF0800014300F4FF0600014F00F1FF4F
:101D1A000500015600EFFF0300016400ECFF01001B
:101D2A000100000000000002010000000000013272
:101D3A000000000000011001FFFF5DFF020000002B
:101D4A0000000001320000000000014B000F00FFFC
:101D5A00FF0146000E00FFFF0148000E00FDFF01D3
:101D6A003E000C00FDFF013B000B00FCFF013C00A4
:101D7A000B00FBFF0136000900FAFF0135000800DD
:101D8A00F9FF012A000600FAFF012B000500F9FFFE
:101D9A000128000400F9FF0128000400F9FF012BC3
:101DAA00000300F8FF0129000200F8FF01280001E2
:101DBA0000F8FF012D000000F7FF0132000000F6D5
:101DCA00FF012E00FEFFF7FF012E00FEFFF7FF01C5
:101DDA002B00FDFFF8FF012F00FBFFF8FF012B008E
:101DEA00FBFFF9FF012E00FAFFF9FF013200F8FFAD
:101DFA00FAFF013200F8FFFAFF012F00F8FFFBFF9C
:101E0A00013800F6FFFBFF013400F6FFFDFF013940
:101E1A0000F5FFFDFF013D00F4FFFEFF014100F365
:101E2A00FFFFFF014100F3FF0000016900EBFF0023
:101E3A0000016000EDFF0200015200F0FF04000102
:101E4A004A00F2FF0500014300F4FF0600013D00CD
:101E5A00F6FF0700014000F7FF0900014000F8FF04
:101E6A000A00013F00FAFF0B00013C00FBFF0B00D8
:101E7A00013D00FEFF0C00013C00FFFF0C00013297
:101E8A000000000A00012E0002000900012E0002D3
:101E9A00000900012D0004000800012D00040008BB
:101EAA0000012F0005000800012E000700060001AE
:101EBA003100070007000132000800060001330064
:101ECA00090005000136000A0004000134000A0076
:101EDA000300013E000C000300013D000C0002005B
:101EEA000146000E0001000146000E00010001003B
:101EFA0000000000000201000000000001320000A2
:101F0A000000000139000000DEFF020000000000AE
:101F1A000001320000000000016900EBFFFFFF0131
:101F2A005B00EEFFFDFF014F00F1FFFBFF01220006
:101F3A00FAFFFDFF012400FAFFFCFF014000F6FF53
:101F4A00F8FF013D00F9FFF6FF013600FCFFF6FF3E
:101F5A00013C00FFFFF4FF013C000100F4FF0136E1
:101F6A00000400F6FF013D000700F6FF0140000AE9
:101F7A0000F8FF0124000600FCFF0122000600FD14
:101F8A00FF0154001000FBFF015B001200FDFF017E
:101F9A0069001500FFFF01640014000100015600EA
:101FAA0011000300014F000F000500012600070081
:101FBA000300012000050004000143000A00090093
:101FCA0001390007000900013B0004000B0001373A
:101FDA000001000B00013C00FFFF0C00013600FC71
:101FEA00FF0A00013D00F9FF0A00014000F6FF0860
:101FFA0000012000FBFF0400012600F9FF03000195
:10200A004F00F1FF0500015B00EEFF0300016400D1
:10201A00ECFF0100010000000000000201000000C6
:10202A0000000132000000000001BC01B0FF02FF05
:10203A00020000000000000132000000000001ACB4
:10204A0000DEFFFBFF014300FDFF0D00013C00FF26
:10205A00FF0C00012800010008000123000100070D
:10206A000001240002000700011D00030005000111
:10207A0019000300040001200005000400011900F2
:10208A0004000300011D00050003000123000700EE
:10209A0001000133000A0002000191001D00010045
:1020AA0001940284000000017300000017000196E9
:1020BA00001E0000000173000000E9FF011D013944
:1020CA0000000001C9001700DFFF019001B0FF0006
:1020DA000001A0000000E0FF019600E2FF000001FD
:1020EA00A00000002000019E027AFF0000014600C5
:1020FA00F2FF0000012300F9FFFFFF011D00FBFFB3
:10210A00FDFF011500FDFFFDFF011B00FEFFFBFFA8
:10211A00011E00FFFFFAFF0147000200F2FF010063
:10212A00000000000002010000000000013200006F
:10213A000000000158075AFF5C040200000000007A
:10214A00000132000000000001C701A8FFE9FF01F9
:10215A0041000000F3FF015C014400F1FF014C0063
:10216A00F1FFFEFF011001CBFFF4FF014100000067
:10217A00F3FF01C7015800E9FF013C0000000C0011
:10218A00010701CDFF0D00015700EFFF04000157C1
:10219A00001100040001050133000B00013C00009E
:1021AA00000C00010601CDFF0C00016100EDFF04E7
:1021BA00000161001300040001060133000C000154
:1021CA00410000000D0001000000000000020100B3
:1021DA00000000000132000000000001FF00A8FF1B
:1021EA0083FF02000000000000013200000000002E
:1021FA0001C601580016000141000000F3FF010565
:10220A0001CDFFF5FF016200EDFFFBFF0161001345
:10221A0000FCFF0105013300F5FF0141000000F356
:10222A00FF010501CDFFF5FF015700EFFFFCFF019C
:10223A0057001100FCFF0107013300F3FF013C00C6
:10224A000000F4FF01C701A8FF17000141000000C8
:10225A000D0001100135000C00014C000F000300B5
:10226A00015C01BCFF0F0001410000000D000201EA
:10227A0000000000000132000000000001AC000074
:10228A000099FF0200000000000001320000000077
:10229A000001C60158001600013C000000F4FF01CD
:1022AA000601CDFFF4FF016200EDFFFBFF016000B4
:1022BA001300FDFF0106013300F4FF014100000095
:1022CA00F3FF010501CDFFF5FF015700EFFFFCFF0A
:1022DA000157001100FCFF0107013300F3FF013C25
:1022EA00000000F4FF01C701A8FF17000141000028
:1022FA00000D0001100135000C00014C000F000315
:10230A0000015C01BCFF0F0001410000000D00024A
:10231A0001000000000001320000000000019B00E3
:10232A000000A3FF020000000000000132000000CC
:10233A000000015500110000000146000000F2FFF4
:10234A00015500EFFF000001460000000E000201E7
:10235A000000000000013200000000000197001C8C
:10236A0000AAFF0200000000000001320000000085
:10237A0000014100FFFFF3FF012400F9FF02000101
:10238A002000FAFF0200011900FCFF0300012000EF
:10239A00FBFF0400011D00FDFF0500011B00FEFFFD
:1023AA000500011B00FEFF0500011E0000000600DB
:1023BA00012800010008000124000200070001248E
:1023CA0000040006000123000500050001240006A0
:1023DA00000400012B0008000300012E000900027E
:1023EA00000132000A0000000137000B0000000162
:1023FA002E000900FEFF012B000800FDFF01280046
:10240A000700FCFF0123000500FBFF012400040074
:10241A00FAFF0126000300F9FF0123000000F9FF7B
:10242A000123000000F9FF012200FDFFFAFF01224B
:10243A0000FDFFFAFF012700FAFFFBFF012400FA63
:10244A00FFFCFF012B00F8FFFDFF012E00F7FFFE46
:10245A00FF013700F5FFFFFF011500FCFF01000136
:10246A00130100003700012300F9FFFFFF012000DC
:10247A00FAFFFEFF011B00FBFFFEFF011600FCFF37
:10248A00FEFF011900FDFFFCFF011500FDFFFDFF26
:10249A00011500FFFFFCFF011900FFFFFBFF011EF2
:1024AA00000100FAFF0120000400FBFF01230005E0
:1024BA0000FBFF012B000800FDFF010000000000E7
:1024CA0000020100000000000132000000000001CB
:1024DA00500019002900020000000000000132002B
:1024EA000000000001CD000000D7FF012D00090007
:1024FA00010001260007000300011C00040004007B
:10250A00011500030003000116000200040001196E
:10251A00000000050001140000000400011600FE7E
:10252A00FF0400011200FEFF0300011500FDFF0376
:10253A0000011900FCFF0300011600FCFF02000164
:10254A001900FBFF0100011900FBFF010001000057
:10255A00000000000201000000000001320000003B
:10256A000000019700C4FFBCFF0200000000000049
:10257A0001320000000000013E00FDFFF4FF0119D6
:10258A0000FBFFFFFF011900FCFFFDFF011D00FD1D
:10259A00FFFBFF012900FEFFF8FF0124000200F9FA
:1025AA00FF0122000300FAFF0120000500FCFF01E1
:1025BA0020000600FEFF0123000700FFFF01410083
:1025CA000D000000012400FAFF0400011D00FDFFB8
:1025DA000500011B00FEFF0500011E00FFFF0600AB
:1025EA000123000100070001240002000700012066
:1025FA000004000500012700060005000126000767
:10260A00000300012B000800030001280008000154
:10261A0000012D0009000100013C000C00FFFF0130
:10262A0039000B00FDFF0138000A00FBFF012E00F4
:10263A000700FAFF0116000200FCFF011600020063
:10264A00FCFF0115000100FCFF0119000000FBFF5F
:10265A00011E000000FAFF012200FDFFFAFF01201F
:10266A0000FCFFFBFF012300FBFFFBFF0132000A16
:10267A000000000137000000F5FF017C01B4FF00F3
:10268A0000015A00EEFF0100011E00FAFF010001DD
:10269A001900FBFF0100012F00F8FF0500012E00C1
:1026AA00FAFF0700012D00FCFF0800013200FFFFBE
:1026BA000A000123000100070001190001000500BA
:1026CA00011B0002000500011D000300050001199D
:1026DA000004000300011D0005000300011E00069E
:1026EA0000010001230007000000010000000000B3
:1026FA000002010000000000013200000000000199
:10270A005A003500F6FF0200000000000001320006
:10271A0000000000012800F8FF0000012300F9FF73
:10272A00FFFF012000FAFFFEFF011D00FBFFFDFF76
:10273A00011500FDFFFDFF011500FDFFFDFF01155D
:10274A0000FFFFFCFF011500FFFFFCFF0115000160
:10275A0000FCFF0115000100FCFF0115000300FD4C
:10276A00FF0119000300FCFF011B000500FEFF0129
:10277A0020000600FEFF011E000600FFFF012800E0
:10278A000800000001280008000000011E000600E1
:10279A00010001200006000200011D0005000300DF
:1027AA0001150003000300011500030003000115D1
:1027BA00000100040001150001000400011500FFDA
:1027CA00FF0400011500FFFF0400011500FDFF03CF
:1027DA0000011500FDFF0300011D00FBFF030001BE
:1027EA001B00FBFF0200012300F9FF010001230087
:1027FA00F9FF0000010000000000000201000000D3
:10280A00000001320000000000019100CBFFBBFF75
:10281A000200000000000001320000000000013E3A
:10282A0000FDFFF4FF011900FBFFFFFF011900FC87
:10283A00FFFDFF012200FDFFFAFF012400FEFFF960
:10284A00FF0129000200F8FF011D000300FBFF0140
:10285A0020000500FCFF0122000600FDFF01230005
:10286A00070000000141000D00FFFF012700FAFFE9
:10287A000500011D00FDFF0500011B00FEFF05000C
:10288A00011E00FFFF0600012300010007000120CE
:10289A0000020006000124000400060001240006CC
:1028AA0000040001280007000400012B00080003AF
:1028BA000001280008000100012D000900010001A3
:1028CA003C000C00FFFF0139000B00FDFF0138003E
:1028DA000A00FBFF012E000700FAFF0116000200A2
:1028EA00FCFF0116000200FCFF0115000100FCFFBD
:1028FA000119000000FBFF011E000000FAFF01227F
:10290A0000FDFFFAFF012000FCFFFBFF012300FB93
:10291A00FFFBFF0132000A0000000137000000F54A
:10292A00FF017C01B4FF0000015A00EEFF01000123
:10293A001E00FAFF0100011900FBFF0100012F0030
:10294A00F8FF0500012A00FAFF0600013100FCFF2A
:10295A000900013200FFFF0A00011E000100060003
:10296A00011E0001000600011B00020005000119FA
:10297A000003000400011C0004000400011B000500
:10298A0000020001200006000200012300070000E7
:10299A000001000000000000020100000000000128
:1029AA00320000000000015A003500F6FF02000064
:1029BA000000000001320000000000012800F8FFBA
:1029CA000000012400F9FFFEFF011E00FAFFFFFFCD
:1029DA00011D00FBFFFDFF011500FDFFFDFF0115B5
:1029EA0000FDFFFDFF011500FFFFFCFF011500FFC1
:1029FA00FFFCFF0115000100FCFF0115000100FCAE
:102A0A00FF0119000300FCFF0115000300FDFF018F
:102A1A001B000500FEFF0120000600FEFF011E004C
:102A2A000600FFFF0128000800FFFF012800080038
:102A3A000100011E0006000100012000060002003C
:102A4A00011B000500020001190003000400011522
:102A5A000003000300011500010004000115000134
:102A6A00000400011500FFFF0400011500FFFF0428
:102A7A0000011500FDFF0300011500FDFF03000121
:102A8A001D00FBFF0300011900FBFF0100012400E8
:102A9A00F9FF0200012300F9FF0000010000000015
:102AAA0000000201000000000001320000000000E6
:102ABA00016F00F7FFBEFF020000000000000132B4
:102ACA000000000000014B000F00000001C30000DD
:102ADA0000D9FF014B00F1FF000001C300000027ED
:102AEA0000020100000000000132000000000001A5
:102AFA007B00DBFFC0FF0200000000000001320083
:102B0A000000000001370000000B000162027A0099
:102B1A000000013C000000F4FF01DC00D4FF0000CB
:102B2A000124000600FCFF011D000300FBFF011D3C
:102B3A00000300FBFF011E000000FAFF0123000052
:102B4A0000F9FF012200FDFFFAFF012400FCFFFA51
:102B5A00FF012000FBFFFCFF012800F9FFFCFF0139
:102B6A002900F8FFFEFF012900F8FFFEFF012D00F2
:102B7A00F7FFFFFF013700F5FF0100013300F6FF01
:102B8A000200012B00F8FF0300012800F9FF0400EE
:102B9A00012300FBFF0500012000FCFF05000120C6
:102BAA0000FEFF0600011E00FFFF0600011E0001D5
:102BBA0000060001200002000600012000040005B2
:102BCA000001240006000400013700F5FF0000029E
:102BDA0001000000000001320000000000014B006B
:102BEA002D00000002000000000000013200000079
:102BFA000000014600F2FFFFFF012F00F7FFFDFF73
:102C0A00011D00FBFFFDFF011C00FCFFFCFF01167C
:102C1A0000FEFFFCFF011900FFFFFBFF0115000189
:102C2A0000FCFF0110000100FDFF0119000300FC78
:102C3A00FF0119000400FDFF011B000500FEFF0152
:102C4A001B000500FEFF0123000700FFFF0128000B
:102C5A000800FFFF01280008000100012300070007
:102C6A000100011E0006000100011D00050003000D
:102C7A0001150003000300011500030003000116FB
:102C8A000002000400011400000004000114000006
:102C9A00000400011200FEFF0300011900FDFF04F9
:102CAA0000011500FDFF0300011D00FBFF030001E9
:102CBA001E00FAFF0100012400F9FF0200012300AF
:102CCA00F9FF0000010000000000000201000000FE
:102CDA00000001320000000000016900FFFFC1FF8F
:102CEA000200000000000001320000000000013C68
:102CFA00000C00FFFF0133000A00FEFF012D00084F
:102D0A0000FCFF012B000700FBFF0120000400FB71
:102D1A00FF011D000300FBFF0120000200FAFF0172
:102D2A0023000000F9FF0123000000F9FF0126003B
:102D3A00FDFFF9FF011D00FDFFFBFF012A00FAFF5D
:102D4A00FAFF012400FAFFFCFF012B00F8FFFDFF48
:102D5A00012E00F7FFFEFF013200F6FF0000014BD3
:102D6A0000F1FF0100011E00FAFF0100011B00FB38
:102D7A00FF0200013300F7FF0500013100F9FF07E8
:102D8A0000013100FCFF0900012D00FFFF090001CD
:102D9A0028000100080001200002000600012400AA
:102DAA0004000600012300050005000124000600B6
:102DBA000400012B00080003000133000A0002008E
:102DCA000132000A000100010000000000000201B7
:102DDA00000000000001320000000000011600009F
:102DEA0000F3FF02000000000000013200000000B2
:102DFA0000012800F8FF0000012400F9FFFEFF018E
:102E0A001E00FAFFFFFF011900FCFFFDFF01190078
:102E1A00FCFFFDFF011900FDFFFCFF011500FFFF8C
:102E2A00FCFF011900FFFFFBFF0115000100FCFF79
:102E3A000115000100FCFF0119000300FCFF011944
:102E4A00000400FDFF011D000500FDFF011B000538
:102E5A0000FEFF0128000800FFFF0128000800000B
:102E6A000001230007000000012300070001000100
:102E7A00200006000200011D0005000300011500E4
:102E8A0003000300011900030004000115000100FA
:102E9A00040001150001000400011900FFFF0500EC
:102EAA00011500FFFF0400011900FDFF04000115D0
:102EBA0000FDFF0300011D00FBFF0300011E00FAD5
:102ECA00FF0100012400F9FF0200012800F8FF00B9
:102EDA0000010000000000000201000000000001E3
:102EEA0032000000000001AB00E1FF9EFF0200007B
:102EFA000000000001320000000000014200F3FF60
:102F0A00FEFF012D00FFFF0900011E000000060060
:102F1A00011B000200050001150003000300011651
:102F2A000004000200012300070001000137000B22
:102F3A0000010001FF0033000000012D000000091C
:102F4A00000137000B000000012D000000F7FF010F
:102F5A006E0016000000014F000900F3FF019B00FC
:102F6A00E1FF0000013C000000F4FF013700F5FF1B
:102F7A000000013C0000000C00010401CCFF00002D
:102F8A00012800F8FF0000011500FDFFFDFF0115F3
:102F9A0000FFFFFCFF0119000000FBFF0100000019
:102FAA0000000002010000000000013200000000E1
:102FBA0000012200F3FFF0FF020000000000000100
:102FCA003200000000000155001100000001460017
:102FDA000000F2FF015500EFFF000001460000006B
:102FEA000E00020100000000000132000000000093
:102FFA000196002000ACFF02000000000000013230
:10300A000000000000013D00FEFFF4FF012300F96B
:10301A00FF0100012000FAFF0200012200FAFF036B
:10302A0000011C00FCFF0400011C00FCFF0400015D
:10303A001D00FDFF0500012000FEFF06000119002A
:10304A00000005000128000100080001200002001C
:10305A000600012400040006000123000500050003
:10306A0001240006000400012B0008000300012DC2
:10307A0000090001000137000B0001000141000DA9
:10308A0000FFFF013E000C00FDFF011B000500FED2
:10309A00FF0119000400FDFF0119000400FDFF01F2
:1030AA0019000300FCFF012D000400F8FF013200A3
:1030BA000100F6FF0119000000FBFF011E00FFFFDF
:1030CA00FAFF011900FDFFFCFF011900FDFFFCFFDB
:1030DA00011C00FCFFFCFF011D00FBFFFDFF011BA3
:1030EA0000FBFFFEFF012300F9FFFFFF013D00FE89
:1030FA00FF0C000129000800020001240006000458
:10310A0000011D0003000500011E00010006000168
:10311A00140000000400011600FEFF04000119005B
:10312A00FDFF0400011500FDFF0300011D00FBFF68
:10313A000300012000FAFF0200012300F9FF010049
:10314A00012800F8FF0000012800F8FF0000012311
:10315A0000F9FFFFFF012000FAFFFEFF011D00FB3F
:10316A00FFFDFF011500FDFFFDFF011500FDFFFD3D
:10317A00FF011500FFFFFCFF011500FFFFFCFF0127
:10318A0024000200F9FF0124000400FAFF011200E2
:10319A000300FEFF0116000400FEFF012E000900D5
:1031AA00FEFF010000000000000201000000000014
:1031BA00013200000000000124000C00EEFF0200B2
:1031CA00000000000001320000000000013C000C79
:1031DA0000FFFF0133000A00FEFF012D000800FC7A
:1031EA00FF012B000700FBFF0120000400FBFF0189
:1031FA001D000300FBFF0120000200FAFF0123006B
:10320A000000F9FF0123000000F9FF012600FDFF7D
:10321A00F9FF012200FDFFFAFF012700FAFFFBFF79
:10322A00012400FAFFFCFF012B00F8FFFDFF012E2D
:10323A0000F7FFFEFF013200F6FF0000014B00F12C
:10324A00FF0100011E00FAFF0100011B00FBFF0243
:10325A0000013300F7FF0500013100F9FF07000103
:10326A003100FCFF0900012D00FFFF0900012300C6
:10327A0001000700012400020007000124000400E5
:10328A0006000123000500050001240006000400D1
:10329A00012B00080003000133000A00020001327A
:1032AA00000A000100010000000000000201000005
:1032BA00000000013200000000000116000000F3C7
:1032CA00FF020000000000000132000000000001BF
:1032DA002800F8FFFFFF012300F9FFFFFF0120008C
:1032EA00FAFFFEFF011600FCFFFEFF011C00FCFFB7
:1032FA00FCFF011500FDFFFDFF011500FFFFFCFFAC
:10330A00011900FFFFFBFF0115000100FCFF011579
:10331A00000100FCFF0119000300FCFF0119000471
:10332A0000FDFF011D000500FDFF011B000500FE59
:10333A00FF0128000800FFFF0128000800FFFF0125
:10334A0023000700010001230007000100012000FB
:10335A0006000200011D000500030001150003001C
:10336A000300011900030004000115000100040014
:10337A0001150001000400011900FFFF05000115F5
:10338A0000FFFF0400011500FDFF0300011900FD05
:10339A00FF0400011B00FBFF0200012000FAFF02EC
:1033AA0000012300F9FF0100012800F8FF010001D4
:1033BA0000000000000002010000000000013200CD
:1033CA0000000000018B00D4FFB9FF0200000000DA
:1033DA0000000132000000000001B801580000009E
:1033EA000137000000F5FF013C00F4FF0000012452
:1033FA00000600FCFF0124000400FAFF012200037A
:10340A0000FAFF0123000100F9FF012300FFFFF981
:10341A00FF012200FDFFFAFF012300FBFFFBFF0172
:10342A002000FAFFFEFF012B000700FBFF01270027
:10343A000500FAFF0120000200FAFF011E00010048
:10344A00FAFF0119000000FBFF011900FFFFFBFF53
:10345A00011900FDFFFCFF011500FDFFFDFF011929
:10346A0000FCFFFDFF011B00FBFFFEFF011E00FA2F
:10347A00FFFFFF012300F9FF0000013101C3FF0034
:10348A0000013C0000000C00011801380000000196
:10349A00230007000100011E0006000100011000C0
:1034AA0003000100011500030003000116000200D9
:1034BA00040001140000000400010F0000000300D2
:1034CA00011500FFFF0400011200FEFF03000112B4
:1034DA0000FDFF0200011500FDFF0300011900FBBA
:1034EA00FF0100013D00F4FF020001FF00CDFF00D3
:1034FA0000013C0000000C00011D01390000000120
:10350A002D0009000100012000060002000112003E
:10351A0003000200010B0001000200011E0001006D
:10352A00060001190000000500011D00FDFF05004D
:10353A00011C00FCFF0400012000FAFF020001291F
:10354A0000F8FF0200013200F6FF000001E600D297
:10355A00FF000001410000000D0002010000000010
:10356A00000132000000000001ED05CB0089FC02D9
:10357A000000000000000132000000000001A40069
:10358A00F5FFE1FF01A100F7FFE1FF012201F1FFD1
:10359A00C8FF010501F5FFCDFF01DA00F9FFD5FFEC
:1035AA0001B100FBFFDDFF018700FEFFE5FF016EB1
:1035BA0000FEFFEAFF0201000000000001320000E5
:1035CA0000000001F8013E0028010200000000008E
:1035DA00000132000000000001800280FF000002AA
:1035EA0001000000000001320000000000010C028E
:1035FA00EC0030FF02000000000000013200000071
:10360A00000001AB00F7FF2100019500F6FF1C0046
:10361A00019600F5FF1C00019D00F4FF1D0001C08A
:10362A0000F0FF230001CE00ECFF2400016300F646
:10363A00FF1100016100F5FF1000016400F4FF10A2
:10364A0000016000F4FF0F00012A00FAFF060001E2
:10365A002700FAFF0500012400FAFF0400012000F8
:10366A00FAFF0200012000FAFF0200011E00FAFF21
:10367A000000013C00F4FF0000013D00F4FFFEFFE2
:10368A00014200F3FFFEFF014200F3FFFEFF014685
:10369A0000F2FF0000013700F5FF0000012D00F7DE
:1036AA00FFFFFF012B00F8FFFDFF012000FBFFFCDD
:1036BA00FF010E00FEFFFEFF010F000000FDFF01EB
:1036CA001000FFFFFDFF0115000100FCFF012D00A6
:1036DA000400F8FF0140000800F6FF012000040082
:1036EA00FBFF0124000200F9FF012E000200F7FF90
:1036FA00012D000000F7FF012D00FFFFF7FF012E4B
:10370A0000FEFFF7FF012800FCFFF9FF012700FB7D
:10371A00FFFAFF0201000000000001320000000071
:10372A0000019E02FF00C9FE020000000000000125
:10373A00320000000000011E000600000001150012
:10374A000400010001120003000200011600020039
:10375A000400011B00020005000119000100050018
:10376A00014600FFFF0E00014C00FEFF0F00014C56
:10377A0000FDFF0F00018E00FBFF1C00018F00FA05
:10378A00FF1C0002010000000000013200000000DE
:10379A0000012902E9FEB400020000000000000155
:1037AA00320000000000015D00EEFFFBFF01470050
:1037BA00F2FFFEFF013700F5FF0000012F00F7FFBF
:1037CA000300012700FAFF0500012700FBFF06009E
:1037DA00012600FDFF0700012E00FEFF0900015629
:1037EA0000FDFF1100012D00FFFF0900012900FE65
:1037FA00FF0800012600FDFF0700012000FCFF056D
:10380A0000012400FAFF0400012800F8FF0100016A
:10381A008A01EFFFB3FF011E000000FAFF01190041
:10382A000100FBFF0136000400F6FF013A00060022
:10383A00F6FF0136000600F7FF0160000C00F1FFF9
:10384A000128000400F9FF0120000200FAFF010B21
:10385A0000FFFFFEFF011000FFFFFDFF012E00F930
:10386A00FFFAFF018A00EBFFEEFF014B00F4FFF7BE
:10387A00FF014A00F6FFF5FF014300F7FFF6FF01DB
:10388A001D00FDFFFBFF011B00FEFFFBFF014B01BB
:10389A00F3FFBFFF010401F6FFCDFF011900050088
:1038AA0000000119000500010001160004000200D1
:1038BA000116000400020001350007000800013A61
:1038CA000006000A000194000C001B00015E0008BB
:1038DA0000110001600009001100011D000300052C
:1038EA0000011C00040004000144000B0008000150
:1038FA004A000D000700014A000E000500014700BA
:10390A000E00020001230007000000012300070047
:10391A00FFFF0120000600FEFF011D000500FDFF5C
:10392A000120000500FCFF0124000400FAFF013118
:10393A00000400F7FF013E000300F4FF014100010B
:10394A0000F3FF0146000000F2FF02010000000040
:10395A000001320000000000010A00060000000217
:10396A0000000000000001320000000000016600B3
:10397A001400040001510010000200013C000C0078
:10398A0000000133000A00FEFF012D000800FCFFC1
:10399A000132000800FAFF0135000800F9FF01436F
:1039AA00000900F6FF014E000A00F4FF014E000A6A
:1039BA0000F4FF019E001200E6FF0138012100CB4E
:1039CA00FF0155000800F1FF015C000900F0FF014A
:1039DA00BE000F00DDFF01BF000D00DCFF01B100DA
:1039EA000A00DEFF01F7000C00D0FF01F5000A0013
:1039FA00D0FF015A000100EEFF011E00FFFFFAFF8F
:103A0A00011500FFFFFCFF011200FEFFFDFF01127E
:103A1A0000FDFFFEFF011000FDFFFFFF011000FD8A
:103A2A00FF0100012E00F7FF0200012F00F7FF033C
:103A3A0000013900F5FF0300013200F6FF01000121
:103A4A003200F6FF0000012E00F7FF0200013100EC
:103A5A00F7FF0400013600F7FF0600013900F7FFFF
:103A6A000700013C00F8FF0900014300F7FF0A00C4
:103A7A00014400F8FF0B00018900F1FF17000192D1
:103A8A0000F1FF1900018B00F2FF1800018000F31A
:103A9A00FF160002010000000000013200000000D1
:103AAA0000019B01C4FFEF000200000000000001BA
:103ABA00320000000000015F00EDFF00000151002C
:103ACA00F0FFFEFF013D00F4FFFEFF013100F7FFAA
:103ADA00FCFF011500FDFFFDFF011500FDFFFDFFC5
:103AEA00011600FEFFFCFF011500FFFFFCFF013C71
:103AFA0000FFFFF4FF014C000200F1FF0156000332
:103B0A0000EFFF0161000400EDFF0162000500ED16
:103B1A00FF0165000700EDFF0165000900EEFF01E6
:103B2A0032000600F8FF0132000600F8FF013500F6
:103B3A000700F8FF0131000700F9FF013200080011
:103B4A00FAFF0133000900FBFF0201000000000038
:103B5A0001320000000000011D00F1FF090002000F
:103B6A0000000000000132000000000001FF00F622
:103B7A00FFCEFF015601F2FFBDFF02010000000067
:103B8A0000013200000000000186023D01DF000250
:103B9A000000000000000132000000000001930054
:103BAA00F7FFE4FF018200F9FFE7FF010701F3FFD6
:103BBA00CDFF019F00F9FFE1FF01C500FAFFD9FF20
:103BCA0001D400FAFFD6FF01DD00FCFFD4FF020199
:103BDA00000000000001320000000000018F01F720
:103BEA00FFEF0002000000000000013200000000A8
:103BFA0000017F000B00E9FF014600F2FFFFFF0111
:103C0A007D00F6FF17000141000D000100010000D0
:103C1A000000000002010000000000013200000064
:103C2A000000011700F2FF0000020000000000007F
:103C3A0001320000000000016A00FDFFEBFF017283
:103C4A00000900EBFF015D000500120002010000FF
:103C5A0000000001320000000000012700F4FF14F8
:103C6A000002000000000000013200000000000114
:103C7A004F01BDFFFFFF02010000000000013200FA
:103C8A0000000000016E004000EFFF02000000008B
:103C9A00000001320000000000010901CBFF000012
:103CAA000201000000000001320000000000016F64
:103CBA00003F00EBFF02000000000000013200009C
:103CCA0000000001FA00CEFF00000201000000001F
:103CDA0000013200000000000179003A002C0002C5
:103CEA000000000000000132000000000001F202A2
:103CFA001D009400020100000000000132000000D3
:103D0A000000010401D5FF6AFF0200000000000064
:103D1A000132000000000001F7021D0095000201B7
:103D2A00000000000001320000000000011D01FC3B
:103D3A00FF55FF02000000000000013200000000F1
:103D4A000001BF021B008A000201000000000001FE
:103D5A00320000000000012B0002001A00020000DD
:103D6A000000000001320000000000012800FFFFEF
:103D7A000800012400FEFF0700010700FFFF010001
:103D8A00010700FFFF0100010E00FEFFFEFF0128F0
:103D9A0000FCFFF9FF0201000000000001320000F0
:103DAA00000000011800F2FFFEFF02000000000000
:103DBA000001320000000000012400020007000197
:103DCA00150003000300010B00020001000141007D
:103DDA000D00000002010000000000013200000096
:103DEA00000001EF007AFF3300020000000000002B
:103DFA00013200000000000126000700FDFF012635
:103E0A00000700FDFF0132000800FAFF012E00073B
:103E1A0000FAFF0135000700F8FF0136000600F737
:103E2A00FF0136000600F7FF013A000600F6FF011F
:103E3A0038000500F6FF013B000400F5FF013900D8
:103E4A000300F5FF0133000200F6FF01370001000D
:103E5A00F5FF012D000000F7FF013200FFFFF6FF1A
:103E6A00012D00FCFFF8FF012600FDFFF9FF0123E9
:103E7A0000FBFFFBFF011D00FBFFFDFF012200FA13
:103E8A00FFFDFF011E00FAFFFFFF011E00FAFFFF00
:103E9A00FF011E00FAFF0100012300F9FF010001E2
:103EAA003F00F4FF0400014300F4FF06000139005B
:103EBA00F7FF0700013500F8FF07000201000000C4
:103ECA0000000132000000000001F30085003C0000
:103EDA00020000000000000132000000000001D6CC
:103EEA0000D7FFF4FF0201000000000001320000C9
:103EFA000000000140002500F5FF0200000000005C
:103F0A00000132000000000001C100DBFF0B0002CB
:103F1A0001000000000001320000000000016B00F7
:103F2A003F000C0002000000000000013200000007
:103F3A000000014001400000000136013E0000007F
:103F4A000176027E00FDFF014C000F00FEFF012DED
:103F5A00000900FFFF0110000300FFFF010B000131
:103F6A0000FEFF0110000100FDFF0119000000FB27
:103F7A00FF012800FFFFF8FF010B00FFFFFEFF0112
:103F8A000B00FEFFFFFF012D00F7FFFFFF015000AE
:103F9A00F0FFFFFF017B0281FF0100013B01C1FF2E
:103FAA000100014001C0FF0300010B00FEFF0100F8
:103FBA00010E00FEFF0200011500FFFF04000119B7
:103FCA0000000005000119000100050001150001AB
:103FDA0000040001120002000300011000030001A6
:103FEA0000010000000000000201000000000001C2
:103FFA003200000000000147001500DBFF0200004C
:10400A00000000000132000000000001BA00EFFFCA
:10401A00DFFF015900F8FFF0FF015E00F8FFEFFF34
:10402A000201000000000001320000000000016DE2
:10403A0000EBFFC2FF020000000000000132000096
:10404A00000000016200FBFFEDFF016000FEFFEDD2
:10405A00FF016000FEFFEDFF015F00FFFFEDFF01C2
:10406A00C3000100D9FF01B9000100DBFF02010012
:10407A000000000001320000000000015B01430063
:10408A00C50002000000000000013200000000002C
:10409A0001C800D8FFFFFF02010000000000013242
:1040AA000000000000015002EBFE22FF02000000A7
:1040BA000000000132000000000001280008000191
:1040CA000001260007000300012700060005000181
:1040DA0023000500050001550008000F00016200D9
:1040EA000800120001B6000D0022000201000000C3
:1040FA0000000132000000000001F20156001E011A
:10410A000200000000000001320000000000010C63
:10411A0001E8FF3000020100000000000132000047
:10412A000000000154002100DAFF02000000000034
:10413A00000132000000000001FF00EAFF2E000229
:10414A0001000000000001320000000000019B0095
:10415A00B4FFCAFF020000000000000132000000A4
:10416A000000011101E6FF3000020100000000001A
:10417A000132000000000001EC008A001F0002006A
:10418A00000000000001320000000000011C01E9EB
:10419A00FF340002010000000000013200000000AC
:1041AA0000017C00E6FFBAFF0200000000000001E7
:1041BA0032000000000001C201A6FF010002010056
:1041CA000000000001320000000000019C005C00B9
:1041DA00F0FF0200000000000001320000000000B1
:1041EA0001C701A5FF020002010000000000013220
:1041FA00000000000001E60068005B000200000009
:10420A000000000132000000000001BD01A7FF010B
:10421A00000201000000000001320000000000015D
:10422A0094005900FFFF0200000000000001320064
:10423A0000000000018C01F2FFB2FF020100000041
:10424A00000001320000000000017C001900460055
:10425A000200000000000001320000000000018797
:10426A0001F2FFB3FF02010000000000013200006A
:10427A0000000001CB00AAFF560002000000000067
:10428A000001320000000000018E01F0FFB2FF02BF
:10429A000100000000000132000000000001DD0002
:1042AA007400C0FF0200000000000001320000009C
:1042BA00000001BD01A7FF0100020100000000008B
:1042CA0001320000000000019B004B003700020091
:1042DA00000000000001320000000000014100F56A
:1042EA00FF07000201000000000001320000000088
:1042FA00000117000000F2FF0200000000000001A8
:10430A00320000000000014600FFFF0E000201001B
:10431A000000000001320000000000011900010045
:10432A00F1FF02000000000000013200000000005E
:10433A000144000B000800020100000000000132E5
:10434A00000000000001B60093FF01000200000017
:10435A0000000001320000000000013500070008DB
:10436A00000201000000000001320000000000010C
:10437A001B000200F0FF02000000000000013200F2
:10438A0000000000013900F7FF07000201000000E9
:10439A0000000132000000000001F2007B004D0025
:1043AA000200000000000001320000000000014489
:1043BA0000F5FF08000201000000000001320000C1
:1043CA0000000001A000A0FFF9FF020000000000A9
:1043DA000001320000000000018A01EFFFB3FF0272
:1043EA0001000000000001320000000000015C0032
:1043FA001A00CFFF02000000000000013200000096
:10440A000000011301E7FF31000201000000000073
:10441A0001320000000000016D002200C8FF020006
:10442A00000000000001320000000000013900F71E
:10443A00FF07000201000000000001320000000036
:10444A000001A4006200F9FF020000000000000160
:10445A00320000000000014E0007000E00020100B9
:10446A00000000000132000000000001D40086FFB5
:10447A0024000200000000000001320000000000D9
:10448A0001410000000D000201000000000001329D
:10449A000000000000017700080047000200000049
:1044AA00000000013200000000000131000700078F
:1044BA0000020100000000000132000000000001BB
:1044CA0043026200B3FE0200000000000001320055
:1044DA0000000000015101F2FFBEFF0201000000CE
:1044EA00000001320000000000016B0019003B00CF
:1044FA000200000000000001320000000000014B31
:10450A0001F3FFBFFF0201000000000001320000BA
:10451A000000000145002300160002000000000010
:10452A000001320000000000014B01F3FFBFFF024F
:10453A000100000000000132000000000001FD003F
:10454A009EFF74000200000000000001320000001B
:10455A000000015501F3FFBDFF0201000000000049
:10456A00013200000000000118000300F2FF0200FF
:10457A0000000000000132000000000001FB001AE8
:10458A0000D5FF0201000000000001320000000017
:10459A0000017B003000380002000000000000012A
:1045AA00320000000000018101B3FF010002010096
:1045BA0000000000013200000000000186004F00E8
:1045CA00F2FF0200000000000001320000000000BB
:1045DA00017C01B4FF00000201000000000001326A
:1045EA000000000000017F004C00000002000000F3
:1045FA000000000132000000000001F4001700D59D
:10460A00FF0201000000000001320000000000016A
:10461A005600F3FF320002000000000000013200E1
:10462A000000000001ED001600D6FF0201000000A4
:10463A0000000132000000000001C400ECFF740019
:10464A0002000000000000013200000000000181A9
:10465A0001B3FF0000020100000000000132000067
:10466A0000000001FD00580084FF02000000000065
:10467A000001320000000000016D01B7FF000002D6
:10468A000100000000000132000000000001E40007
:10469A00490074000200000000000001320000001E
:1046AA00000001ED001600D6FF0201000000000024
:1046BA0001320000000000015B00D3FFE1FF0200AD
:1046CA00000000000001320000000000013D000A65
:1046DA000007000201000000000001320000000093
:1046EA0000011600F4FF06000200000000000001AD
:1046FA003200000000000143000C00FAFF02010032
:10470A000000000001320000000000011700F4FF61
:10471A000700020000000000000132000000000053
:10472A000147000200F2FF0201000000000001320E
:10473A000000000000018500B1FF0D00020000002A
:10474A0000000001320000000000013E000300F4F6
:10475A00FF02010000000000013200000000000119
:10476A007F0004004C00020000000000000132003B
:10477A0000000000015001F3FFBEFF02010000002B
:10478A000000013200000000000102000000FFFFEB
:10479A000200000000000001320000000000014396
:1047AA00000900F6FF0201000000000001320000CB
:1047BA00000000011600F7FF0A00020000000000D6
:1047CA00000132000000000001240006000400027B
:1047DA0001000000000001320000000000010D008D
:1047EA00FAFFFBFF02000000000000013200000097
:1047FA0000000102011B00D4FF02010000000000BA
:10480A00013200000000000102000000FFFF020068
:10481A00000000000001320000000000013500081D
:10482A0000F9FF0201000000000001320000000050
:10483A000001CB00EBFF780002000000000000013D
:10484A0032000000000001200005000400020100FF
:10485A0000000000013200000000000182004E004A
:10486A000000020000000000000132000000000009
:10487A000141000B00F9FF020100000000000132B3
:10488A00000000000001C30001008BFF02000000CD
:10489A000000000132000000000001390008000891
:1048AA0000020100000000000132000000000001C7
:1048BA00AF0E3200CF0802010000000000013200F2
:1048CA0000000000020100000000000000000000DB
:1048DA000000E9CFE4FFEACFE4FFE652D9CFE6FFD2
:1048EA00DACFE6FFE1CFD9FFE2CFDAFFE6529EA0A8
:1048FA00DFD29E908E0ECE6ECF6815C62CF60601BC
:10490A002D6B0601010E2E6F060116511711181193
:10491A00191117E0D880000E06011655000E17551A
:10492A00190E1855000E195506E20601166B176B7B
:10493A00186B196B06D006011607000E175B185B79
:10494A00195B0601165117111811191102E0060117
:10495A002E6B0601000501E03DD106010D510E1135
:10496A000F11101107E1060111511211131114113F
:10497A0001E12FD10601C3510DE1060115A302D0B1
:10498A008C8E01D08C9E060115A702D08C8A01D08C
:10499A008C9A0FD00601C3050CE1060115A302D0BB
:1049AA008B8401D08B94060115A702D0898401D08B
:1049BA00899406010D510E110F11101164E0010EB8
:1049CA00E96E060EEA6E0E01B751EE240E01B76FBC
:1049DA000E01B851EE200E01B86F0E01B951EE204A
:1049EA000E01B96F0E01BA51EE200E01BA6FD880CE
:1049FA00000E0E01B755000EB855000EB955800EBF
:104A0A00BA5529E2B7CEB7FEB8CEB8FEB9CEB9FECE
:104A1A00BACEBAFE800E0E01BA5F010E06012C1143
:104A2A0006012C6F0601010E2D6F06010D07000EFF
:104A3A000E5B0F5B105B060115A307D00601240766
:104A4A00000E255B265B275B06D00601242B000E91
:104A5A0025232623272309C64CF00AC64DF04E6AA1
:104A6A004F6A4DAE02D04E684F684C50060101277E
:104A7A004D50060102234E50060103234F500601F2
:104A8A00042306012E6B0601115112111311141180
:104A9A0064E0050EE96E060EEA6E0E01BB51EE24C5
:104AAA000E01BB6F0E01BC51EE200E01BC6F0E0150
:104ABA00BD51EE200E01BD6F0E01BE51EE200E015A
:104ACA00BE6FD880000E0E01BB55000EBC55000EFD
:104ADA00BD55800EBE5529E2BBCEBBFEBCCEBCFE88
:104AEA00BDCEBDFEBECEBEFE800E0E01BE5F040E62
:104AFA0006012C1106012C6F0601010E2D6F06010D
:104B0A001107000E125B135B145B060115A707D091
:104B1A0006012807000E295B2A5B2B5B06D00601DB
:104B2A00282B000E29232A232B230BC64CF00CC654
:104B3A004DF04E6A4F6A4DAE02D04E684F684C50E7
:104B4A00060105274D50060106234E50060107238C
:104B5A004F500601082306012E6B06012D5139E03C
:104B6A000601C35107E106012CB18C8C06012CB554
:104B7A008C8809D00601C30506E106012CB18B8C8D
:104B8A0006012CB5898A0000000000000000000020
:104B9A00000000000000000000000000000000000B
:104BAA0000000000000000000000000000000000FB
:104BBA000000000000000000000000000601C351D0
:104BCA0003E18C9C8C9805D00601C30502E18B9CFD
:104BDA00899AD7D0030E0601005D01E0A0D0060134
:104BEA00D05101E179D006011D05DF6E06011A5187
:104BFA001B1137E1DF50EA6A310FE96E0E0EEA2225
:104C0A00EF500E01EA6AAC25E96EAD51EA22EF6A6D
:104C1A00EA6ADF34FE0BEA36E96E790EE9260E0EF1
:104C2A00EA22EE6AED6AEA6ADF34FE0BEA36E96ED8
:104C3A00490EE9260E0EEA22EE6AED6ADF50EA6AAA
:104C4A00310FE96E0E0EEA22EF6AEA6ADF34FE0BD2
:104C5A00EA36E96E010EE9260E0EEA22EE6AED6ADE
:104C6A003BD0EA6ADF34FE0BEA36E96E790EE926B2
:104C7A000E0EEA221EC6EEFF1FC6EDFFEA6ADF34F9
:104C8A00FE0BEA36E96E490EE9260E0EEA221AC62C
:104C9A00EEFF1BC6EDFFDF50EA6A310FE96E0E0E1A
:104CAA00EA221CC6EFFFEA6ADF34FE0BEA36E96E37
:104CBA00010EE9260E0EEA22EE50ED100DE1EA6A27
:104CCA00DF34FE0BEA36E96E010EE9260E0EEA2201
:104CDA001AC6EEFF1BC6EDFF0E01B65106011C5D9A
:104CEA001DE10E01B05106011A1904E10E01B1517C
:104CFA0006011B190AE10601010EC46F0601C06B09
:104D0A000601CF5101E08A9809D00601C46B060159
:104D1A00010EC06F0601CF5101E08A8832D0040E1D
:104D2A000601005D2EE10601205124E021C64CF067
:104D3A0022C64DF0D8904D324C32D8904D324C327A
:104D4A004C50BB6ECDC64EF0CEC64FF0040ED89076
:104D5A004E364F36E804FBE1300E4E16000E4F1663
:104D6A00CF0EBA1400014E104C6E4FC04DF04C508D
:104D7A00BA6E04D0BB6ACF0EBA14BA6E0601010E1F
:104D8A002E6F06012E5101E187D006011651171127
:104D9A001811191101E080D00601006B0601235198
:104DAA0076E130C600F631C601F632C602F633C6DF
:104DBA0003F634C604F635C605F636C606F637C611
:104DCA0007F638C608F639C609F63AC60AF63BC6E1
:104DDA000BF63CC60CF63DC60DF63EC60EF63FC6B1
:104DEA000FF640C610F641C611F642C612F643C681
:104DFA0013F644C614F645C615F646C616F647C651
:104E0A0017F648C618F649C619F64AC61AF64BC620
:104E1A001BF64CC61CF64DC61DF64EC61EF64FC6F0
:104E2A001FF650C620F651C621F652C622F60601D2
:104E3A00306B0601316B326B336B346B0601356BA9
:104E4A00366B376B386B06013D6B3E6B3F6B406BC5
:104E5A000601416B426B436B446B0601456B0601CD
:104E6A00466B476B486B496B06014A6B4B6B0601F5
:104E7A004C6B06014D6B06014E6B4F6B0601506B76
:104E8A000601516B526B0601010E236F05D0060114
:104E9A00166B176B186B196B8050800B06E00601B6
:104EAA00CB5106E08150010B03E10601010ECA6FE6
:104EBA00E552E552E5CFDAFFE7CFD9FFE552E5CF74
:104ECA00EAFFE5CFE9FF1100D9CFE6FFDACFE6FF27
:104EDA00E1CFD9FFE2CFDAFFE652DF6ADFCF00F097
:104EEA00020EE76E0018E8AE02D0E73402D0E750AF
:104EFA00005C37E2DFCFE9FFEA6AE9BEEA68D890E8
:104F0A00E936EA36D890E936EA36010EE926060E7F
:104F1A00EA22010EEE6EEE6AEE6AEE6ADFCFE9FF72
:104F2A00EA6AE9BEEA68D890E936EA36D890E936FC
:104F3A00EA360D0EE926060EEA22EE6AEE6AEE6AF5
:104F4A00EE6ADFCFE9FFEA6AE9BEEA68D890E93695
:104F5A00EA36090EE926060EEA22EE6AED6ADF2A29
:104F6A00BDD70601006B0601156B0601166B176BA0
:104F7A00186B196B06011A6B1B6B06011C6B060179
:104F8A001D6B06011E6B1F6B0601010E236FCD926E
:104F9A00CD9ECD9CCD8ACD98CD96CD948E0ECE6EDB
:104FAA00CF68CD809F809E909D8092809F9C010EAD
:104FBA00E66EE66AD7EC3EF0E552E552010EE66E81
:104FCA000B0EE66ED7EC3EF0E552E5528D849694D0
:104FDA008D829692898C929C8D8096908B829492E7
:104FEA008C9C959C8C9E959E8C9895988C9A959A5B
:104FFA00949E828E00000000000000000000000065
:10500A000000000000000000000000000000000096
:10501A0000000000000000000000948E829E06013D
:10502A00010ECF6F0601010ED06F8A989398060180
:10503A00010EC06F0601C36B0601010EC46F0601A3
:10504A00C96B0601C56BC66BC76BC86B0601CA6B19
:10505A009380F19E0601010ECB6F9396819610EC18
:10506A0033F0E552E552E5CFDAFFE7CFD9FF120078
:10507A0062EC33F0D9EC34F071EC34F029EC37F00F
:10508A00E66AD95015EC37F00701B45101E0B3D004
:10509A00DF0424E1E2EC34F00CE10601010ECF6FEB
:1050AA00D06BABEC34F002E2E16AE552E16E0050FB
:1050BA000DD048EC35F006E1ED5004E10601CF6B66
:1050CA00010E03D00601010ECF6FD06F000EE66EFF
:1050DA00E66AC4C6E6FF78EC35F08BD0020EDF5CD8
:1050EA002EE1E2EC34F009E10601C36B969094924A
:1050FA00959C959E9598959A1BD048EC35F00DE1B4
:10510A00ED500BE10601010E86EC35F09494929471
:10511A00949C929A959292926CD0FFEC36F0020E81
:10512A00EE1867E1ED5065E10601020E86EC35F0F6
:10513A0094849284948C928A958292825AD0040E94
:10514A00DF5C07E1010EDBCFB0FE020EDBCFB1FE62
:10515A0050D0050EDF5C07E1010EDBCFAEFE020E7A
:10516A00DBCFAFFE46D0080EDF5C0FE1FFEC36F076
:10517A00180ED880EE54000EED5403E2180E92EC8D
:10518A0035F0010EDBCFAAFE34D0090EDF5C0FE149
:10519A00FFEC36F0060ED880EE54000EED5403E212
:1051AA00060E92EC35F0010EDBCFABFE22D00A0ED2
:1051BA00DF5C03E199EC35F009D00B0EDF5C03E10B
:1051CA0099EC35F016D00C0EDF5C07E1010EDBCF4F
:1051DA00B4FE020EDBCFB5FE0CD00D0EDF5C09E18A
:1051EA00E2EC34F004E00601010ECB6F02D00601B6
:1051FA00CB6B3EEC3EF011EC37F071EF33F062EC22
:10520A0033F0200EE12402E3E168E65231EC36F095
:10521A004CEC35F0E66AD950040FE6EC33F096EC24
:10522A0036F0060FE6EC33F096EC36F0080F16EC83
:10523A0036F0E66AD9500C0F16EC36F0D950040F46
:10524A0034EC35F004E2580E006EB30E7BD2D9501E
:10525A00060F34EC35F004E22A0E006EB30E72D259
:10526A0026EC35F0040E005C000E015804E2000E34
:10527A00006EB30E67D2060EDBCF00F0070EDBCF4F
:10528A0001F0040E005C000E015804E2D80E006E14
:10529A00B20E58D20701B45101E05DD2080EDBCF3D
:1052AA0010F0090EDBCF11F00A0EDBCF12F00B0E55
:1052BA00DBCF13F010C038F011C039F012C03AF049
:1052CA0013C03BF0080EDBCF3DF0090EDBCF3EF0FA
:1052DA000A0EDBCF3FF00B0EDBCF40F047EC64F059
:1052EA0034C00CF035C00DF036C00EF037C00FF0E8
:1052FA000C0EDBCF14F00D0EDBCF15F00E0EDBCF4C
:10530A0016F00F0EDBCF17F014C038F015C039F0C5
:10531A0016C03AF017C03BF00C0EDBCF3DF00D0E75
:10532A00DBCF3EF00E0EDBCF3FF00F0EDBCF40F0AF
:10533A0047EC64F00C503424086E0D503520096E89
:10534A000E5036200A6E0F5037200B6E2DEC35F0BA
:10535A003B6E3AEC55F00AEC34F039C0E6FF3AC03D
:10536A00E6FF3BC0E6FF3CC0E6FFB7EC5AF011ECA3
:10537A0037F0E552B7EC36F038C039F0D9EC36F0F0
:10538A00AAEC56F0140E38C0DBFF150E39C0DBFF4D
:10539A00160E3AC0DBFF170E3BC0DBFF0601235196
:1053AA00FDE0466B476B486B496B456B8D908B9262
:1053BA00D950080FE96E000E61EC34F002E668EC91
:1053CA0034F006E2020E456FDFEC35F02DEC34F0D6
:1053DA00D9500C0FE96E000E61EC34F002E668EC6D
:1053EA0034F012E2080E06014511456F0C0EDBCFB0
:1053FA0038F00D0EDBCF39F00E0EDBCF3AF00F0E80
:10540A00A6EC33F03AEC34F0EBEC35F002E6B8EC0B
:10541A0033F004E2AA0E006EB20E94D1F7EC35F026
:10542A0002E6B8EC33F004E27C0E006EB20E8AD1CA
:10543A00E6EC34F00AEC34F0AC0E3E6EC50E3F6E6C
:10544A00A70E406E470E416EA6EC55F03BEC35F0C8
:10545A00DBCF0CF0150EDBCF0DF0160EDBCF0EF006
:10546A00170EDBCF0FF00CC038F00DC039F00EC0AC
:10547A003AF00FC03BF038EC55F055EC35F09EECA5
:10548A0033F053EC55F0180E39C0DBFF190E3AC051
:10549A00DBFF1A0E3BC0DBFF1B0E3CC0DBFFFFEC41
:1054AA0034F0080EDBCF08F0090EDBCF09F00A0E44
:1054BA00DBCF0AF00B0E1AEC36F038C031F639C0E1
:1054CA0032F63AC033F63BC034F6080EDBCF3DF66F
:1054DA00090EDBCF3EF60A0EDBCF3FF60B0EDBCF13
:1054EA0040F65EEC35F055EC35F05EEC35F039C03F
:1054FA000CF03AC00DF03BC00EF03CC00FF0CDEC02
:10550A0035F008C039F009C03AF00AC03BF00BC0C8
:10551A003CF0A6EC55F00AEC34F0E6EC34F039C075
:10552A0014F03AC015F03BC016F03CC017F0E6EC98
:10553A0034F039C018F03AC019F03BC01AF03CC038
:10554A001BF0CDEC35F014C039F015C03AF016C096
:10555A003BF017C03CF0A6EC55F039C010F03AC049
:10556A0011F03BC012F03CC013F0CDEC35F004C092
:10557A0039F005C03AF006C03BF007C03CF013EC26
:10558A0056F03BEC35F0DBCF28F0150EDBCF29F0D7
:10559A00160EDBCF2AF0170EDBCF2BF028C038F01F
:1055AA0029C039F02AC03AF02BC03BF038EC55F04C
:1055BA0039C024F03AC025F03BC026F03CC027F0A1
:1055CA00140EDBCF30F0150EDBCF31F0160EDBCF29
:1055DA0032F0170EDBCF33F030C038F031C039F07B
:1055EA0032C03AF033C03BF038EC55F039C02CF0F9
:1055FA003AC02DF03BC02EF03CC02FF0CDEC35F078
:10560A0024C039F025C03AF026C03BF027C03CF050
:10561A00A6EC55F039C020F03AC021F03BC022F088
:10562A003CC023F03E6A3F6A406A400E416EA6ECD7
:10563A0055F039C01CF03AC01DF03BC01EF03CC00A
:10564A001FF09EEC33F053EC55F01C0E39C0DBFF13
:10565A001D0E3AC0DBFF1E0E3BC0DBFF1F0E3CC017
:10566A00DBFF080EDBCF04F0090EDBCF05F00A0ED4
:10567A00DBCF06F00B0E77EC33F038C039F639C0C1
:10568A003AF6FFEC34F00C0EDBCF08F00D0EDBCF50
:10569A0009F00E0EDBCF0AF00F0E1AEC36F038C006
:1056AA0035F639C036F63AC037F63BC038F60C0E36
:1056BA00DBCF41F60D0EDBCF42F60E0EDBCF43F603
:1056CA000F0EDBCF44F6C2EC35F077EC33F038C07E
:1056DA003BF639C03CF626EC35F0060EDB500018D6
:1056EA0003E1070EDB50011812E0060139513A11A5
:1056FA000EE1D880000E3D55000E3E55000E3F5576
:10570A00000E405504E2510E006EB20E1BD026EC7C
:10571A0035F0060EDB50001803E1070EDB500118C6
:10572A0014E006013B513C1110E1D880000E4155AE
:10573A00000E4255000E4355000E445506E2260E51
:10574A00006EB20E36EC36F006D00601010E306F4E
:10575A00236B3EEC3EF0200EE15C02E2E16AE55288
:10576A00E16E71EF33F062EC33F0100EE12402E3E4
:10577A00E168E65231EC36F071EC34F096EC36F032
:10578A00040F16EC36F08EEC35F0080F16EC36F0F6
:10579A000E01BF516FE0A3EC33F002E10701B48DB3
:1057AA000701B45173E1EEEC34F004E2F30E006E3B
:1057BA00B10E5DD03EEC36F002E628EC34F005E29C
:1057CA00D950040F8AEC34F004D04AEC36F03AECA3
:1057DA0034F0F7EC35F002E6B8EC33F004E2AA0E46
:1057EA00006EB20E44D056EC36F004E2C30E006EE0
:1057FA00B10E3DD023EC33F00C0FC2EC33F009E3C9
:10580A00C2EC35F013EC34F004E09D0E006EB10EDC
:10581A002ED0EBEC35F002E628EC34F005E2D95054
:10582A00080F8AEC34F004D0DFEC35F03AEC34F0AF
:10583A00F7EC35F002E6B8EC33F004E27C0E006EC9
:10584A00B20E15D056EC36F004E26D0E006EB10EB3
:10585A000ED023EC33F00C0FC2EC33F00BE3C2ECA6
:10586A0035F013EC34F006E0470E006EB10E36EC5C
:10587A0036F00CD027EC36F002E2E16AE552E16E2E
:10588A0000500701E35102E03EEC3EF0100EE15CED
:10589A0002E2E16AE552E16E71EF33F062EC33F055
:1058AA00180EE12402E3E168E65231EC36F04CECE2
:1058BA0035F0140EDB6A150EDB6A160EDB6A170E5C
:1058CA00DB6A71EC34F096EC36F00C0F16EC36F01D
:1058DA00E66AD950100F16EC36F0A3EC33F002E169
:1058EA000701B48D100EDBCF00F0110EDBCF01F0F3
:1058FA00120EDBCF02F0130EDBCF03F0D9500C0FE0
:10590A00BDEC35F0EE500026EE500122EE50022298
:10591A00EE500322040E00C0DBFF050E01C0DBFFC0
:10592A00060E02C0DBFF070E03C0DBFFC2EC35F038
:10593A00DBCF07F0D950100FBDEC35F0EE50045C08
:10594A00006EEE500558016EEE500658026EEE508B
:10595A000758036E080E00C0DBFF090E01C0DBFF0B
:10596A000A0E02C0DBFF0B0E03C0DBFF3EEC36F073
:10597A0002E628EC34F005E2D950040F98EC34F032
:10598A0004D04AEC36F00CEC35F0EEEC34F004E2DC
:10599A00F30E006EB10E4AD062EC36F002E6B8ECB5
:1059AA0033F004E2AA0E006EB20E40D06EEC36F06E
:1059BA0004E2C30E006EB10E39D023EC33F0140F9B
:1059CA00C2EC33F007E37AEC36F004E09D0E006E89
:1059DA00B10E2CD0EBEC35F002E628EC34F005E2FF
:1059EA00D950080F98EC34F004D0DFEC35F00CEC09
:1059FA0035F062EC36F002E6B8EC33F004E27C0EE5
:105A0A00006EB20E13D06EEC36F004E26D0E006E2C
:105A1A00B10E0CD023EC33F0140FC2EC33F009E3CF
:105A2A007AEC36F006E0470E006EB10E36EC36F030
:105A3A000CD00701B45109E127EC36F002E2E16A21
:105A4A00E552E16E00503EEC3EF0180EE15C02E2D7
:105A5A00E16AE552E16E71EF33F062EC33F0330E36
:105A6A00E12402E3E168E65231EC36F0CCEC33F0A3
:105A7A0024EC37F017E186EC36F014E1020EF36EEF
:105A8A00100EF3CFDBFFEBEC33F0260E34C0DBFF56
:105A9A00270E35C0DBFF280E36C0DBFF290E37C0C4
:105AAA00DBFF72D1260EDB6A270EDB6A280EDB6A61
:105ABA00290EDB6A250EDB6A8D908B92D950F60F80
:105ACA00D5EC36F002E668EC34F01FE2250EDB5026
:105ADA000209E76E250EE7CFDBFFF60EDBCF38F0C3
:105AEA00F70EDBCF39F0F80EDBCF3AF0F90EA6EC61
:105AFA0033F0F60E34C0DBFFF70E35C0DBFFF80ECD
:105B0A0036C0DBFFF90E37C0DBFFD950F20FD5ECF8
:105B1A0036F002E668EC34F01FE2250EDB50080985
:105B2A00E76E250EE7CFDBFFF20EDBCF38F0F30E80
:105B3A00DBCF39F0F40EDBCF3AF0F50EA6EC33F0FA
:105B4A00F20E34C0DBFFF30E35C0DBFFF40E36C0B5
:105B5A00DBFFF50E37C0DBFFD950F60FD5EC36F078
:105B6A0002E666EC35F030E2EBEC33F0040E34C0BA
:105B7A00DBFF050E35C0DBFF060E36C0DBFF070E66
:105B8A0037C0DBFFCCEC33F00F0E1F0B03E0D9EC70
:105B9A0033F0FDE130EC33F0FFEC33F0CCEC33F0D2
:105BAA000F0E1F0B03E0D9EC33F0FDE1E0EC36F009
:105BBA0014E2BAEC34F003E0D9EC33F0FDE130EC56
:105BCA0033F019EC35F009D0CCEC33F01AEC34F0A0
:105BDA00A0EC35F0FDE10DEC36F0F9EC34F00CE216
:105BEA00AEEC33F0120E006EB10E9BEC36F002E210
:105BFA00E16AE5523EEC35F0A3EC33F012E1F60E21
:105C0A00DBCF04F0F70EDBCF05F0F80EDBCF06F0A2
:105C1A00F90E13EC34F005E0E70E006EB00E1AEC44
:105C2A0037F0B0EC33F009E2C9EC34F003E0A7EC4A
:105C3A0035F0FDE174EC34F006D0D5EC34F003E035
:105C4A00D9EC33F0FDE19EEC34F0110EEECFDBFF20
:105C5A00120EEECFDBFF130EEECFDBFF140EEECFEC
:105C6A00DBFFD950F60FF1EC36F01D0EEECFDBFF5D
:105C7A001E0EEECFDBFF1F0EEECFDBFF200EEECFA8
:105C8A00DBFF190EDB6A1A0EDB6AD950F20FD5EC6C
:105C9A0036F002E666EC35F022E247EC34F00F0EFD
:105CAA001F0B03E0D9EC33F0FDE130EC33F0FFECED
:105CBA0033F047EC34F00F0E1F0B03E0D9EC33F04E
:105CCA00FDE1E0EC36F014E2BAEC34F003E0D9EC92
:105CDA0033F0FDE130EC33F019EC35F009D047EC44
:105CEA0034F01AEC34F0A0EC35F0FDE10DEC36F0AE
:105CFA00F9EC34F00CE2AEEC33F0B20E006EB00EFA
:105D0A009BEC36F002E2E16AE5523EEC35F0A3EC98
:105D1A0033F008E186EC36F005E0870E006EB00E2F
:105D2A001AEC37F0B0EC33F009E2C9EC34F003E0D6
:105D3A00A7EC35F0FDE174EC34F006D0D5EC34F084
:105D4A0003E0D9EC33F0FDE19EEC34F0A4EC36F03C
:105D5A00180EEECFDBFFD950F20FF1EC36F0210E20
:105D6A00EECFDBFF220EEECFDBFF230EEECFDBFF03
:105D7A00240EEECFDBFF1B0EDB6A1C0EDB6A010E64
:105D8A00F36E100EF3CFDBFF06012351FDE0100E78
:105D9A00DBCF30F6110EDBCF31F6120EDBCF32F647
:105DAA00130EDBCF33F6140EDBCF34F6150EDBCF32
:105DBA0035F6160EDBCF36F6170EDBCF37F6180E92
:105DCA00DBCF38F6190EDBCF39F61A0EDBCF3AF6EF
:105DDA001B0EDBCF3BF61C0EDBCF3CF61D0EDBCFDA
:105DEA003DF61E0EDBCF3EF61F0EDBCF3FF6200E32
:105DFA00DBCF40F6210EDBCF41F6220EDBCF42F697
:105E0A00230EDBCF43F6240EDBCF44F6250EDBCF81
:105E1A0045F6260EDBCF46F6270EDBCF47F6280ED1
:105E2A00DBCF48F6290EDBCF49F62A0EDBCF4AF63E
:105E3A002B0EDBCF4BF62C0EDBCF4CF62D0EDBCF29
:105E4A004DF62E0EDBCF4EF62F0EDBCF4FF6300E71
:105E5A00DBCF50F6310EDBCF51F6320EDBCF52F6E6
:105E6A00236B330EE15C02E2E16AE552E16E71EF07
:105E7A0033F062EC33F0110EE12402E3E168E652FA
:105E8A006FEC35F04FEC33F0100EDB6A060123514C
:105E9A0002E1300502E0000502E1010EDF6E300585
:105EAA0027E1306B090E3DC6DBFF0A0E3EC6DBFF5B
:105EBA000B0E3FC6DBFF0C0E40C6DBFF0D0E41C6C4
:105ECA00DBFF0E0E42C6DBFF0F0E43C6DBFF100ED2
:105EDA0044C6DBFF3D6B3E6B3F6B406B416B426BD5
:105EEA00436B446B396B3A6B3B6B3C6B010E236F14
:105EFA00000525E1006B010E0DC6DBFF020E0EC682
:105F0A00DBFF030E0FC6DBFF040E10C6DBFF050E18
:105F1A0011C6DBFF060E12C6DBFF070E13C6DBFF38
:105F2A00080E14C6DBFF0D6B0E6B0F6B106B116B3B
:105F3A00126B136B146B096B0A6B0B6B0C6BD950DE
:105F4A00050FB9DBD950010FB6DBD9500D0FB3DB02
:105F5A00D950090FB0DBDFCFE6FFE66A720E006E9A
:105F6A00B00EB1DB036E150EE15C02E2E16AE552A6
:105F7A0082EC35F0110EE15C02E2E16AE552E16E73
:105F8A00ABD3C4C600F0016A00BE0168AEEC35F0BE
:105F9A006D0E026EB00E54EC34F002E2E16AE55284
:105FAA00E16E05503EEF3EF092EC36F0DE6ADD6AB5
:105FBA00010EE66EF6EC36F0030E3ADB0701B45139
:105FCA000FE10601C40504E1B3EC35F0E66A04D03A
:105FDA00B3EC35F0010EE66E78EC35F03EEC3EF0AF
:105FEA00E552E55279D392EC36F0D9EC34F07CECF8
:105FFA0035F039EC36F0C0EC36F0B8EC35F0070184
:10600A00B45129E1030EDB50070802E27CEC35F0BB
:10601A00DF50010802E2010EDF6E030EDB50030FB0
:10602A000E01B65D0CE0ABEC34F002E2E16AE55237
:10603A00E16E0050030EDB50030F0E01B66F010E26
:10604A00DBCFE6FF020EDBCFE6FFDFCFE6FF78EC21
:10605A0035F03EEC3EF0050EE15C02E2E16AE55203
:10606A00E16E3AD392EC36F0E652E652FD0EDB04CC
:10607A000BE1B0CEDEFFB1CEDDFF020EB2CEDBFF0A
:10608A00030EB3CEDBFF0AD0AECEDEFFAFCEDDFF0E
:10609A00020EB4CEDBFF030EB5CEDBFFFB0EDBCF69
:1060AA00E6FFFC0EDBCFE6FF020EDBCFE6FF030EB8
:1060BA00DBCFE6FFB6CEE6FFB3EC35F0A2EC5FF03D
:1060CA00006E070EE15C02E2E16AE552E16E005001
:1060DA00040EE15C02E2E16AE552E16EFDD292EC65
:1060EA0036F0E65271EC34F0C5EC36F039E10701CE
:1060FA00B45156E10601C35103E0020EC35D28E123
:10610A00DF50000821E2C35101E18D90DF0403E171
:10611A008D848D82898C020EDF5C03E18D848D82F1
:10612A00899C030EDF5C03E18D948D82899C040EA9
:10613A00DF5C03E18D848D92899C050EDF5C10E1A2
:10614A008D948D92899C0CD0C3510AE18D8008D020
:10615A00C30506E1DF50000802E28C9201D08C826E
:10616A008EEC35F0010F2DDBC5EC36F017E1070197
:10617A00B45116E10601C35108E1010EDB500008D3
:10618A0002E28B920BD08B8209D0C30507E1010E84
:10619A00DB50000802E2899201D089823EEC3EF08F
:1061AA0011EC37F099D2FE0E0601C55DFF0EC659F5
:1061BA00FF0EC759FF0EC85905E2C52B000EC623AC
:1061CA00C723C8233EEF3EF00601C551C611C711C9
:1061DA00C81105E0C507000EC65BC75BC85B3EEF8A
:1061EA003EF092EC36F0E652E652E65275DB070EC6
:1061FA001FDAB8EC35F0DB500BE1DFCFC5F6010E44
:10620A00DBCFC6F6020EDBCFC7F6030EDBCFC8F62E
:10621A003EEC3EF0050EE15C02E2E16AE552E16E17
:10622A005BD2C5C6E6FFC6C6E6FFC7C6E6FFC8C656
:10623A00E6FF640E006EB00E9BEC36F002E2E16AF5
:10624A00E55282EF35F0E66AC90EE66E060EE66E94
:10625A0029EC37F00701B45101E012003EEF3EF09D
:10626A00C9C600F0016A00BE0168AEEC35F05D0EE9
:10627A00026EB00E14DB02E2E16AE552E16E0550ED
:10628A003EEF3EF0CAC600F0016A00BE0168AEECFD
:10629A0035F0570E026EB00E02DB02E2E16AE552F9
:1062AA00E16E05500601CA6B3EEF3EF09DBCFED77B
:1062BA0016C1E6FF17C1E6FF00C1E6FF01C1E6FF0E
:1062CA004B0E006EB00E9BEC36F002E2E16AE5522C
:1062DA0082EF35F092EC36F067DB030EDB6A39ECBD
:1062EA0036F0B8EC35F0C0EC36F00701B45101E0F5
:1062FA0080D0FFEC36F0FF0ED880EE54030EED543A
:10630A0007E2010EDB68030EF36E020EF3CFDBFF2A
:10631A00DF50010802E2010EDF6E030EDB500108B6
:10632A0001E2E5DBDF0409E1040EDB50030805E1C5
:10633A000601CD6B020ECE6F06D0010EDBCFCDF675
:10634A00020EDBCFCEF6CAB415D0CB68FC0ECA1447
:10635A000009CA6E9D920F0152815293F00EBA142F
:10636A000C09BA6E3F0EBA140009BA6E0E010E0E6F
:10637A00CC6FCA84030EDB502AE1DF5023E0CDC67E
:10638A0000F0CEC601F0D89001320032D890013226
:10639A0000320050BB6ECDC602F0CEC603F0040E2A
:1063AA00D89002360336E804FBE1300E0216000EDE
:1063BA000316CF0EBA1400010210006E03C001F0DA
:1063CA00E85003D0BB6ACF0EBA14BA6E10D00601D9
:1063DA002351FDE0CDC651F6CEC652F6466B476B49
:1063EA00486B496BDFCF50F6040E306F236B3EECDF
:1063FA003EF0050EE15C02E2E16AE552E16E6CD123
:10640A0012005BD9270EE12402E3E168E65262DB5F
:10641A00F29E040E00C6DBFF050E01C6DBFF060E68
:10642A0002C6DBFF070E03C6DBFF080E04C6DBFF4E
:10643A00090E05C6DBFF0A0E06C6DBFF0B0E07C6F2
:10644A00DBFF0C0E08C6DBFF0D0E09C6DBFF0E0EC6
:10645A000AC6DBFF0F0E0BC6DBFF100E0CC6DBFFF6
:10646A00110E0DC6DBFF120E0EC6DBFF130E0FC692
:10647A00DBFF140E10C6DBFF150E11C6DBFF160E6E
:10648A0012C6DBFF170E13C6DBFF180E14C6DBFF9E
:10649A00190E15C6DBFF1A0E16C6DBFF1B0E17C632
:1064AA00DBFF1C0E18C6DBFF1D0E19C6DBFF1E0E16
:1064BA001AC6DBFF1F0E1BC6DBFF200E1CC6DBFF46
:1064CA00210E1DC6DBFF220E1EC6DBFF230E1FC6D2
:1064DA00DBFF240E20C6DBFF250E21C6DBFF260EBE
:1064EA0022C6DBFFF28E1A0EDBCF00F01B0EDBCFCB
:1064FA0001F01C0EDBCF02F01D0EA0EC36F002E01C
:10650A00010EDF6E040EDB5002E0010EDF6E0601A3
:10651A00235106E1010EDF6EF36E030EF3CFDBFFAC
:10652A00DF5010E0110EDBCF00F0120EDBCF01F0CE
:10653A00130EDBCF02F0140EA0EC36F003E0DE52AD
:10654A00010EDD6EDF5011E0150EDBCF00F0160EE6
:10655A00DBCF01F0170EDBCF02F0180EECDB05E003
:10656A00010EF36E020EF3CFDBFF030EDBCFE6FF65
:10657A00E66A020EDBCFE6FFE66A010EDBCFE6FF34
:10658A00E66ADFCFE6FFE66A3A0E006EB00E9BD8E7
:10659A00036E0B0EE15C02E2E16AE552E16E035022
:1065AA00270EE15C02E2E16AE552E16E95D085D8F8
:1065BA00080EE12402E3E168E652E16EF29E24C687
:1065CA00DFFF010E25C6DBFF020E26C6DBFF030E28
:1065DA0027C6DBFF040E28C6DBFF050E29C6DBFF34
:1065EA00060E2AC6DBFF070E2BC6DBFFF28E1FEC58
:1065FA0037F0300E006EB00E66D8036E0B0EE15CFB
:10660A0002E2E16AE55279DA080EE15C02E2E16A45
:10661A00E552E16E61D0F29E0601246B256B266B72
:10662A00276B286B296B2A6B2B6BF28E3EEF3EF0A1
:10663A00E66E9DEC43F0F0DBE5521200DFDA1F0E46
:10664A003D6E050E3E6E3F6A406AABDAA5EC64F019
:10665A0089DBD9501200A5DA040EDBCF3DF0050E16
:10666A00DBCF3EF0060EDBCF3FF0070EFBEF36F036
:10667A00DBCF03F096DADFCF3DF0010EDBCF3EF041
:10668A00020EDBCF3FF0030EB1DBD880190E38546F
:10669A00E4EF36F0040EDB6A050EDB6A060EDB6AEF
:1066AA00070EDB6A080EDB6A090EDB6A0A0EDB6A72
:1066BA000B0EDB6AA8D35CDA4CD393DBE1CFD9FFAC
:1066CA00E2CFDAFF1200016E026A00C0E6FFE66E50
:1066DA0002C0E6FF71EF63F0E552E5CFDAFFE7CFDC
:1066EA00D9FF1200DBCF07F004C038F005C039F03B
:1066FA0006C03AF007C03BF03AEC55F01C0EDBCF6F
:10670A003EF01D0EDBCF3FF01E0EDBCF40F01F0E1A
:10671A00DBCF41F0A6EC55F03ADB210E3E6EE60ED9
:10672A003F6E5B0E406E400E416EA6EC55F0AAEF2E
:10673A0056F02EDA00C039F0D9EF36F05FDA24EFDE
:10674A0037F0DBCF3BF03D683E683F68406847EF73
:10675A0064F054DBFED2D950FA0F3EDBD8801E0E0D
:10676A00EE54000E33D3D880FF0E3954FF0E3A543C
:10677A00FF0E3B54000E3C541200FAD9EE50385C1E
:10678A00EE503958EE503A58EE503B581200F60E79
:10679A00DBCF00F0F70EDBCF01F0F80EDBCF02F013
:1067AA00F90EDBCF03F01200D8900036013602361C
:1067BA000336E8061200DBCF3CF03C34000E3C18EE
:1067CA001200E66E000EDA20E66E1200FA0EDBCF39
:1067DA0000F0FB0EDBCF01F0FC0EDBCF02F0FD0E6A
:1067EA00DBCF03F0190E3D6E3E6A3F6A406AD9D983
:1067FA0047EF64F038C0DEFF39C0DEFF3AC0DEFF83
:10680A003BC0DDFFDD52DD52120039C004F03AC050
:10681A0005F03BC006F03CC007F01200DBCF07F0E2
:10682A0004500510061007101200BBD9FA0EDBCF70
:10683A003DF0FB0EDBCF3EF0FC0EDBCF3FF0FD0E52
:10684A00D5DA0F0E1200D880BADA000E3C541200C4
:10685A00080E34C0DBFF090E35C0DBFF0A0E36C056
:10686A00DBFF0B0E37C0DBFF12000C0E34C0DBFF60
:10687A000D0E35C0DBFF0E0E36C0DBFF0F0E37C024
:10688A00DBFF1200F20EDBCF00F0F30EDBCF01F0DC
:10689A00F40EDBCF02F0F50EDBCF03F01200036E2D
:1068AA00046A02C0E6FFE66E04C0E6FF71EC63F01C
:1068BA00056E050EE15C1200DA20EA6ED890030E2E
:1068CA00EB50000A1200000EEE5C000EEE58000EAD
:1068DA00EE58000EEE581200E66AF6EF36F0D9507E
:1068EA000C0F46D90450EE24006E0550EE20016EBE
:1068FA000650EE20026E0750EE20036E1200DE6A8A
:10690A00DE6ADD6ADD52DD52120032D90C0EEECF9C
:10691A00DBFF0D0EEECFDBFF0E0EEECFDBFF0F0E11
:10692A00EECFDBFF120024D9140EEECFDBFFA4EF6B
:10693A0036F000C0DFFF010E01C0DBFF020E02C00D
:10694A00DBFF030E03C0DBFF03EF37F0000EE66E3A
:10695A00E66AE66EE66AB6CEE6FFE66EE66AA2EC9E
:10696A005FF0006E070EE15C1200080EDBCF00F04C
:10697A00090EDBCF01F00A0EDBCF02F00B0EDBCFE4
:10698A0003F0100E1F0B120039DAEECF04F0EECF2F
:10699A0005F0EECF06F0EFCF07F0100E1F0B120036
:1069AA002DD9100E1F0B1200E652E652E652DF6A8C
:1069BA00010EDB6A020EDB6A12001CDAEE50ED10E1
:1069CA001200040EDBCF3AF0050EDBCF3BF023EFCB
:1069DA0055F014DAD880FF0EEE54FF0EEE54FF0E77
:1069EA00EE54000EEE54120009DAD880000EEE546E
:1069FA00800EECD1180EDBCF00F0190EDBCF01F0C0
:106A0A001A0EDBCF02F01B0EDBCF03F01200140EBE
:106A1A0034C0DBFF150E35C0DBFF160E36C0DBFFB8
:106A2A00170E37C0DBFF12000C0E38C0DBFF0D0E4D
:106A3A0039C0DBFF0E0E3AC0DBFF0F0E3BC0DBFF97
:106A4A001200040EDBCF00F0050EDBCF01F01200BE
:106A5A0008C038F009C039F00AC03AF0120088D8E4
:106A6A00A80ED880EE54610EED54120090D9140E7F
:106A7A001200E16E0350DE6A800EDE6EDE6ADD6AA7
:106A8A00DD52DD521200B6D9010EEE181200100EB8
:106A9A00DB6A110EDB6A120EDB6A130EDB6A120066
:106AAA0039C008F03AC009F03BC00AF03CC00BF00C
:106ABA001200060EDBCF3AF0070EDBCF3BF023EFD6
:106ACA0055F0FF0EEE5CFF0EEE58010EEE58000E6A
:106ADA00EE581200E16EDF6A010EDB6A020EDB6A13
:106AEA00030EDB6A120037EC30F011EF37F0010EBB
:106AFA00F36E030EF3CFDBFF1200E16E03503EEF9D
:106B0A003EF0C36F96809482958C958E9588958A6F
:106B1A001200010EE66ED9501200F36E010EF3CF89
:106B2A00DBFF020EDB6A1200010EDBCFB2FE020EA1
:106B3A00DBCFB3FE1200D890383639363A363B36B8
:106B4A00E8061200D8900436053606360736E806F7
:106B5A00120000C0E6FF01C0E6FF1200DECFE6FF2A
:106B6A00DDCFE6FF1200E76E040EE7CFDBFF12006F
:106B7A00E96E000EDA20EA6E12000C0EDBCF04F08A
:106B8A000D0EDBCF05F00E0EDBCF06F00F0E120056
:106B9A0039C03EF03AC03FF03BC040F03CC041F043
:106BAA00120000C038F001C039F002C03AF003C048
:106BBA003BF01200080EDBCF38F0090EDBCF39F0BC
:106BCA000A0EDBCF3AF00B0EA6EF33F0080EDBCF3E
:106BDA0039F0090EDBCF3AF00A0EDBCF3BF00B0E91
:106BEA00E0EF33F00C0EDBCF39F00D0EDBCF3AF0CD
:106BFA000E0EDBCF3BF00F0EE0EF33F0FFD8EECFF7
:106C0A0000F0EECF01F0EECF02F0EFCF03F012006A
:106C1A00190E3D6E3E6A3F6A406AA5EC64F0EADDF1
:106C2A00F2D0CFDD060E1DEF33F0DBCF0BF010DF15
:106C3A000BC03BF03AEC55F0E8DD7BDDA6EC55F0F5
:106C4A00AAEF56F0D950080F36DDF4D832EC2DF001
:106C5A00006E0C0EE15C1200E16EDE6A50DE4FEF50
:106C6A0033F031DD11EF37F037DEEED852DF15EFB2
:106C7A0037F0040EDBCF39F0050EDBCF3AF0060E03
:106C8A00DBCF3BF0070EE0EF33F0040EDBCF38F03A
:106C9A00050EDBCF39F0060EDBCF3AF0070EA6EF72
:106CAA0033F00C0EDBCF00F00D0EDBCF01F00E0E31
:106CBA00DBCF02F00F0E3DEF33F0140EDBCF39F0CD
:106CCA00150EDBCF3AF0160EDBCF3BF0170EE0EFD6
:106CDA0033F0140EDBCF00F0150EDBCF01F0160EE9
:106CEA00DBCF02F0170E3DEF33F0140EDBCF04F0CA
:106CFA00150EDBCF05F0160EDBCF06F0170E13EFDD
:106D0A0034F0F20EDBCF04F0F30EDBCF05F0F40E15
:106D1A00DBCF06F0F50E13EF34F0CFDCE652E65285
:106D2A001200070E85DCE66AD9501200CCDC036E2D
:106D3A00070EE15C1200DBCF03F024EF37F0150EEB
:106D4A00EECFDBFF160EEECFDBFF170EEECFDBFF2B
:106D5A001200EECFE6FFEECFE6FFEECFE6FFEFCF73
:106D6A00E6FF120038C000F039C001F03AC002F064
:106D7A003BC003F01200CDDE030F23DD29EF37F00D
:106D8A0063D8E76E020EE7CFDBFFDB50120039C093
:106D9A0000F03AC001F03BC002F03CC003F0120020
:106DAA00E96EFF0E61EF34F001C03AF002C03BF029
:106DBA0003C03CF012004FDC4BDDB0EF33F0000EA5
:106DCA003954000E3A54000E3B541200EE54000E91
:106DDA00EE54000EEE541200E96EFF0EDA20EA6E4F
:106DEA001200D9CFE6FFDACFE6FF1200DBCF40F080
:106DFA00A5EF64F0D950010FBDEF35F0D9CFE9FF07
:106E0A00DACFEAFF12000C0EDB6A0D0EDB6A0E0EF9
:106E1A00DB6A0F0EDB6A1200E552E552E5521200F8
:106E2A00010FCFDC030E1DEF33F01BDF010EDE6E08
:106E3A0084EF34F0D950040F3EDCAEEF33F000504B
:106E4A000110021003101200010E1DEF33F0D8CF0B
:106E5A00E4FFE0CFE4FFE46EE9CFE4FFEACFE4FF2A
:106E6A00F3CFE4FFF4CFE4FFE65296EC47F0FBECF5
:106E7A0046F0030EDB6AA4A69ED1A4960E01002B4F
:106E8A000E01AB510E01005D01E284D0006B0E01D0
:106E9A00C6EC46F0EF6A79907B6A7A6A0E01A92BF2
:106EAA000E01AA510E01A95D01E3A96B8EEC47F010
:106EBA00EA22EE50ED106EE030EC48F0E0EC47F0DC
:106ECA0002E14B50491847E0A4EC47F0EA22EE50A1
:106EDA00ED103AE0BAEC47F0A1EC46F08EEC47F040
:106EEA00EA22EE504A5C486EEE504B58496E020E4A
:106EFA0048C0DBFF030E49C0DBFF1AEC47F04934F8
:106F0A0012E248500008000E49540DE21AEC47F00C
:106F1A00A4EC47F0CAEC47F017E217EC48F0EE266B
:106F2A004950ED2218D01AEC47F0486C491E000E61
:106F3A004922A4EC47F0CAEC47F006E217EC48F005
:106F4A00EE5E4950ED5A07D030EC48F0EA2248C0CC
:106F5A00EEFF49C0EDFFC6EC46F0120EEF6EF29E50
:106F6A000E018EEC47F05DEC46F049C048F0496AE4
:106F7A004850B66E8EEC47F05DEC46F04850B56E60
:106F8A00F00EB4140009B46EF00EB4140909B46E0C
:106F9A007980F28E0701000ED880AA55000EAB55F3
:106FAA002EE2B82B000EB923AA51B85DAB51B959DC
:106FBA0026E3B86BB96B030EAE5D1FE2AC51EA6A09
:106FCA00200FE96E010EEA2280CFEFFFAC51EA6A88
:106FDA00230FE96E010EEA2281CFEFFFAC51EA6A74
:106FEA00260FE96E010EEA2282CFEFFFAC2B030EC9
:106FFA00AC5D01E3AC6BAE2B02D0AA6BAB6B000E9F
:10700A00D880AF55000EB0551CE2000ED880BE5590
:10701A00000EBF5516E2BA2B000EBB23AF51BA5D64
:10702A00B051BB590EE3BA6BBB6B030EB35D07E2FB
:10703A00B12B030EB15D01E3B16BB32B02D0AF6B81
:10704A00B06BBE51BF110BE0050EBD5D07E3C18CED
:10705A009E9C9D8CC280C282BD6B01D0BD2B050156
:10706A00005101E1A4D0DE6ADD6ADECF48F0DDCF4F
:10707A0049F0040E485C000E495801E398D063ECCD
:10708A0046F0A7EC46F0FDE1010EE926050EEA22DC
:10709A00EE50ED1070E063EC46F0A7EC46F0FDE12F
:1070AA00E4EC47F0EE50ED1016E1E9EC47F001E1AF
:1070BA008180EDEC47F003E1ED5001E18182F1ECD2
:1070CA0047F003E1ED5001E18184F5EC47F003E17B
:1070DA00ED5001E1818663EC46F0A7EC46F0FDE154
:1070EA00C4EC47F0A7EC46F0FDE1010EE926050ED7
:1070FA00E0EC47F019E14B50491816E1E9EC47F08A
:10710A0001E18190EDEC47F003E1ED5001E181925C
:10711A00F1EC47F003E1ED5001E18194F5EC47F021
:10712A0003E1ED5001E1819663EC46F0A7EC46F0ED
:10713A00FDE1E4EC47F0EE2A000EEF2263EC46F0A4
:10714A00A7EC46F0FDE1C4EC47F0A7EC46F0FDE100
:10715A00090EE926050EE0EC47F023E14B504918E9
:10716A0020E163EC46F0A7EC46F0FDE1E4EC47F0E1
:10717A00EE6AED6A16D0E9EC47F001E18190EDEC98
:10718A0047F003E1ED5001E18192F1EC47F003E1B0
:10719A00ED5001E18194F5EC47F003E1ED5001E196
:1071AA008196DF2A010E01E260D7DB2A5ED706014B
:1071BA00CC5101E0CC079EAC3DD09E9CC1AC07D01F
:1071CA00C19C010E0701C06FC16BBC6B18D0C450C3
:1071DA004A6E4B6E4A6AC35000014A10486E4BC051
:1071EA0049F00701BC51E96EEA6AEBEC46F048C087
:1071FA00EEFF49C0EDFFD890C037C137BC2B100E47
:10720A00BC5D0EE2C051BE15486EC151BF15496E34
:10721A004850491005E1BC2BD890C037C137EFD789
:10722A00100EBC5D02E39D9C05D0BC51040DF328F1
:10723A00C26EC282F2A435D0D59EF294F29A040E9E
:10724A00486E0701B75101EC47F0EF50485C29E15D
:10725A00080EB75D0AE23AEC47F004E0E846FE0B96
:10726A004806FCE1E81C891616D0100EB75D0AE242
:10727A003AEC47F004E0E846FE0B4806FCE1E81C5D
:10728A008A1609D03AEC47F004E0E846FE0B4806B5
:10729A00FCE1E81C8B160701B75101EC47F0020E1E
:1072AA00EF6E040EE15C02E2E16AE552E16EE5523C
:1072BA00E5CFDAFFE7CFD9FFE552E5CFF4FFE5CF17
:1072CA00F3FFE5CFEAFFE5CFE9FFE550E5CFE0FFC1
:1072DA00E5CFD8FF10001DEC48F0896A92680701D3
:1072EA00BE6BBF6B8A6A93688B6A94688C968C941F
:1072FA0095969594928E010EE36F0701F369F469EE
:10730A000701B26BB16BB36BAD6BAC6BAE6BAA6BB7
:10731A00AB6BAF6BB06BB86BB96BBA6BBB6BBC6B5F
:10732A0076827680769C769A76887696FA0E776E4C
:10733A00DF6ADFCF00F0100EE76E0018E8AE02D069
:10734A00E73402D0E750005C0BE2DFCFE9FFEA6ADC
:10735A00E9BEEA68EBEC46F0EE6AED6ADF2AE9D7A5
:10736A000701DD6BDE6BDB6BDC6BDF6BE06BE16B0C
:10737A00E26BB56BB66BB76BDF6ADFCF00F0180E46
:10738A00E76E0018E8AE02D0E73402D0E750005C9E
:10739A0016E2DFCFE9FFEA6AE9BEEA684FEC47F096
:1073AA00EE6AED6ADFCFE9FFEA6AE9BEEA68290E0A
:1073BA00E926010EEA22010EEF6EDF2ADED7D58614
:1073CA00D59AD59CF294F29AF1940F01498FBE0E88
:1073DA00C16ED08E7694A386A59669EC27F0D6EC7A
:1073EA005EF0F28EF28C7684E552E55240EF46F07A
:1073FA001DEC48F0FBEC46F0030EDB6A040EDB6A78
:10740A0064EC45F00701AE5100080AE286EC3FF051
:10741A000701AD2B030EAD5D01E1AD6BAE07F2D7EF
:10742A00B35100080AE2A8EC3FF00701B22B030EA1
:10743A00B25D01E1B26BB307F3D7200E0201E76E2A
:10744A008019E8AE02D0E73402D0E750805D01E24D
:10745A0039D16550020B01E035D1400EE66E400E7F
:10746A00E66E020EE66E6DEC5DF02CEC48F0E76E0F
:10747A00030EE7CFDBFFDB50000801E3E5D0040E83
:10748A00DB6A030EDB50F36E040EF1EC46F001E307
:10749A00DBD0040EDB50EA6A400FE96E020EEA22E4
:1074AA00EFCFDFFF05015D5132E10D0E71EC46F0C1
:1074BA0005E00A0E016EDF50015C29E1010E5D6FE5
:1074CA000701AFEC46F00D0EEF6EDD2B010EDB6A05
:1074DA00DD51F36E010EF1EC46F014E246EC47F092
:1074EA00E9BEEA68000EE926030EEA22EF50E66ECC
:1074FA0046EC47F0E9BEEA68190EE926050E5BEC90
:10750A0047F0E6D73CD90701DD6BDE6B8DD01B0E49
:10751A00DF5C09E1595107E1010E596F1B0E5A6FE1
:10752A005B6B5C6B81D059050BE15B0EDF5C08E19C
:10753A001B0E5A5D05E15B5103E15B0E5B6F74D074
:10754A0059054AE1410EDF5C47E11B0E5A5D44E1F1
:10755A005B0E5B5D41E15A6B5B6B5C6B596B010EB9
:10756A00DB6ADBCFE9FFEA6AE9BEEA68000EE926D0
:10757A00030EEA22EF500D0814E046EC47F0E9BE8C
:10758A00EA68190EE926050EEA22EF50E66E46EC85
:10759A0047F0E9BEEA68000EE926030E5BEC47F005
:1075AA00E0D7010EDBCFDDF70701AFEC46F0EF6A5B
:1075BA00610E006EB50E87EC47F0000EE66E030E04
:1075CA00E66E5E0E006EB50E93EC47F002E2E16ADB
:1075DA00E552E16E035028D0080EDF5C0EE1070188
:1075EA00DD5100080AE2DD07AFEC46F0EF6A5B0EF8
:1075FA00006EB50E87EC47F017D00D0EDF5C14E075
:10760A000A0EDF5C11E0200EDF5C0EE305015A6B07
:10761A005B6B5C6B596B0701AFEC46F0DFCFEFFF9A
:10762A0005015D6B0701DD2B0701DD51006E016A63
:10763A00000E001806E1010E011803E1B487DD6BA4
:10764A00DE6B040EDB2A1DD70701B4513AE0B4A160
:10765A0005D0550E006EB50E87EC47F00701B4A3AE
:10766A0005D0360E006EB50E87EC47F00701B4A5BB
:10767A0005D01A0E006EB50E87EC47F00701B4A7C5
:10768A0005D0FE0E006EB40E87EC47F00701B4A9D0
:10769A0005D0DF0E006EB40E87EC47F00701B4ADDB
:1076AA0005D0BE0E006EB40E87EC47F0000E07013F
:1076BA00B41505E0A50E006EB40E87EC47F007017D
:1076CA00B46B37D8050EE15C02E2E16AE552E16E7D
:1076DA0040EF46F096EC47F0DBC7DFFFDF2A400EAB
:1076EA0071EC46F001E1DF6A0701DC51DF5C01E180
:1076FA0020D80701DB51EA6A000FE96E020EEA227E
:10770A00FD0EDBCFEFFFDB2B400EDB5D01E1DB6B18
:10771A00DC51DB5D01E1B485FD0EDBCF00F0016ACF
:10772A0000BE016800C0F3FF01C0F4FFE55240EF5C
:10773A0046F096EC47F00701DB51DC5D1DE00701DE
:10774A00905105E0F7EC5DF0B6EC48F0F8D7070188
:10775A00DC51D880DB5507E2DC51DB5D88EC46F072
:10776A00DBC7DCF707D0400ED880DC5588EC46F042
:10777A000701DC6BF7EC5DF0E55240EF46F01DECDB
:10778A0048F0E652E652DE6ADD6A020EDB6A030E52
:10779A00DB6A070150EC46F062EC47F0020EF3CFC9
:1077AA00DBFF07016AEC46F004E1010E011801E172
:1077BA00DE6B020EDB50DE6EDD6A50EC46F02C0802
:1077CA0024E050EC46F00D0820E050EC46F062EC64
:1077DA0047F0030EF3CFDBFF07016AEC46F004E142
:1077EA00010E011801E1DE6B020EDBCF02F002C0CE
:1077FA0003F0026A030EDB5000010224006E000E41
:10780A000320016E00C0DEFFDD6E000EDFCF3AF00E
:10781A00010EDBCF3BF0530E3A1802E1430E3B1840
:10782A0001E1F7D1530E3A1802E1510E3B1801E17A
:10783A00EDD14D0E3A1802E1580E3B1801E1E3D1A1
:10784A00530E3A1802E1450E3B1801E1D9D1430E15
:10785A003A1802E1410E3B1801E1D0D14D0E3A1817
:10786A0002E1510E3B1801E1C6D14D0E3A1802E170
:10787A00520E3B1801E1BCD1320E3A1802E1530E06
:10788A003B1801E1B2D1450E3A1802E1530E3B18FA
:10789A0001E1A8D1430E3A1802E1510E3B1801E169
:1078AA009ED14B0E3A1802E1430E3B1801E194D1E6
:1078BA004C0E3A1802E1420E3B1801E18AD1440EFD
:1078CA003A1802E14E0E3B1801E180D1490E3A18EE
:1078DA0002E14E0E3B1801E176D1420E3A1802E15E
:1078EA00510E3B1801E16CD14C0E3A1802E1510ECF
:1078FA003B1801E162D14C0E3A1802E1530E3B18D3
:10790A0001E158D14E0E3A1802E1510E3B1801E13D
:10791A004ED14E0E3A1802E1530E3B1801E144D102
:10792A00430E3A1802E1530E3B1801E13AD14D0ECB
:10793A003A1802E1450E3B1801E130D1500E3A18CF
:10794A0002E1510E3B1801E126D1500E3A1802E12C
:10795A00540E3B1801E11CD1500E3A1802E1530EA5
:10796A003B1801E112D14D0E3A1802E1410E3B18C3
:10797A0001E108D14D0E3A1802E1530E3B1801E11C
:10798A00FED0470E3A1802E1500E3B1801E1F4D03E
:10799A00430E3A1802E1500E3B1801E1EAD0490EB3
:1079AA003A1802E1430E3B1801E1E0D0490E3A18B9
:1079BA0002E1520E3B1801E1D6D0490E3A1802E113
:1079CA00530E3B1801E1CCD0530E3A1802E1520E85
:1079DA003B1801E1C2D0530E3A1802E1530E3B188C
:1079EA0001E1B8D0530E3A1802E1420E3B1801E108
:1079FA00AED0430E3A1802E1420E3B1801E1A4D080
:107A0A00430E3A1802E1520E3B1801E19AD04F0E8A
:107A1A003A1802E1420E3B1801E190D0570E3A188B
:107A2A0002E14D0E3B1801E187D0520E3A1802E1ED
:107A3A004D0E3B1801E17ED0440E3A1802E1500E79
:107A4A003B1801E175D04F0E3A1802E1500E3B186F
:107A5A006DE0490E3A1802E1500E3B1865E0580EE7
:107A6A003A1802E1540E3B185CE0540E3A1801E150
:107A7A003B5055E0410E3A1801E13B504EE0560E9C
:107A8A003A1801E13B5047E0490E3A1801E13B50F0
:107A9A0040E04F0E3A1801E13B5039E0550E3A18D2
:107AAA0002E1430E3B1831E0580E3A1802E1430E48
:107ABA003B1828E0430E3A1801E13B5021E0520EF0
:107ACA003A1801E13B501AE0580E3A1802E1520EF8
:107ADA003B1811E0030EDB5001E09ED0020E0BECC6
:107AEA0047F00BEC47F0820E006EB40EBFEC47F085
:107AFA0001E3A1D09ED0DAEC41F09FD0C3D89DD04B
:107B0A0029D99BD0DCEC41F098D0C0D896D0C5D901
:107B1A0094D0F7D992D012DA90D015DA8ED0F1D863
:107B2A008CD0D8EC41F089D036DB87D0A7DB85D062
:107B3A009DDA83D07CDA81D068DA7FD04EEC42F0CD
:107B4A007CD0DEEC41F079D04CEC42F076D050ECAF
:107B5A0042F073D052EC42F070D054EC42F06DD047
:107B6A0056EC42F06AD058EC42F067D05AEC42F038
:107B7A0064D05CEC42F061D0B6EC42F05ED0B8EC76
:107B8A002BF05BD004EC29F058D0F8EC2FF055D04C
:107B9A00D9EC2FF052D0C6EC2FF04FD074EC30F065
:107BAA004CD03DEC28F049D0F6EC30F046D016EC3B
:107BBA0031F043D028EC31F040D035EC31F03DD0F3
:107BCA0047EC31F03AD0D8EC30F037D0E9EC30F06D
:107BDA0034D0EBEC42F031D0F3EC42F02ED05BEC37
:107BEA0031F02BD06FEC31F028D04DEC5FF025D07E
:107BFA0005EC32F022D006EC32F01FD03AD91DD073
:107C0A003EEC2FF01AD053EC2CF017D0DCEC32F00B
:107C1A0014D010EC33F011D0D0EC47F0D0EC47F090
:107C2A005A0E006EB40E31EC46F0036E0B0EE15C98
:107C3A0002E2E16AE552E16E0350070150EC46F0B8
:107C4A000D080DE0B4510BE1520E006E016ADF50CF
:107C5A00001803E1DE52DD50011801E0B48FDDC7E0
:107C6A00DEF7040EE15C02E2E16AE552E16E40EF02
:107C7A0046F00701E35105E0920E006EC90E87EC4B
:107C8A0047F0120070EC39F03EEF3EF096EC47F008
:107C9A000EEC48F04BEC46F0020E13EC48F02FE1E4
:107CAA00DF0414E1D950010F21EC47F00AE0010E7C
:107CBA00006E016ADB50001808E1020EDB50011861
:107CCA0004E1010EDBCFE3F701D0B48D020E71ECB3
:107CDA0046F014E1D950010F21EC47F00AE0010EF9
:107CEA00006E016ADB50001808E1020EDB50011831
:107CFA0004E1010EDBCFBFFE01D0B48DBADF99EFEC
:107D0A0047F03AEC46F0FBEC46F0E66AA80EE66E5F
:107D1A00070EE66E34EC48F01BE1020EDB500CE174
:107D2A00A851A91103E1AA6BAB6B11D07684A8C73D
:107D3A00AAF7A9C7ABF70BD0A851A91103E1AF6BFA
:107D4A00B06B05D07684A8C7AFF7A9C7B0F791DFA3
:107D5A0099EF47F01DEC48F0E6520EEC48F043EC80
:107D6A0048F0020F43EC48F0030F43EC48F0040FCD
:107D7A008AEC47F00FE1DF50926E010EDB50936EF2
:107D8A00020EDB50946E030EDB50956E040EDB5030
:107D9A00966E6FDF050EE15C02E2E16AE552E16E82
:107DAA0040EF46F03AEC46F0FD0EDB50100805E2D3
:107DBA00100EF36EFD0EF3CFDBFFFC0EDB502AE054
:107DCA00FD0EDB5026EC65F0F3500701BE13F450AC
:107DDA00BF13080EF36EFD0EF1EC46F00DE2010E34
:107DEA00F36EFD0EDB5003E066EC46F0FDE1F35066
:107DFA00F31C0F0148173BD0FD0EDB500C0837E38C
:107E0A0069EC47F003E04BEC47F0FDE1E81C0F0199
:107E1A0049172DD0FD0EDB5026EC65F0F3CF00F0AC
:107E2A00F4CF01F0001E011E00500701BE170150D9
:107E3A00BF17080EF36EFD0EF1EC46F00CE2010ED0
:107E4A00F36EFD0EDB5003E066EC46F0FDE1F35005
:107E5A000F0148130CD0FD0EDB500C0808E369EC47
:107E6A0047F003E04BEC47F0FDE10F01491340EF07
:107E7A0046F03AEC46F00EEC48F08AEC47F009E19D
:107E8A00010EDBCFE6FFDFCFE6FF8CDFE552E552DE
:107E9A00F0DEE552E55240EF46F03AEC46F059EC96
:107EAA0046F0010E2EEC46F096EC46F026E1010E65
:107EBA00DB5002E1DF50896EA0EC47F01EE1010EB3
:107ECA00DB5002E1DF508A6EA0EC47F016E1010EAA
:107EDA00DB5002E1DF508B6EA0EC47F00EE1010EA1
:107EEA00DB5002E1DF508C6EA0EC47F006E1010E98
:107EFA00DB5002E1DF508D6EBCDEE552E55240EF09
:107F0A0046F08450E66EE66A8350E66EE66A825070
:107F1A00E66EE66A8150E66EE66A8050E66EE66ACA
:107F2A003D0E006EB40E31EC46F0036E0D0EE15CB0
:107F3A0002E2E16AE552E16E035012009A0E006E07
:107F4A00C90E87EF47F01DEC48F0E652DF6A010ED2
:107F5A00F36EDB6E020EDB6A3B0E006EB40E87EC2C
:107F6A0047F09DBCFED7DF6ADFCF00F0100EE76E48
:107F7A000018E8AE02D0E73402D0E750005C3EE2D7
:107F8A00010EDB500701BE150001006E020EDB5028
:107F9A000701BF150001016E005001101EE0DFCF7E
:107FAA00E9FFEA6AE9BEEA68EBEC46F0EECFE6FFE3
:107FBA00EFCFE6FFDFCF00F0016A00BE0168F9ECFF
:107FCA0047F0300E026EB40E0FEC47F0070EE15C7C
:107FDA0002E2E16AE552E16E0550010EDBCF00F0E4
:107FEA00020EDBCF01F0D89000360136010E00C038
:107FFA00DBFF020E01C0DBFFDF2AB6D7970E006E49
:10800A00C90E87EC47F099EF47F096EC47F059EC28
:10801A0046F034EC48F009E131EC47F005E2FEECB9
:10802A0047F0020EDBCFEFFF24DE99EF47F096EC24
:10803A0047F059EC46F0030E13EC48F015E131EC29
:10804A0047F005E2FEEC47F0020EEFCFDBFF020E2F
:10805A000BEC47F0260E006EB40E93EC47F002E2EA
:10806A00E16AE552E16E035099EF47F047EC48F0B8
:10807A0001E08FD0020EDB50010801E287D0010E29
:10808A00DB50070801E282D0410E71EC46F016E19E
:10809A00020EDB500AE175EC46F003E066EC46F0AE
:1080AA00FDE1F350F31C921673D075EC46F003E031
:1080BA0066EC46F0FDE1F35092126AD0420E71EC82
:1080CA0046F016E1020EDB500AE175EC46F003E0D9
:1080DA0066EC46F0FDE1F350F31C931659D075ECAB
:1080EA0046F003E066EC46F0FDE1F350931250D0FF
:1080FA00430E71EC46F016E1020EDB500AE175EC14
:10810A0046F003E066EC46F0FDE1F350F31C9416EA
:10811A003FD075EC46F003E066EC46F0FDE1F35023
:10812A00941236D0440E71EC46F016E1020EDB5082
:10813A000AE175EC46F003E066EC46F0FDE1F35027
:10814A00F31C951625D075EC46F003E066EC46F074
:10815A00FDE1F35095121CD0450E71EC46F016E184
:10816A00020EDB500AE175EC46F003E066EC46F0DD
:10817A00FDE1F350F31C96160BD075EC46F003E0C4
:10818A0066EC46F0FDE1F350961202D0B48D01D0B0
:10819A0070DD99EF47F03AEC46F0FBEC46F03DEC27
:1081AA0048F0050E83EC47F0010F8AEC47F064E1D2
:1081BA00010EDB5007084CE3410E71EC46F00AE170
:1081CA00C0EC46F003E04BEC47F0FDE1E8407F0BE2
:1081DA00801437D0420E71EC46F00AE1C0EC46F04A
:1081EA0003E04BEC47F0FDE1E8407F0B811429D016
:1081FA00430E71EC46F00AE1C0EC46F003E04BECAA
:10820A0047F0FDE1E8407F0B82141BD0440E71EC6D
:10821A0046F00AE1C0EC46F003E04BEC47F0FDE122
:10822A00E8407F0B83140DD0450E71EC46F010E147
:10823A00C0EC46F003E04BEC47F0FDE1E8407F0B71
:10824A008414E76E020EE7CFDBFFDB5008E002D0B2
:10825A00B48D12D0010EF36E020EF3CFDBFF020EC5
:10826A000BEC47F01D0E006EB40E93EC47F002E2E1
:10827A00E16AE552E16E035099EF47F047EC48F0A6
:10828A0001E08FD0020EDB50010801E287D0010E17
:10829A00DB50070801E282D0410E71EC46F016E18C
:1082AA00020EDB500AE175EC46F003E066EC46F09C
:1082BA00FDE1F350F31C891673D075EC46F003E028
:1082CA0066EC46F0FDE1F35089126AD0420E71EC79
:1082DA0046F016E1020EDB500AE175EC46F003E0C7
:1082EA0066EC46F0FDE1F350F31C8A1659D075ECA2
:1082FA0046F003E066EC46F0FDE1F3508A1250D0F6
:10830A00430E71EC46F016E1020EDB500AE175EC01
:10831A0046F003E066EC46F0FDE1F350F31C8B16E1
:10832A003FD075EC46F003E066EC46F0FDE1F35011
:10833A008B1236D0440E71EC46F016E1020EDB5079
:10834A000AE175EC46F003E066EC46F0FDE1F35015
:10835A00F31C8C1625D075EC46F003E066EC46F06B
:10836A00FDE1F3508C121CD0450E71EC46F016E17B
:10837A00020EDB500AE175EC46F003E066EC46F0CB
:10838A00FDE1F350F31C8D160BD075EC46F003E0BB
:10839A0066EC46F0FDE1F3508D1202D0B48D01D0A7
:1083AA0068DC99EF47F03EEF3EF03EEF3EF03EEFDD
:1083BA003EF01DEC48F008EC48F0B7EC47F060E1FD
:1083CA00D950020F03EC48F0720ED880EE542E0EEC
:1083DA00ED543BE3D950020F21EC47F01FE003684C
:1083EA000468056A2D0EE76E020EDBCF06F0030E57
:1083FA00DBCF07F0E7500626000E0722086A065070
:10840A00035C006E07500458016E08500558026E4E
:10841A00020E00C0DBFF030E01C0DBFF010EDB50C2
:10842A00070813E3410E71EC46F002E1DF6A0FD050
:10843A00420E71EC46F002E1080E05D0430E71ECD3
:10844A0046F003E1100EDF6E02D0B48D19D0010E92
:10845A00DB50DF24E96EEA6A4FEC47F070EC47F034
:10846A00010EDB50DF2401EC47F0EF0407E1010EB7
:10847A00DB50DF2401EC47F0020EEF6E3EEC3EF0DB
:10848A00040EE15C02E2E16AE552E16EF4D33EEFEA
:10849A003EF03EEF3EF03EEF3EF03EEF3EF03EEF66
:1084AA003EF03EEF3EF03EEF3EF03EEF3EF0DDDBCB
:1084BA00070EE12402E3E168E652E16E3DEC48F082
:1084CA00030E83EC47F0B7EC47F044E1DECF01F549
:1084DA00DDCF02F5020EDBCF09F5030EDBCF0AF57D
:1084EA00040EDB6A030EF36E040EF1EC46F030E282
:1084FA009DEC46F0030EADDBE76E050EE7CFDBFF22
:10850A00010EE66ED95039EC48F0A3DBE76E060E91
:10851A00E7CFDBFF0701B4511DE1050EDB5018E17F
:10852A00060EDB5015E155EC47F0010EE926050E63
:10853A00EA22DECFEEFFDDCFEDFF55EC47F0090E64
:10854A00E926050EEA2270EC47F0040EDB2ACAD7A8
:10855A003EEC3EF0070EE15C02E2E16AE552E16EB2
:10856A008AD396EC47F03DEC48F0010E13EC48F044
:10857A000DE1DF5007E0F00E9314936E0501010E32
:10858A00006F02D00501006B3EEC3EF0E55273D35A
:10859A00D9CFE6FFDACFE6FFE1CFD9FFE2CFDAFFA4
:1085AA00E652DF6AFF0EDF5C0AE2E868E85005E09F
:1085BA00E80600D000D000D0F9D7DF2AF3D7E55279
:1085CA00E552E5CFDAFFE7CFD9FF1200F29EF29C1F
:1085DA006592656ADDDF0FEF00F0120046DB100ED0
:1085EA00E12402E3E168E652E16EE66AD950010F3E
:1085FA004DDBE66AD5EC47F03DEC48F0010E83EC22
:10860A0047F0040F43DB020E83EC47F039EC48F0E5
:10861A0083EC47F00A0F3ADB060E83EC47F0060FAD
:10862A0035DB070E83EC47F00E0F30DB040E83ECCC
:10863A0047F00F0F2BDB050E0CDB010EDBCF00F032
:10864A00016A00BE0168F9EC47F0110E026EB40E21
:10865A00E1DB050EE15C02E2E16AE552E16E0550FA
:10866A00DFCFE6FFE66A050E006EB40E93EC47F024
:10867A0002E2E16AE552E16E0350040EDBCFE6FF47
:10868A00050EDBCFE6FFF90E006EB30E93EC47F052
:10869A0002E2E16AE552E16E0350020EDBCFE6FF29
:1086AA00030EDBCFE6FFED0E006EB30E93EC47F040
:1086BA0002E2E16AE552E16E0350D9500A0F6FDB1C
:1086CA00E00E006EB30EBFEC47F002E2E16AE5523B
:1086DA00E16E0350D950060F62DBD30E006EB30E63
:1086EA00BFEC47F002E2E16AE552E16E03500E0E7A
:1086FA008DDBC70E006EB30E93EC47F002E2E16A1F
:10870A00E552E16E03500F0E81DBBB0E006EB30E15
:10871A0093EC47F002E2E16AE552E16E03503EEC67
:10872A003EF0100EE15C02E2E16AE552E16EA3D28C
:10873A009CDA090EE12402E3E168E652E16E080ED2
:10874A00DB6A0D0E006E0701A6DA005C05E1FA0E7F
:10875A00DB5027E1B48925D09EDA2C0813E0FA0E03
:10876A00DB500EE198DAE66EE66A940E006EB30EFE
:10877A00D5DB02E2E16AE552E16E03500701B48BF0
:10878A00020E25D1A2DA04E1010E011801E1DE6B25
:10879A000D0E006E80DA005C06E1FA0EDB5001E194
:1087AA00B489030E14D12D0E006E75DA005C20E137
:1087BA00040E4DDB1DE0050E026EFD0EDB50025C61
:1087CA0017E0FD0EDB0401E1C8D0030E0ADB01E16C
:1087DA00C4D0070E3CDB01E1C0D0010EF36E080ED7
:1087EA00F3CFDBFF72DA04E1010E011801E1DE6B5F
:1087FA00040EF7DA0AE0050E2ADB07E00A0EE66E37
:10880A0095DBEED82CEC48F036D0DE519DDBEFCF6D
:10881A0000F0000E00C0DFFF010EDB6A020EDB6A09
:10882A00030EDB6A050EDDDA1FE1000EDFCFE6FF7D
:10883A00010EDBCFE6FF7FEC64F0E552E552F3CFA1
:10884A0000F0F4CF01F0026A036A01AE02D00268B6
:10885A00036800C0DFFF010E01C0DBFF020E02C089
:10886A00DBFF030E03C0DBFF07012FDA04E1010E71
:10887A00011801E1DE6B080EDB5042E0FD0EDB5011
:10888A0007E140EC48F0800E38DA000EEE5412E3AD
:10889A00020EA7DA06E1EFDB000EEE54800E2DDAA7
:1088AA0009E3060ED4DA08E1E6DB000E26DA800ECA
:1088BA00EE5402E2070151D0F2D97BDA080EDB50FE
:1088CA0054E0040EDBCF38F0050EDBCF39F0060E8C
:1088DA00DBCF3AF0070EDBCF3BF03D683E683F68DE
:1088EA00406847EC64F0040E34C0DBFF050E35C067
:1088FA00DBFF060E36C0DBFF070E37C0DBFF35D0C5
:10890A00FD0EDB5006E1B7DB7F0EEE54000EF5D903
:10891A0023E3FD0EDB0404E11DDB000EEED91CE3AC
:10892A00020E5FDA04E116DB7F0EE7D915E3030EC8
:10893A008EDA04E10FDBFF0EE0D90EE3060E026EBB
:10894A00FD0EDB50025C0CE105DBFF0EEE54FF0E60
:10895A00EE547F0EEE5404E20701B48D010E37D0B7
:10896A00070E3FDA02E09BD924DAFD0EDB50070A34
:10897A0021E0010A17E0050A11E0010A0FE0030AE3
:10898A0008E0050A06E0010A04E0050A02E0040E0E
:10899A001ED0E3D9040EDBCFEFFF18D006DBDBCF06
:1089AA00EDFF14D002DBDBCFEEFF060EDBCFEEFFCE
:1089BA00070E0AD0D2D9DFCFEEFF010EDBCFEEFFD2
:1089CA00020EDBCFEEFF030EDBCFEEFF000E006ED2
:1089DA00090EE15C02E2E16AE552E16E00504BD118
:1089EA0027DB2EDAEE6AEE6AEE6AEE6A010EDB6ABF
:1089FA00FB0EDB50F36E010EEFD94FE20701DE5199
:108A0A00A3DAEFCFDFFF300EDF5C42E3DF50390835
:108A1A003FE316DAEECF00F0EECF01F0EECF02F030
:108A2A00EFCF03F00A0E3D6E3E6A3F6A406A00C00D
:108A3A0038F001C039F002C03AF003C03BF047EC0D
:108A4A0064F034C000F035C001F036C002F037C01F
:108A5A0003F0300EDF5C046E056A066A076AE850A6
:108A6A000026055001220650022207500322E8D9A7
:108A7A0000C0EEFF01C0EEFF02C0EEFF03C0EEFF32
:108A8A00070123D907E1010E011804E1DE6B02D0C8
:108A9A00000E04D0010EDB2AABD7010EE552E552D7
:108AAA00EAD00701AE51E66EE66A880E006EB30E92
:108ABA0035DA02E2E16AE552E16E03501200020180
:108ACA00805108E0010E006E6550020B01E0010EB4
:108ADA00005C17E1D0D90BE16151621111E18C867A
:108AEA00A00E616F0F0E626F010E636F120061516B
:108AFA00621152E18C96A00E616F0F0E626F636B6A
:108B0A001200800509E0020E805D06E0040E805D19
:108B1A0003E0100E805D17E1AED90BE161516211DD
:108B2A0011E18C86200E616F4E0E626F010E636F2B
:108B3A0012006151621130E18C96200E616F4E0E67
:108B4A00626F636B1200200E805D26E194D907E103
:108B5A006151621121E18C86CCD9010E15D06305D1
:108B6A0007E16151621118E18C96C3D9020E0CD04B
:108B7A00020E635D0BE1615162110EE18C86A00E5B
:108B8A00616F860E626F030E636F1200615162118C
:108B9A0003E18C96AED9636B120067D8A3D9E8AE0D
:108BAA0002D0003403D0E750D880005423E3FC0EEF
:108BBA00DB5010E0CAD8E9BEEA6896D804E0E84675
:108BCA00FE0B0106FCE1006EC0D8E9BEEA6833DAA2
:108BDA00EF1210D0BAD8E9BEEA6886D804E0E846AF
:108BEA00FE0B0106FCE1E81C006EAFD8E9BEEA689C
:108BFA0022DAEF1640D039D875D9E8AE02D000345F
:108C0A0003D0E750D880005423E3FC0EDB5011E177
:108C1A009CD8E9BEEA6868D804E0E846FE0B01067B
:108C2A00FCE1E81C006E91D8E9BEEA680ADAEF16A0
:108C3A000FD08BD8E9BEEA6857D804E0E846FE0BA5
:108C4A000106FCE1006E81D8E9BEEA68FAD9EF12A2
:108C5A0012D0E66ED5EF47F0016E026A00C0E6FF59
:108C6A00E66E02C0E6FF71EF63F060D9E1CFD9FF8B
:108C7A00E2CFDAFF1200E552E5CFDAFFE7CFD9FFFC
:108C8A001200A951E96EEA6AB3EF47F0E66E000EE8
:108C9A00DA20E66E1200DE5157D9EF501200D9CF12
:108CAA00E9FFDACFEAFF1200E652E6523DEF48F05A
:108CBA00EA22EECF48F0EFCF49F012009AD9010E1E
:108CCA001200D890F336E8061200DE2BDE51006E51
:108CDA00016A000E00181200006EDF50005C1200DC
:108CEA00010EF36EDB501200C80EE926050EEA22C9
:108CFA00EF50016E010E01521200EE54000EEE54B6
:108D0A00000EEE541200DF6EDFCFE6FFDC51016A7F
:108D1A00000F006E020E012267D9B0EC5DF02CEF55
:108D2A0048F0E76E010EE7CFDBFF0701B4511200EE
:108D3A00010EE66E9BEF47F0EA22EECF4AF0EFCF44
:108D4A004BF012000BD9E8061200FD0EDBCFE9FF4B
:108D5A00EA6A1200DD51A9EF47F0FB0EDBCFE9FF0B
:108D6A00FC0EDBCFEAFF1200EA22EE50EFCFEAFF59
:108D7A00E96E00501200010EDB28006E010E00524F
:108D8A001200A951EA6A310FE96E0E0EEA22EF507B
:108D9A000E01EA6AAC25E96EAD51EA2212002ED91B
:108DAA00EECFE6FFEECFE6FFEECFE6FFEFCFE6FF30
:108DBA001200040EEECFDBFF050EEECFDBFF060E30
:108DCA00EECFDBFF070EEECFDBFF1200C7D8000E97
:108DDA00E926010EEA221200DBCFF4FFF350F45C1D
:108DEA001200006EFD0EDB50005C1200E652E652E5
:108DFA00E652020EDB6A1200EA6A290FE96E010ED8
:108E0A00EA221200036E050EE15C1200DBCFE6FFD8
:108E1A00E66A1200036E046A02C0E6FFE66E04C048
:108E2A00E6FF71EC63F0056E1200020EDBCF48F02C
:108E3A00030EDBCF49F01200E1D8EE50ED1012001C
:108E4A00FC0EDBCFE9FFFD0EDBCFEAFF1200016E5D
:108E5A00FD0EDB50015C1200DECF00F0DDCF01F029
:108E6A00000E005C100E01581200070EB715486E6E
:108E7A00010E4852120005016107000E625B635140
:108E8A001200010EDBCFE9FFEA6A1200E846FE0B88
:108E9A000006120063D8410EE926010EEA221200EA
:108EAA00040EDB28E96EEA6AB3EF47F0EA22E552DC
:108EBA00E750EF6E010EDB2A1200E66EE66A7FECDF
:108ECA0064F0E552E5521200FD0EDB50F80F006E19
:108EDA00010E00521200020EDBCFEEFF030EDBCFB3
:108EEA00EDFF1200FD0EDBCF00F0190EE76E001841
:108EFA001200100E616F270E626F1200AADEE66A78
:108F0A00D9501200A9DE2CEF48F0C0DE010E13EF93
:108F1A0048F0B7DE010EE9260E0E12009DDE07EFBD
:108F2A0047F0A3DEE652120092D8A5D6D9CFE6FFC3
:108F3A00DACFE6FF1200FCDE8CDE96EF46F0A1DE09
:108F4A00790EE9260E0E1200EA6A000FE96E030E88
:108F5A00EA22120090D8FF0EEE541200D890E93699
:108F6A00EA36120081D813EF48F08BDE490EE92663
:108F7A000E0E120071DE036E070EE15C1200110E76
:108F8A00E926050E95DE63EF46F0D6DE48504A5CC8
:108F9A0049504B581200030E39DF020E0BEF47F00F
:108FAA009DEC43F054D8E5521200D7DE040EDBCF15
:108FBA00EEFF050E1200C0DE4A5048181200110ECC
:108FCA00E926050EEA2212006ADEEE50ED101200C2
:108FDA0066DE010EEE18120062DE020EEE181200B4
:108FEA005EDE030EEE18120000C0E6FF01C0E6FFC7
:108FFA001200DECFE9FFDDCFEAFF1200E96E000EB4
:10900A00DA20EA6E120050DE050E78DF010F43EF18
:10901A0048F04ADE010E72DF010F12001ADE070164
:10902A00B45112008CDF44DE74DFEA224850120089
:10903A0078DFE652120092DF960EE926050EB9EFA6
:10904A0046F08CDF640EE926050EB9EF46F0E552CC
:10905A00E552E552120089DF2BDE8EEF47F0030E50
:10906A004DDF020F8AEF47F0020F10DE030E1200E7
:10907A00E66A9BEF47F013DED880120007DE010E86
:10908A0083EF47F04EDFBFDF020F8AEF47F0E3ECD2
:10909A004DF0A098636A626A0F01266BBAEC4EF033
:1090AA0002E2E16AE552E16E00500F0177EC4EF000
:1090BA00DF6ADF50006E016A0C0E005C000E015878
:1090CA0010E2DF50040DF3CFE9FFF4CFEAFF000E00
:1090DA00E926040EEA22EE6AEE6AEE6AEE6ADF2AF0
:1090EA00E8D7658C0F01386B6598659C62A607D036
:1090FA0062960201976B9C6B9D6B9E6BF7D7020180
:10910A00010EB06FB16FB26BB36BA46BDF6A030E63
:10911A00DF5C11E2EA6ADF34E7EC4EF0EA22EE6A3B
:10912A00ED6AEA6ADF34EEEC4EF0EA22EE6AED6AA4
:10913A0021EC4EF0ECD70201080E8D6F040E8E6FF3
:10914A000F01160E266F0401300E026F040E036F14
:10915A00400E016F840E006F0201816B806BE6EF97
:10916A004DF0E3EC4DF082BE06D0656A0F01366B16
:10917A000201806B7CD0020180510CE1656A0F010B
:10918A00366B77EC4EF065B602D06586FCD70201E5
:10919A00010E806F80050AE165BA08D0626A0F0184
:1091AA00366B368136890201020E806F6250040BDB
:1091BA0006E00F013651040B02E062943EDB65B211
:1091CA0056D06250010B09E00F013651010B05E040
:1091DA005EDF0201040E806F62906250100B06E09F
:1091EA000F013651100B02E018DB629862AC15D001
:1091FA000F0136AD0AD07EEC4EF0730EEDEC4DF059
:10920A0002E2E16AE552E16E0050629C0201AE514F
:10921A0001E0AE07AE5101E1F3D86250200B05E040
:10922A000F013651200B01E0E7DA6250020B14E01D
:10923A000F013651020B10E07EEC4EF0E6687F0E0D
:10924A00E66ECBEC60F0006E060EE15C02E2E16ACB
:10925A00E552E16E0050636A040E0201E76E80195E
:10926A00E8AE02D0E73402D0E750805D02E2A1986E
:10927A0034D00F0136A730D0DF6A040EDF5C2CE24F
:10928A0062A62AD064CFA5F20201A551780BE84262
:10929A00E842E842A66F6296A5B504D0A651F5EC5D
:1092AA004EF003D0A651FAEC4EF0EA22EF70A65126
:1092BA0002E1D5DA0FD0000EE66EE66AA50EE66E7A
:1092CA00020EE66E720EEDEC4DF002E2E16AE55234
:1092DA00E16E0050DF2AD1D7A198E6EF4DF0E4EC19
:1092EA004EF0FC0EDBA403D0E66A5FEC4EF0FC0EF7
:1092FA00DBA204D0010EE66E5FEC4EF0FD0EDB50F1
:10930A00016A260F006E0F0E59EC4EF0F5EC4DF087
:10931A00FC0EDBCFEFFFE552E6EF4DF0E4EC4EF04A
:10932A00FC0EDB5003E0E8EC4DF002D012EC4EF0FC
:10933A0045EC4EF0D9CFE9FFDACFEAFFEE50ED1057
:10934A0003E1F36AF46A28D0F5EC4DF009EC4FF02A
:10935A00FA0EDBCFEEFFFB0EDBCFEDFFF5EC4DF0A7
:10936A00EE52F90EDBCFEFFF400EFFEC4EF0880E07
:10937A000EEC4FF0FC0EDB5003E0E8EC4DF002D0AF
:10938A0012EC4EF0EA22EF74DECF00F0DDCF01F0EE
:10939A0000C0F3FF01C0F4FFE552E6EF4DF0E4EC44
:1093AA004EF0FD0EDB5003E1C3EC4EF009D017EC92
:1093BA004EF098EC4EF017EC4EF0010F98EC4EF090
:1093CA00E552E6EF4DF0CAEC4EF065A817D0DDEC99
:1093DA004EF0400EEE16EE6AEE6AEE6ADDEC4EF0E4
:1093EA00EE7CE8EC4DF0EA22EF74400E006EDDEC04
:1093FA004EF00050EF16DDEC4EF0EF7CB4EF4EF07D
:10940A000201B05123E1010EB06FB1511FE1010E0B
:10941A00B16F020E945D07E1E8DBEE52EF6AE5DB1D
:10942A00C80EEF6E1200940511E1A76B07EC4EF01F
:10943A00EE52400EEF6EE6DBA4EC4EF0E3DB840E58
:10944A00EF6E010EA76FB6DB800EEF6E12000201FF
:10945A00B26BB36B020E945D06E103EC4FF0D7DBFF
:10946A0093EC4EF010D098510401365D02019951E7
:10947A000401375904E236C498F237C499F25CD829
:10948A00B4DBC5DBB2DBC80EEF6E1200E4EC4EF0C3
:10949A00000EDE6E040EDD6EC5DB040DF4CF01F0A6
:1094AA00D9CFE9FFDACFEAFFF350EE260150ED22D9
:1094BA0097DBEF9EFC0EDB5002E1AFDB01D083DBD2
:1094CA00EA22DECFEEFFDDCFEDFF8ADBEF9C88DB01
:1094DA00040EE926000EEA22EF8CE55272D3659853
:1094EA00020197BF0DD09CAF09D0020E946FB35101
:1094FA0001E1ADDF0201B16BB06B1200C3EF4EF0B8
:10950A00040130AF0DD00201010E946FB25101E196
:10951A009EDF0201B16BB06BAF510DE105EF4AF06E
:10952A000201020E946F46DB840EEF6EB16BB06BD4
:10953A00AF5101E165DF120041DB400EDF6E02012F
:10954A00985D000E99590AE298C2DFFF935102E131
:10955A00010E03D0930502E1020E936FDF50016AF8
:10956A00E850985D986F01509959996F3EDBEE5219
:10957A00DFCFEFFF380EA16F040EA26F97B10DD0A7
:10958A00DF5017E095C2F6FF96C2F7FF952B000E43
:10959A0096230800F55067DBF3D7DF500AE095C23F
:1095AA00E9FF96C2EAFF952B000E9623EF505BDB8C
:1095BA00F4D707D3E4EC4EF025DBEE52EFCFDFFF12
:1095CA00DFCF00F0005002019D5D000E9E5902E2BD
:1095DA009DC2DFFFDF50006E016AE8509D5D9D6FFE
:1095EA0001509E599E6F010EDB6ADF50F36E010E29
:1095FA00DBCFF4FFF350F45C16E2010EDB50EA6AAB
:10960A00380FE96E040EEA22EF50E66E9AC2E9FFBD
:10961A009BC2EAFF9A2B000E9B23E552E750EF6E9E
:10962A00010EDB2AE2D7000ED8809D55000E9E550A
:10963A000DE2E4DBECDAE6DAEF50400B03E16EDB35
:10964A00C80E02D06BDB880EEF6E12D0B3DA840E2E
:10965A00EF6E9F51A01107E005D0A0C2FAFF0201E8
:10966A009F51F96EFADF02019C9FAF5101E1C8DEFA
:10967A00E552A7D2A3DA0201978F77DB02E2E16A09
:10968A00E552E16E0050300EE66EE66AE66A000EBA
:10969A00E66E040EDBDA02E2E16AE552E16E0050A0
:1096AA00658CDF6A030EDF5C02E2C6DAFBD7010EC5
:1096BA00E66EE66AE66A820EE66E020EC7DA02E233
:1096CA00E16AE552E16E0050659C0201080E8D6F59
:1096DA00040E8E6F000E836F040E846F83C285F2B0
:1096EA00866F32C481F2815102E1100E10D0010E50
:1096FA00E66EE66A810EE66E020EE66E010E68DA24
:10970A0002E2E16AE552E16E00500201200E806F2A
:10971A0058D2800E0401305D38E10201C00E976F05
:10972A0004013351030A1AE0010A09E0030A2BE192
:10973A0002017A0E956FC70E966F120E1ED0E7DAE7
:10974A00010EF626C80EBEDA020E0201D9DAF5CFEC
:10975A0098F2030ED5DAF5CF99F21200030E325DB4
:10976A000FE2D5DA030EF626C80EACDA95C2F6FF7A
:10977A0096C2F7FF0800F5500201986F996B120024
:10978A000201976B12000201976B120018DB0401A9
:10979A00386B396B30511F0B020A11E0030A0CE0D7
:1097AA00010A1EE10201978F040138810201A30513
:1097BA0017E10401388314D00201978F11D00201F6
:1097CA00978F040134BF02D0E9DA01D0ECDA58DA13
:1097DA00F2DA06E005DAEF50040B02E0010E386F08
:1097EA00020197AF07D0380E956F040E966F9781D6
:1097FA00020E986FE552E5D10F0126A10CD002DACC
:10980A00EF50800807E1F1D9EF50840803E1FAD953
:10981A008C0EEF6E2691629A12000F0136856298BD
:10982A0065820201010EA46F31DA750ED1D902E206
:10983A00E16AE552E16E005012000201A46B26DAD9
:10984A00740EC6D902E2E16AE552E16E00506592F1
:10985A000F01369562A402D06294FCD71200AED9E9
:10986A0002012D0EAE6FFD0EA51539E17E0EA5156E
:10987A00E8407F0B040DF3CF83F2F4CF84F2000E9D
:10988A008327040E842383C285F284C286F28575F7
:10989A00B9D9EF503C0BE842E8420D081EE1DF6AF5
:1098AA00080EDF5C16E2AED9020EE926000ED5D903
:1098BA00EF50E66EDF50EA6A300FE96E040EEA22D4
:1098CA00E552E750EF6E9ED99FDAEE2AEF22DF2AA1
:1098DA00E7D798D934DA09D807D027D805D0FD0EAA
:1098EA00A515040801E130D86CD10201936BAF6B66
:1098FA00B26BB36BA76B946B78D9EF9E8D7575D9E4
:10990A00EF9E8D750BDAEF9E976B986B996B9C6B3C
:10991A009D6B9E6B55D8BAD9030E5AD902E2E16AF9
:10992A00E552E16E005074EF4AF0020E0201945DB6
:10993A0002E1DFEF4AF0946BA75104E13BD98C0EA8
:10994A00EF6E1200A76B120039D94FD9EF50400BB6
:10995A0001E0010EDF6E02018D75080E805D0BE1DC
:10996A0032C438FF0F01385103E00201100E02D051
:10997A000201040E806F940513E137D948D9DCDD62
:10998A00020E0201935D03E130D9840E07D0DF5045
:10999A0003E12BD9C80E02D028D9880EEF6E0FD05A
:1099AA009CAF0CD09F51A01107E005D0A0C2FAFFCE
:1099BA0002019F51F96EFADF02019C9F946B01D15B
:1099CA0004013051600BE842E842E842E842E842CA
:1099DA00000901E0120031510C0A4AE00B0A3FE08B
:1099EA000C0A31E0010A22E00B0A1EE0020A1CE01E
:1099FA00030A18E0080A10E0010A0CE00F0A08E05E
:109A0A00030A01E012000201978F080E806F12000C
:109A1A008EEF4BF03FEF4BF00201810E956F020E75
:109A2A00966F0CD0CBEF4BF03EEF4DF03451020164
:109A3A00956F966B820E9527020E96239781010EDB
:109A4A00986F978F12000201978F04013451EA6AC6
:109A5A00820FE96E020EEA2232C4EFFF120016D913
:109A6A00020EB6D802E2E16AE552E16E0050120037
:109A7A001200A5D9E652E652E6520401320510E177
:109A8A0030511F0B00090CE10201978F030E0401EC
:109A9A00315D04E10201010EA36F02D00201A36B42
:109AAA000401325101E07FD030511F0B020801E05E
:109ABA007AD034510F0B000901E175D034510F0BE4
:109ACA00020871E3200E0201805D6DE1978F0401A7
:109ADA0034BF04D063D9D4D8DFD803D064D9D0D85E
:109AEA00DFD8EA22020EEFCFDBFFF4D8010B02E146
:109AFA00DF9401D0DF8434BF02D050D901D053D9CA
:109B0A00EA22DECFEEFFDDCFEDFF030E315D0CE181
:109B1A0052D907E034BF02D0BFD801D0C1D8EA2257
:109B2A00EF82840E76D93FD0DF7445D90BE058D83E
:109B3A00EF9E56D8EF8C09D902E2E16AE552E16E4E
:109B4A00005002D04DD8EF8CDF74C4D8020B02E16A
:109B5A0032D912E0040134BF02D09ED801D0A0D875
:109B6A00EA22EF923B0E006E45D9EFD802E2E16A93
:109B7A00E552E16E005002D03B0E3CD9040134514B
:109B8A000F0B016A260F006E0F0E0122030E00C092
:109B9A00DBFF040E01C0DBFF030EDBCFE9FF040E7F
:109BAA00DBCFEAFFEF90050EE15C02E2E16AE552E3
:109BBA00E16ED5D023D9C3D893EF4EF0E6D8E6525A
:109BCA001200E552CCD0FD0EEA6ADB34E7EF4EF024
:109BDA00E66EE66ACBEC60F0006E060EE15C1200FF
:109BEA00DECFE9FFDDCFEAFF12008DC2E9FF8EC2A8
:109BFA00EAFF120034510F0BE96EEA6AD890E9368F
:109C0A00EA36120083C2E9FF84C2EAFF1200FCD8D6
:109C1A00380EEE6E040EED6E1200FD0EEA6ADB34AB
:109C2A00EEEF4EF0FC0EDB50E824026EFD0EDB5028
:109C3A00040DF35002241200DF50D7D8EA22EF6A4B
:109C4A00DF50CED8EA22EF6ADF2A1200E66E24EC51
:109C5A0063F0006E050EE15C1200EA22EE50EFCFCF
:109C6A00EAFFE96E1200E66EA1C2E9FFA2C2EAFFAC
:109C7A00A12B000EA223E552E750EF6EDF06120079
:109C8A00EA22EECFDEFFEDCFDDFF1200000EE66E18
:109C9A00E66AE66EE66A120034510F0BF5EF4EF0F3
:109CAA0034510F0BFAEF4EF0012200C0DEFF01C063
:109CBA00DDFF1200FD0EDBCFE6FF4BEC4AF0E5526A
:109CCA00E5521200F7220900F5CF95F20A00F5CF06
:109CDA0096F21200D950020FE96E000EDA20EA6EEF
:109CEA00EF501200160E396F9F0E376F7B0E366FCC
:109CFA001200010EE66EE66A000EE66EE66A1200D1
:109D0A00F76A9525F66E9651F7220800120032512D
:109D1A00F66EF76AD890F636F736120085C2E9FF72
:109D2A0086C2EAFF1200040DF3CF00F0F4CF01F06F
:109D3A00000E0026040EB8DF840E0EEF4FF064D832
:109D4A00300EEE6E040EED6E1200020EE66EE66A3C
:109D5A00DECFE6FFDDCFE6FF050EEDEF4DF0E55273
:109D6A00E5CFDAFFE7CFD9FF1200020EE66EE66A08
:109D7A00E66A270EE66E0F0E2BEF4EF01BDF8C0EF7
:109D8A00EF6E33DF840EEF6E1200D9CFE6FFDACF23
:109D9A00E6FFE1CFD9FFE2CFDAFF12002BDF870E11
:109DAA00E926020E120026DF8D0EE926020E1200A7
:109DBA000ADF32EF4EF014DFEF50800B1200FEDEA6
:109DCA00E6521200FE0BEA36E96E8D0EE926020E05
:109DDA001200FE0BEA36E96E870EE926020E120021
:109DEA00EA6AAB0FE96E020E1200EA6AA80FE96E80
:109DFA00020E1200F5DEE850EF1612008FDFEE5267
:109E0A00400EEF6E93EF4EF0020EE926000EEA22A4
:109E1A001200E6DEE850EF1212004EEC54F0FB0E90
:109E2A00DBCFF3FFDB06F35000090AE09CEC54F0A9
:109E3A00FA0E07EC55F0F3E1011CF1E1010E01D035
:109E4A00000E7DEF54F04EEC54F03B0EE12402E399
:109E5A00E168E652E16E010EDB6A020EDB6AF90E78
:109E6A00DBCFF6FFFA0EDBCFF7FFFB0EDBCFF8FFF7
:109E7A000800F550DF6EDF5002E1A1EF53F0250E26
:109E8A00DF5C02E094EF53F0030EDB6A040EDB6A38
:109E9A00050EDB6A060EDB6A070EDB6AB6EC53F0C8
:109EAA002D0EDF5C0CE02B0EDF5C09E0200EDF5C80
:109EBA0006E0230EDF5C03E0300EDF5C1AE1DF50C0
:109ECA00300A14E0130A0FE0030A0AE00B0A05E05D
:109EDA00060AE4E1030EDB80E1D7030EDB82DED75C
:109EEA00030EDB84DBD7030EDB86D8D7030EDB88B1
:109EFA00D5D72A0EDF5C1BE1B2EC53F000EC54F02C
:109F0A0010E0030EDB803A683B68130EDBCF3FF0AC
:109F1A00140EDBCF40F0EBEC57F0040E38C0DBFF39
:109F2A0003D0130EE9EC53F0B6EC53F00BD0090E44
:109F3A00DB6A57EC54F003E0CBEC54F0FAD7090E85
:109F4A00E9EC53F0030EDBB0DB982E0EDF5C1BE16D
:109F5A00B6EC53F02A0EDF5C0BE1B2EC53F000ECE6
:109F6A0054F003E1130E3BEC54F0B6EC53F00BD073
:109F7A00090EDB6A57EC54F003E0CBEC54F0FAD745
:109F8A00090E3BEC54F0680EDF5C07E1B6EC53F0C7
:109F9A00680EDF5C1DE1030E18D0740EDF5C17E05B
:109FAA007A0EDF5C14E0480EDF5C06E0540EDF5CDC
:109FBA0003E05A0EDF5C02E1020E07D06C0EDF5C92
:109FCA0003E06A0EDF5C04E1010E8EEC54F0C9DB9B
:109FDA00DF506E0A01E17FD31E0A01E192D1200A05
:109FEA0001E18FD13F0A01E149D11A0A01E146D1C3
:109FFA000D0A01E143D1200A01E140D13A0A01E107
:10A00A003DD1200A01E13AD1260A01E135D10D0AF2
:10A01A0001E132D11A0A01E1D9D0200A4AE0300A14
:10A02A001FE0460A0EE0250A01E083D3D950F90F52
:10A03A00E96EFF0EDA20EA6E010EEE5E000EEE5AAF
:10A04A00EE5A9CEC54F0250EE66E95DB03E1011CFA
:10A05A0001E169D398EC54F001E26BD3DB2A69D3AE
:10A06A00080EDB6A040EDB50010806E2040EDB046C
:10A07A0060EC54F0DB508BDB080EDB5009E0030E7A
:10A08A00DB50010B05E172DB01E04DD3080EDB6A00
:10A09A0064DBEFCFDFFF10EC55F003E1011C01E1B7
:10A0AA0042D398EC54F001E3DB2A60DB01E141D3AF
:10A0BA003AD3070EDB5002080FE1DCEC54F0030E32
:10A0CA00A3EC54F00E0EEECFDBFF0F0EEECFDBFF4C
:10A0DA00100EEECFDBFF20D0F70EDBCF03F0F80E29
:10A0EA00DBCF04F0020E035E000E045AF70E03C023
:10A0FA00DBFFF80E04C0DBFF03C0E9FF04C0EAFF80
:10A10A0093EC54F0026A0E0E00C0DBFF0F0E01C082
:10A11A00DBFF100E02C0DBFF0E0EDBCFE6FF0F0ED9
:10A12A00DBCFE6FF100EDBCFE6FF4CEC63F0E55227
:10A13A00E552E552130E39C0DBFF140E3AC0DBFFBD
:10A14A00060EDB5005E0130ED7EC54F001E26ADB91
:10A15A00FBEC54F002E2130E37DBBEEC54F006E0DF
:10A16A00040ED7EC54F002E2050E2EDB030EDBB030
:10A17A0005D0FCDA01E0D7D2080EDB6A090EDB6AE9
:10A18A000E0EDBCFF6FF0F0EDBCFF7FF100EDBCF85
:10A19A00F8FF0800F550DF6EDF5014E001EC55F0CF
:10A1AA0011E210EC55F003E1011C01E1BCD2BBDB6A
:10A1BA0001E3DB2A090EDB2AD9500E0FE96E000EE5
:10A1CA00CBDBE7D7D3DA01E1B4D2ADD2C6DA110ECE
:10A1DA00EECFDBFF120EEDCFDBFF110EDBCFE6FF7A
:10A1EA00120EDBCFE6FF3EEC63F0E552E552130EAA
:10A1FA00F3CFDBFF140EF4CFDBFF060EDB5004E0D7
:10A20A00130ED0DB01E20EDBFBEC54F002E2130E7C
:10A21A00DBDAAFDB05E0040EC5DB02E2050ED4DAB9
:10A22A00030EDBB005D0A2DA01E07DD2080EDB6AAC
:10A23A00090EDB6A110EDBCFE9FF120EDBCFEAFF54
:10A24A00EFCFDFFFDF5014E0D7DB12E2E4DB03E1FC
:10A25A00011C01E168D267DB01E3DB2A090EDB2A74
:10A26A00110EDB2ADBCFE9FF120EE8E3DB2AE6D781
:10A27A007DDA01E15ED257D2030EDB8E070EDB04D4
:10A28A0010E195DB040E5ADB0A0EEECFDBFF0B0E54
:10A29A00EECFDBFF0C0EEECFDBFF0D0EEECFDBFFBA
:10A2AA006CD0070EDB5003082CE1030EDBAE0DD099
:10A2BA00B2DA020E76DAEFCF00F0016A026A036AB6
:10A2CA0000AE39D00168026835D0F70EDBCF01F055
:10A2DA00F80EDBCF02F0020E015E000E025AF70EF4
:10A2EA0001C0DBFFF80E02C0DBFF01C0E9FF02C0BC
:10A2FA00EAFFEFCF00F00A0E00C0DBFF0B0EDB6AAD
:10A30A0038D0070EDB50020809E1030EDBAE04D099
:10A31A0059DB02AE10D00ED055DB0DD0030EDBAEEA
:10A32A0012D079DA020E3DDAF9DA026A036A01AE6C
:10A33A0002D002680368E2DA0C0E02C0DBFF0D0EDF
:10A34A0003C0DBFF1AD0F70EDBCF02F0F80EDBCF2B
:10A35A0003F0020E025E000E035AF70E02C0DBFF84
:10A36A00F80E03C0DBFF02C0E9FF03C0EAFFD6DA3A
:10A37A00C5DA0C0EDB6A0D0EDB6A060EDB5005E150
:10A38A00010EF36E050EF3CFDBFF150EDB6A160E18
:10A39A00DB6AD950370F006E000EDA20016E390ED3
:10A3AA0000C0DBFF3A0E01C0DBFF380EDB6A080E85
:10A3BA00DB6A0A0EAEDADF50780A12E0200A10E0F1
:10A3CA00280A0CE0200A0AE03F0A06E00D0A02E029
:10A3DA00200A08E1020E05D0080E03D0080EDF2677
:10A3EA00100E97DA030EDBBE02D0DB92DB94DB5051
:10A3FA00800B24E08ADAD890030EEB50000A08E6B4
:10A40A00000EEE5C000EEE58000EEE58000EEE58EE
:10A41A0015E213DA3D683E683F68406847EC64F02D
:10A42A000A0E34C0DBFF0B0E35C0DBFF0C0E36C044
:10A43A00DBFF0D0E37C0DBFF2D0E08D0030EDBA2AB
:10A44A0002D02B0E03D0DBA408D0200EF36E170E19
:10A45A00F3CFDBFF150EDB2A02D0170EDB6A050EDF
:10A46A00DB5003E1B7D901E189D0620E006ECA0E52
:10A47A00016E000E026E070EDBCF03F0046A056A56
:10A48A00066A03C03DF004C03EF005C03FF006C0B6
:10A49A0040F0D3D9A5EC64F000503424F36E015097
:10A4AA003520F46E02503620F86EF4CFF7FFF3CF62
:10A4BA00F6FF0800090EF5CFDBFF580EDF5C0FE14F
:10A4CA00610EF36E090E7BD90AE3200E006E090EA7
:10A4DA00DBCFE7FF0050E75E090EE7CFDBFF070E91
:10A4EA00DBCF00F0016A026A036A0FDA00C03DF0AE
:10A4FA0001C03EF002C03FF003C040F0EECF38F09A
:10A50A00EECF39F0EECF3AF0EFCF3BF0A5EC64F0A6
:10A51A003BC0EDFF3AC0EDFF39C0EDFF38C0EFFF99
:10A52A00390EDBCFE9FFDB063A0EDBCFEAFF01E2A9
:10A53A00DB06090EDBCFEFFF150EDB2A4BD995E1BF
:10A54A00030EDBA61DD06F0EDF5C06E1C1D918E34E
:10A55A00150EDB285BDA14D0780EDF5C09E0580EA2
:10A56A00DF5C06E0620EDF5C03E0420EDF5C08E1BE
:10A57A00020EF36E160EF3CFDBFF02D0150EDB6A66
:10A58A00030EDB50100B0EE0040EDBCF00F0050EBD
:10A59A00DB50D880005406E2060EDB5003E1040EBD
:10A5AA00DB5034DA95D90AE2050EDBCFE7FF150E48
:10A5BA00DB50E75E050EE7CFDBFF02D0050EDB6A54
:10A5CA00040EDBCF00F0160E45D9D880005414E2F1
:10A5DA00160EDBCFE6FF150EDBCFE6FF040EDBCF50
:10A5EA00E6FF050EDB50E552E75CE552D880E754FA
:10A5FA00E552D880E7545FD9030EDB50010B0BE11B
:10A60A00080EDB5008E0B2D801E08DD0080EDB500E
:10A61A00BED8080EDB6A170EDB5007E088D9170E82
:10A62A00F1D903E1011C01E17ED0160EDB5016E0E0
:10A63A007ED9300EE66E9FD802E1011C74E077D90C
:10A64A00DFCFE6FF05EC64F0E552E552E552F4CFC0
:10A65A0001F00001F31C02E1011C65E0050EDBCFED
:10A66A0000F0160EDB50D880005409E2050EDBCF4D
:10A67A00E7FF160EDB50E75E050EE7CFDBFF300E75
:10A68A00E66E050ECBD94FE1390EDB2ADBCFE9FFA7
:10A69A003A0E01E3DB2ADBCFEAFF090EEFCFDBFF3D
:10A6AA00DB500EE044D9090EADD902E1011C3BE0B2
:10A6BA00390EDB2ADBCFE9FF3A0EEDE3DB2AEBD7D3
:10A6CA0055D831E1160EDBCFE6FF080EC3D8E552A6
:10A6DA00E7245DD82ED0070EDB50030A1CE0010ADE
:10A6EA0014E0030A07E07BD9DBCFEEFF020EDBCFD3
:10A6FA00EDFF1FD0F5D8056A03AE02D004680568DD
:10A70A002CD8BCD805C0EEFF14D0EAD803BE046822
:10A71A0024D8B4D80ED063D9DBCFEFFF0AD07BD9C7
:10A72A0005E1011C03E1F368F46810D0FCD801E3E9
:10A73A00DB2A79D93DEF4FF0010EDBCF00F0020E94
:10A74A00DBCF01F000C0F3FF01C0F4FF3B0EE15C78
:10A75A0002E2E16AE552E16ECBD029D9020EA3EFFB
:10A76A0054F061D90800F550DF6E1200200EE66E33
:10A77A00080E13EF55F005EC64F0E552E552E55288
:10A78A00F3CF00F0F4CF01F00001F31C1200006EC9
:10A79A00016AD950010F4DD90050EE260150ED2221
:10A7AA001200045E000E055AF70E04C0DBFFF80E15
:10A7BA0005C0DBFF04C0E9FF05C0EAFF1200DBCFDA
:10A7CA00F4FFF350F45C1200DB50E76E040EE7CF9F
:10A7DA00DBFF12000A0EDBCF00F00B0EDBCF01F01D
:10A7EA000C0EDBCF02F00D0EDBCF03F00050011090
:10A7FA00021003101200130EEECFDBFF140EEDCF82
:10A80A00DBFF130EDBCF00F0140EDBCF01F00001EB
:10A81A00800E01141200F70EDBCF04F0F80EDBCF26
:10A82A0005F01200050EDB50E66ED950130F01D960
:10A83A00E552E750EE6EED6A12000A0EDBCF38F0F1
:10A84A000B0EDBCF39F00C0EDBCF3AF00D0EDBCF5F
:10A85A003BF01200DBCFE6FF150EDBCFE6FF050E5D
:10A86A00DB50E552E724E552E7241200DB50CED84C
:10A87A00010EF36E060EF3CFDBFF1200EE50EFCFA0
:10A88A00EAFFE96E02C0EEFF03C0EEFF04C0EEFF6E
:10A89A001200D9CFE6FFDACFE6FFE1CFD9FFE2CF48
:10A8AA00DAFF1200DFCFE6FFE66A93EC64F0E552C6
:10A8BA00E552F3501200E76E080EE7CFDBFF1200F5
:10A8CA00EECF00F0EECF01F0EFCF02F0036A1200F4
:10A8DA00050EDBCF00F0150EDB50D88000541200B5
:10A8EA00010EDBCF02F0020EDBCF03F0046A120086
:10A8FA00E552E5CFDAFFE7CFD9FF12000A0E00C012
:10A90A00DBFF0B0E01C0DBFF1200D9500A0F1EEF4E
:10A91A0055F0F36E070EF3CFDBFF1200EECF00F017
:10A92A00EFCF01F01200010EDB2A020E1200FC0E1C
:10A93A00DBCFE6FFFD0EDBCFE6FF1200005E000E66
:10A94A00015AF70E00C0DBFFF80E01C0DBFF00C0A2
:10A95A00E9FF01C0EAFF1200DA20EA6EEF2AEECF21
:10A96A00F6FF000EEF22EECFF7FFEF22EECFF8FF51
:10A97A001200040EDBCFE6FF130EDB50E552E75C54
:10A98A009ADFDB5004DF060EDB501200090EDB50A3
:10A99A000A0DF350DF24D00FE76E090EE7CFDBFF75
:10A9AA00B6EF53F0DB50F36E050EE4EF53F0F70EFB
:10A9BA00DBCF00F0F80EDBCF01F01200DFCFE6FFAD
:10A9CA00C0EF53F028DF030EECDE65EF54F012EC13
:10A9DA004FF0E552E552E552E55200091200BDDE9C
:10A9EA00EE50EFCFEAFFE96E010E1200130EDB50B4
:10A9FA00F36E040EE4EF53F0040EDB50F36E090E0F
:10AA0A00E4EF53F0DBCFE6FFC0EF53F0E76E050E3D
:10AA1A00E7CFDBFF12008BDFE3EF54F0DBCFE6FF7B
:10AA2A0086DFECEF54F0D950F90FE96EFF0EB1EF63
:10AA3A0054F0E96E000EDA20EA6E1200439E08D046
:10AA4A00439E3BAE05D03A6C3B1EE86A3B22438EDE
:10AA5A003BC035F03AC034F0476A466A8E0E366E0D
:10AA6A00376AFDEF56F0439E0CD0439E3BAE09D0A9
:10AA7A00386C391E3A1E3B1EE86A39223A223B22BA
:10AA8A00438E3BC035F03AC034F039C047F038C085
:10AA9A0046F09E0E366E376AFDEF56F0436A39EC81
:10AAAA0057F051EC57F043B6E1EF56F043A205D008
:10AABA0043BAE1EF56F0E8EF56F043BAF4EF56F036
:10AACA0043A005D043B8E1EF56F0F4EF56F043B88F
:10AADA00E8EF56F0376A7F0E3C24366EE86A372272
:10AAEA004150365EE86A375A1A0E446E3C6A466A24
:10AAFA00476A346A356A3E50395E3F503A5A405086
:10AB0A003B5A000E3C5A09E73E5039263F503A223A
:10AB1A0040503B22000E3C2201D0468AD89039365A
:10AB2A003A363B363C36D890463647363436353692
:10AB3A00442EE1D73B503A103910D8A4468AFDEF8B
:10AB4A0056F0436A39EC57F051EC57F043B6E1EF4F
:10AB5A0056F043A205D043B8E1EF56F0E8EF56F0BD
:10AB6A0043AA05D043B0E1EF56F0E8EF56F043B000
:10AB7A0002D043A802D0F4EF56F0376A41503C2481
:10AB8A00366EE86A37227E0E365EE86A375A466AB9
:10AB9A00476A346A356A40503B02F4CF35F0F3CF46
:10ABAA0034F03F503B02F3504726F4503422000E53
:10ABBA00352240503A02F3504726F4503422000E10
:10ABCA0035223E503B02F3504626F4504722000EEF
:10ABDA00342235223F503A02F3504626F450472297
:10ABEA00000E3422352240503902F3504626F450E2
:10ABFA004722000E342235223E503A02F4504626AD
:10AC0A00000E4722342235223F503902F45046269C
:10AC1A00000E472234223522FDEF56F0417E436A68
:10AC2A0039EC57F051EC57F043B6E1EF56F043A236
:10AC3A000AD043AA03D043BEE1EF56F043A4EDEF96
:10AC4A0056F0EAEF56F043AA05D043ACEDEF56F0C2
:10AC5A00EAEF56F043A00AD043A808D043BE04D076
:10AC6A0043A402D0F6EF56F0FAEF56F0466A376A76
:10AC7A0041503C5C456E10E339C047F03AC034F0AD
:10AC8A003BC035F03CC044F03EC039F03FC03AF01A
:10AC9A0040C03BF0433A09D03EC047F03FC034F0D1
:10ACAA0040C035F041C044F0456C439E43BC438EDE
:10ACBA0044C036F043B029EF57F01A0E456029EF29
:10ACCA0057F0366A3C6A43A408D0396C3A1E3B1ED8
:10ACDA003C1EE86A3A223B223C2243AC08D0476C2D
:10ACEA00341E351E361EE86A342235223622386A68
:10ACFA00455207E03C343B323A3239323832452E3B
:10AD0A00F9D7395047263A5034223B5035223C5025
:10AD1A00362238C046F0439E36AE0BD0466C471EEC
:10AD2A00341E351E361EE86A472234223522362260
:10AD3A00438E36A006D0D880353234324732463276
:10AD4A00442A44C036F0FDEF56F0436A39EC57F016
:10AD5A0043B6B4EF56F043A20FD043B407D07F0EE8
:10AD6A003B6EFF0E3A6E396E386E25D0800E3B6E02
:10AD7A0001D03B6A000EF6D743B0FBD7386A9F0E64
:10AD8A003C60EBD77E0E3C64F4D79E0E3C5C07E039
:10AD9A00D8903B323A32393238323C2AF6D743A479
:10ADAA000AD0386C391E3A1E3B1EE86A39223A220A
:10ADBA003B223BAEDED712007F0E3C6EFF0E3B6E8F
:10ADCA003A6E396E12007F0E43BEFF0E3C6E02D001
:10ADDA007F0E3C6E800E3B6E3A6A396AF3D743AEF9
:10ADEA0004D0800E3C6E3B6AF7D73C6A3B6AF4D7C4
:10ADFA003550341047104610F8E037BEF0D735BE4C
:10AE0A000CD036503710EBE0D890463647363436F9
:10AE1A0035363606D8A03706F2D73750D4E1362869
:10AE2A00D2E046AE11D07F0E461402E147A00CD004
:10AE3A00472AE86A3422352207E3D8803532343289
:10AE4A004732362A3628BFE03650C9E047C039F0C3
:10AE5A0034C03AF035343B6E36303C6E3B323C9E61
:10AE6A0043BE3C8EE7EF56F03B363C3602E3438462
:10AE7A00437E06E143803C6A3B6A3A6A396A1200B9
:10AE8A003C2803E0D8803B321200D8903B3202E1E2
:10AE9A0043821200438612004036413602E3438C55
:10AEAA00437E06E14388416A406A3F6A3E6A12006D
:10AEBA00412803E0D88040321200D8904032EAE1BB
:10AECA00438A1200426A40AE70EF57F03F6C401E50
:10AEDA00E86A4022421E3BAE78EF57F03A6C3B1EBE
:10AEEA00E86A3B22421EE4EC64F03BBE88EF57F06E
:10AEFA0042AE000C3A6C3B1EE86A3B22366C371EA7
:10AF0A00E86A3722000C42BE7FEF57F04388FF0CF5
:10AF1A0096EC57F043B6000C43B0000C43A4000C67
:10AF2A00010C436A39EC57F051EC57F043B6120062
:10AF3A0043AE08D043A004D043A802D043801200F5
:10AF4A004390120041503C5C0BE140503B5C08E1ED
:10AF5A003F503A5C05E13E50395C02E14380120001
:10AF6A00D8A002D0438E10D03C5041C03CF0416E74
:10AF7A003B5040C03BF0406E3A503FC03AF03F6E03
:10AF8A0039503EC039F03E6E41503C5C10E0FF0F34
:10AF9A0009E0439043B403D043AE4384120043AE66
:10AFAA0043941200412AD89040323F323E323E50FA
:10AFBA00395E3F503A5A40503B5A3BBEEAD7D89086
:10AFCA0039363A363B363C2EF8D7C8D73BC047F01D
:10AFDA003AC046F03A503F02F4CF39F0F3CF38F096
:10AFEA003B504002F4CF3BF0F3CF3AF03F02F3502C
:10AFFA003926F4503A22E86A3B2246504002F3507E
:10B00A003926F4503A22E86A3B2240AE11EF58F052
:10B01A0046503A5E47503B5A47AE000C3F503A5EA4
:10B02A0040503B5A000C256C692C256C690A0D00AE
:10B03A00514D2C25692C25692C25692C25690A0D69
:10B04A0000253034692C253034690D0A0025316910
:10B05A000D0A00253033690D0A00253031306C7530
:10B06A000D0A0025640A0D0025642C256C752C2513
:10B07A006C752C256C752C256C750A0D004D616A52
:10B08A006F72206D616C66756E6374696F6E2041B4
:10B09A00786973322053746570436F756E74657284
:10B0AA00207A65726F0A0D004D616A6F72206D61B8
:10B0BA006C66756E6374696F6E20417869733220AD
:10B0CA0053746570436F756E74657220746F6F2068
:10B0DA0068696768203A20256C750A0D004D616A17
:10B0EA006F72206D616C66756E6374696F6E204154
:10B0FA00786973312053746570436F756E74657225
:10B10A00207A65726F0A0D004D616A6F72206D6157
:10B11A006C66756E6374696F6E204178697331204D
:10B12A0053746570436F756E74657220746F6F2007
:10B13A0068696768203A20256C750A0D002130205D
:10B14A004572723A203C61786973323E20737465A5
:10B15A00702072617465203C20312E3331487A2E7A
:10B16A000A0D002130204572723A203C61786973D9
:10B17A00323E20737465702072617465203E2032FD
:10B18A00354B2073746570732F7365636F6E642E0D
:10B19A000A0D002130204572723A203C61786973A9
:10B1AA00313E20737465702072617465203C2031D1
:10B1BA002E3331487A2E0A0D002130204572723A18
:10B1CA00203C61786973313E207374657020726126
:10B1DA007465203E2032354B2073746570732F736B
:10B1EA0065636F6E642E0A0D002130204572723A33
:10B1FA00203C6D6F76655F6475726174696F6E3E2F
:10B20A00206C6172676572207468616E203136370E
:10B21A003737323135206D732E0A0D002130204523
:10B22A0072723A203C61786973323E2061636365C9
:10B23A006C65726174696F6E2076616C75652069E0
:10B24A007320302E0A0D002130204572723A203CBC
:10B25A0061786973313E20616363656C65726174FC
:10B26A00696F6E2076616C756520697320302E0ACD
:10B27A000D002130204572723A203C6178697332A0
:10B28A003E206C6172676572207468616E20313687
:10B29A003737373231352073746570732E0A0D00D3
:10B2AA002130204572723A203C61786973313E2020
:10B2BA006C6172676572207468616E203136373747
:10B2CA00373231352073746570732E0A0D002130C0
:10B2DA00204572723A203C76656C6F636974795FB7
:10B2EA0066696E616C3E206C657373207468616E6A
:10B2FA0020342E0A0D002130204572723A203C7605
:10B30A00656C6F636974795F696E697469616C3EB3
:10B31A00206C657373207468616E20342E0A0D00E8
:10B32A002130204572723A203C76656C6F636974ED
:10B33A00795F66696E616C3E206C61726765722026
:10B34A007468616E2032353030302E0A0D0021309B
:10B35A00204572723A203C76656C6F636974795F36
:10B36A00696E697469616C3E206C617267657220EE
:10B37A007468616E2032353030302E0A0D005374F5
:10B38A00617475733D25690D0A0021352045727275
:10B39A003A204E65656420636F6D6D61206E657835
:10B3AA00742C20666F756E643A20272563270D0A70
:10B3BA0000506172616D383D25630D0A005061725B
:10B3CA00616D373D25630D0A00506172616D363D2E
:10B3DA00256C750D0A00506172616D353D256C64EE
:10B3EA000D0A00506172616D343D25750D0A0050D9
:10B3FA006172616D333D25640D0A00506172616DA1
:10B40A00323D25640D0A00506172616D313D25643B
:10B41A000D0A0050492C2531750D0A004D522C2574
:10B42A003033750D0A002C253032753A25303475C3
:10B43A00004100492C253033692C253033692C25ED
:10B44A003033692C253033692C253033690D0A00D5
:10B45A002138204572723A20556E6B6E6F776E20D6
:10B46A00636F6D6D616E642027256325633A25320B
:10B47A0058253258270D0A002138204572723A2081
:10B48A00556E6B6E6F776E20636F6D6D616E6420A3
:10B49A002725633A253258270D0A0021372045729D
:10B4AA00723A204578747261207061726D617465B8
:10B4BA00720D0A002136204572723A20496E766171
:10B4CA006C696420706172616D7465722076616C5A
:10B4DA0075650D0A002134204572723A204D697350
:10B4EA0073696E6720706172616D65746572287325
:10B4FA00290D0A002133204572723A2052582042FF
:10B50A007566666572206F76657272756E0D0A00D1
:10B51A002132204572723A20545820427566666577
:10B52A0072206F76657272756E0D0A0021312045A0
:10B53A0072723A2043616E277420737465702074A6
:10B54A0068617420666173740D0A002130200D0A47
:10B55A00002008002573001B5B421B5B314B1B5B01
:03B56A0030470067
:10B56E00D9CFE6FFDACFE6FFE1CFD9FFE2CFDAFFA0
:10B57E00240EE12402E3E168E652E16ED950FA0F9F
:10B58E00E96EFF0EDA20EA6E020EEECFDBFF030E3F
:10B59E00EECFDBFF040EEECFDBFF050EEECFDBFFB3
:10B5AE00E8D9F2D9BAEC61F0006E060EE15C02E267
:10B5BE00E16AE552E16E0050E76E0D0EE7CFDBFF5C
:10B5CE00DB50800815E0A0D93E6A3F6A406A416AA6
:10B5DE0000C039F001C03AF002C03BF003C03CF0AD
:10B5EE008DEC57F0010A10E1210E0701F16FF26B9D
:10B5FE00020EDB68030EDB68040EDB687F0EF36E53
:10B60E00050EF3CFDBFF66D10D0EDB50050B01E00F
:10B61E0061D10A0EDBCF00F00B0EDBCF01F0830EF3
:10B62E000026FF0E012200C0DEFF01C0DDFFD95053
:10B63E00060F65D976D9DF50010B0FE0DF06010E3C
:10B64E0001E2DB06D950180F5AD9D890EF36010E09
:10B65E00EB36020EEB36030EEB36D9CFE9FFDACF1F
:10B66E00EAFF020E3F6E406AEECF3AF0EDCF3BF0AE
:10B67E0067EC57F03AC0EEFF3BC0EDFF140EDB6AED
:10B68E00150EDB6A160EDB6A170EDB6A1C0EDB6A02
:10B69E001D0EDB6A1E0EDB6A010EF36E1F0EF3CF5C
:10B6AE00DBFF010EF36E0E0EF3CFDBFF0F0EDB6A28
:10B6BE000E0EDBCF00F00F0EDBCF01F0D890015055
:10B6CE0004E61A0E005C000E015801E398D0180E25
:10B6DE00DBCF00F0190EDBCF01F01A0EDBCF02F03C
:10B6EE001B0EDBCF03F0010E1F0B07E0D8900036C8
:10B6FE00013602360336E806F9E1180E00C0DBFF0C
:10B70E00190E01C0DBFF1A0E02C0DBFF1B0E03C0B9
:10B71E00DBFF140EDBCF08F0150EDBCF09F0160E93
:10B72E00DBCF0AF0170EDBCF0BF0010E1F0B07E07D
:10B73E00D890083609360A360B36E806F9E1D950A4
:10B74E001C0FDDD80850EE24046E0950EE20056E55
:10B75E000A50EE20066E0B50EE20076ED950180FD1
:10B76E00CED80450EE5C006E0550EE58016E0650B9
:10B77E00EE58026E0750EE58036E200E00C0DBFF2F
:10B78E00210E01C0DBFF220E02C0DBFF230E03C021
:10B79E00DBFF200EDBCF39F0210EDBCF3AF0220E8D
:10B7AE00DBCF3BF0230EDBCF3CF03C34000E3C18DD
:10B7BE0009E6D880000E3954000E3A54000E3B5460
:10B7CE00000E3C5411E2D950200F99D8AAD8D8D8DF
:10B7DE001C0EDB50EE121D0EDB50EE121E0EDB5059
:10B7EE00EE121F0EDB50EE12D9501C0F88D8AFD8B8
:10B7FE000E0EDB2A0F0E01E25BD7DB2A59D7C9D812
:10B80E00100E00C0DBFF110E01C0DBFF180EDBCFE8
:10B81E003AF0190EDBCF3BF0120E3AC0DBFF130EDF
:10B82E003BC0DBFFADD893D8D950100F68D8EE507F
:10B83E00ED1012E0D950120F62D8EE50ED1006E165
:10B84E00A8D8005001100210031006E099D8EE2A75
:10B85E00000EEE22EE22EE220C0EDB6A91D8060EC0
:10B86E00EECFDBFF070EEECFDBFF080EEECFDBFFDA
:10B87E00090EEECFDBFF7E0EF36E0A0EF3CFDBFF6B
:10B88E000B0EDB6AD950020FE66E000EDA20E66E62
:10B89E0070D848EC62F0E552E552E552E552DECF43
:10B8AE00E6FFDDCFE6FF70D81EEC61F0006E060EEF
:10B8BE00E15C02E2E16AE552E16E0050020E38C030
:10B8CE00DBFF030E39C0DBFF040E3AC0DBFF050EB3
:10B8DE003BC0DBFF19D800C038F001C039F002C000
:10B8EE003AF003C03BF0240EE15C02E2E16AE5525D
:10B8FE00E16EE552E5CFDAFFE7CFD9FF1200E96E30
:10B90E00000EDA20EA6E1200020EDBCF00F0030EFC
:10B91E00DBCF01F0040EDBCF02F0050EDBCF03F020
:10B92E001200180EEECFDBFF190EEECFDBFF1A0E54
:10B93E00EECFDBFF1B0EEECFDBFF1200EECFE6FFEE
:10B94E00EECFE6FFEECFE6FFEFCFE6FF1200D89088
:10B95E00030EEB32020EEB32010EEB32EF3212001F
:10B96E00EE500016EE500116EE500216EE50031673
:10B97E001200D950060FE66E000EDA20E66E1200A7
:10B98E00D950140F86EF5CF0D950020FB8DFA5EF37
:10B99E005CF0010E006E016A026A036AF1DFB7EF16
:10B9AE005CF0040130511F0B010801E01200305110
:10B9BE00600BE842E842E842E842E842010801E052
:10B9CE001200345103E0340501E012003151220A15
:10B9DE0031E0030A24E0010A15E0210A0DE0010A14
:10B9EE0001E012000201A00E956F070E966F080E71
:10B9FE00986F996B978121D00201A00E956F070E5B
:10BA0E00966F1BD036C49DF237C49EF20201800E93
:10BA1E009A6F070E9B6F9F6BA06B9C8F120002019B
:10BA2E00800E956F070E966F070E986F996BC10E6D
:10BA3E00976F120032C49BF70201978F1200070115
:10BA4E00806B4B0E816F826B836B846B856B080EE4
:10BA5E00866F8F6B1A0EE66E010EE66E74EC49F071
:10BA6E00E552E5521E0EE66E020EE66E74EC49F0DD
:10BA7E00E552E5522FD902E2E16AE5524FD90701AC
:10BA8E00996B9A6B906B12001CD982D9050E3A18DD
:10BA9E0001E13B5002E0000E18D051D90701975139
:10BAAE00001808E19851011805E114D902E2E16A83
:10BABE00E55234D944D907019951001805E19A513C
:10BACE00011802E1906B956B010E0CD1FAD80701AB
:10BADE008F6B9751981102E1000E05D045D9EF50AA
:10BAEE00800B01E0010E000931E1FB0EDBCF00F00F
:10BAFE003BD9EE52EF50D880005405E235D9EE52C4
:10BB0E00FB0EEFCFDBFF8F6BFB0EDB508F5D19E271
:10BB1E008F51EA6A400FE96E070EEA22EF50E66E89
:10BB2E008F51E76EFC0EDBCFE9FFFD0EDBCFEAFF98
:10BB3E00E750E926000EEA22E552E750EF6E8F2B12
:10BB4E00E3D7C8D802E2E16AE552E8D807018F517F
:10BB5E00C9D0B7D80701905107E1E7D8FB0EDBCF6C
:10BB6E0095F7010E966F906FBDD00BD917E1C0D827
:10BB7E00EDD802E101500BE0010EDBCFE9FFDB2A2D
:10BB8E00020EDBCFEAFF01E3DB2AEF50F1E1CDD865
:10BB9E00DFCF95F70701010E966F906FE552E552D4
:10BBAE00E552A0D0EED818E1A3D8D0D802E10150CA
:10BBBE000CE0010EDBCFF6FFDB2A020EDBCFF7FF28
:10BBCE0001E3DB2A0800F550F0E1AFD8DFCF95F79F
:10BBDE000701966B010E906FE552E552E55282D049
:10BBEE0070D8E652E652070199519A1102E1000E01
:10BBFE0008D099C7E9FF9AC7EAFFEF50800B01E022
:10BC0E00010E00095BE1030E905D01E1906B905116
:10BC1E0055E0020E905D0DE1E66A000EE66EE66AF4
:10BC2E008BD802E2E16AE55298D80701030E906FB5
:10BC3E0045D0900543E1400E006E016A9551005CBF
:10BC4E00000E015803E2400EDF6E02D095C7DFFFF3
:10BC5E00DF50955D956F000E936F070E946F010E7A
:10BC6E00DFCFDBFF96510BE1010EDB5012E091C7E7
:10BC7E00F6FF92C7F7FF0800F55043D8F5D7010E2F
:10BC8E00DB5007E091C7E9FF92C7EAFFEF5039D8C2
:10BC9E00F6D70701955107E1400EDF5C02E1020E77
:10BCAE0001D0030E906FDFCFE6FF000EE66E070E9B
:10BCBE00E66E42D802E2E16AE5524FD8E552E5520D
:10BCCE0011D0D9CFE6FFDACFE6FFE1CFD9FFE2CF31
:10BCDE00DAFF1200400EE66E400EE66E070EE66EBE
:10BCEE00E66A47D0E552E5CFDAFFE7CFD9FF12007B
:10BCFE00DF6A4ED8DE523AC0DEFF3BC0DDFFDD52BA
:10BD0E00120093C7E9FF94C7EAFFEF6E932B000E64
:10BD1E009423912B9223010EDB061200E16E00504C
:10BD2E00F3CF97F7F4CF98F71200FC0EDBCF91F715
:10BD3E00FD0EDBCF92F71200010EE66E1AD0FA0E50
:10BD4E00DBCF00F0FB0EDBCF01F01200DF2ADF505D
:10BD5E00006E016AFF0E00181200E16E0050F3CF64
:10BD6E0099F7F4CF9AF7120097C7E9FF98C7EAFF41
:10BD7E001200020EE66E93EC49F0006E050EE15CC9
:10BD8E0012009FDFE652E652E65207019051120072
:10BD9E00FC0EDBCF3AF0FD0EDBCF3BF012006AD982
:10BDAE00E6520E01006BA96BDF6A180EDF5C14E21F
:10BDBE0083D9010EE9260E0E85D9DF5077D9EF6AA9
:10BDCE007BD9490EE9260E0E7DD976D9790EE92654
:10BDDE000E0E78D9DF2AE9D70E01C60EAC6F0E0E05
:10BDEE00AD6F3F0E79140009796ECF0E79140009EC
:10BDFE00796E79827B6A7A6A79900F0152815293B9
:10BE0E00F00EB4140909B46E0E01080EAA6F030EDB
:10BE1E00AB6F800EAE6F3E0EAF6FE00EB06F2E0E9C
:10BE2E00B16F040EB66F900EB26F010EB36F900E1F
:10BE3E00B46F010EB56F000EE66EE66A010EE66E89
:10BE4E0037EC30F0E552E552E552E55229D112D9E0
:10BE5E00E652DF6A180EDF5C0AE2DF5027D9EFCF19
:10BE6E0000F0FD0EDB50005C0AE0DF2AF3D7DF6A3C
:10BE7E00180EDF5C08E2DF5019D9EF5002E1DF281F
:10BE8E0003D0DF2AF5D7000EE5520AD1F3D8070EFC
:10BE9E00E12402E3E168E652E16EDE6ADD6A020E3B
:10BEAE00DB6A030EDB6A040EDB6A050EDB6A060E26
:10BEBE00DB6A010EE66ED9CFE6FFDACFE6FF030EA0
:10BECE00E2D8020F03D9010EDED8030FFFD8030EFE
:10BEDE00DAD8050FFBD8030EFED80701B45124E1C2
:10BEEE00020EDB50180802E2B48D1ED0050EDBCF19
:10BEFE00E6FF060EDBCFE6FF030EDBCFE6FF040EFA
:10BF0E00DBCFE6FF020EDBCFE6FFDECFE6FFDDCFB7
:10BF1E00E6FF11D8006E070EE15C02E2E16AE5521F
:10BF2E00E16E00503EEC3EF0070EE15C02E2E16A8B
:10BF3E00E552E16EB5D09ED8E652E652FB0EDBCF4F
:10BF4E00E6FF85DFE552E76E010EE7CFDBFFDB5044
:10BF5E0002E1000E8CD0D950FC0FE96EFF0EDA20F4
:10BF6E00EA6EEE50ED101FE1010EDB049FD8EF508C
:10BF7E000E01EA6AAC25E96EAD51EA22EF6A88D865
:10BF8E00790EE9260E0E9ED883D8490EE9260E0E9E
:10BF9E0099D8010EDB048AD8EF6A7AD8010EE92609
:10BFAE000E0E90D862D0010EDB04006E0E01AA5167
:10BFBE00005C5BE2FB0EDB50180857E3FB0EDB5018
:10BFCE00070802E10601CF6B63D8010EE9260E0EBB
:10BFDE00EA22EE50ED1010E1E66AFB0EDBCFE6FF33
:10BFEE0000EC46F0E552E552E66AFB0EDBCFE6FFCB
:10BFFE00D2EC45F0E552E55206012351FDE0060173
:10C00E00030E306FF70EDBCF46F6F80EDBCF47F69A
:10C01E00486B496B190E3D6E3E6A3F6A406A46C6D2
:10C02E0038F047C639F048C63AF049C63BF047ECFF
:10C03E0064F034C046F635C047F636C048F637C011
:10C04E0049F6010EDBCF4DF6FB0EDBCF4CF6FC0EA8
:10C05E00DBCF4AF6FD0EDBCF4BF6F90EDBCF4EF6FD
:10C06E00FA0EDBCF4FF60601236B010EDB50E552C5
:10C07E00E55216D0D9CFE6FFDACFE6FFE1CFD9FFF2
:10C08E00E2CFDAFF120027D8010EE66ED950120069
:10C09E00010EDB04E96EEA6AD890E936EA36120040
:10C0AE00E552E5CFDAFFE7CFD9FF1200EA6A310F8A
:10C0BE00E96E0E0EEA221200EA6ADF34FE0BEA3651
:10C0CE00E96E1200EA22EE6AED6A1200E66E000ECA
:10C0DE00DA20E66E1200E66E9DEC43F0E552E55274
:10C0EE00E552E552120005D8B6EC48F0FDEC39F0F9
:10C0FE00FBD78ED8E652E6520F0148694969600EA9
:10C10E00D36E9B8C580EDE6E020EDD6EDFCF00F00E
:10C11E00DF06010EDBCF01F001E2DB06005001105D
:10C12E00F5E1948E70EC39F04CEC48F0E552E552A6
:10C13E0078D01200120012001200D8EF5CF012003C
:10C14E0026EF5DF00201A3051EE10201A4051BE12D
:10C15E00F1DF65920201A46B0701100EEF6F0E0E58
:10C16E00F06FEF07000EF05BEF51F011FAE165840E
:10C17E00080EEF6F070EF06FEF07000EF05BEF513A
:10C18E00F011FAE16594120043D8FC0EDBCF3AF0C1
:10C19E00FD0EDBCF3BF0050E3A1801E13B5036E0C9
:10C1AE00E8683A1802E17F0E3B182FE0030E3A18AA
:10C1BE0001E13B5028E0020E3A1801E13B5021E02C
:10C1CE00010E3A1801E13B501AE0740E3A1801E1E3
:10C1DE003B5013E0750E3A1801E13B500CE0730E24
:10C1EE003A1801E13B5005E0720E3A180FE13B5050
:10C1FE000DD0A1DF0BD09DDF09D09CDF07D0A0DFD3
:10C20E0005D09DDF03D099DF01D096DF010E09D056
:10C21E00D9CFE6FFDACFE6FFE1CFD9FFE2CFDAFFE3
:10C22E001200E552E5CFDAFFE7CFD9FF120096D81C
:10C23E00E1CFD9FFE2CFDAFF0C0EE12402E3E16891
:10C24E00E652E16ED950FA0FE96EFF0EDA20EA6E71
:10C25E00080EEECFDBFF090EEECFDBFF0A0EEECFA0
:10C26E00DBFF0B0EEECFDBFF79D8D950080FE96E4E
:10C27E00000EDA20EA6EEECFE6FFEECFE6FFEECF4F
:10C28E00E6FFEFCFE6FFBAEC61F0006E060EE15C62
:10C29E0002E2E16AE552E16E0050E76E070EE7CF6B
:10C2AE00DBFFDB50840B3AE1070EDB041AE1060ECE
:10C2BE00DB5006E0006A016A026A800E036E04D04B
:10C2CE00006A016A026A036A080E00C0DBFF090EEB
:10C2DE0001C0DBFF0A0E02C0DBFF0B0E03C0DBFF4B
:10C2EE001DD0F80EDBCF00F0F90EDBCF01F0D950E8
:10C2FE00040FE96E000EDA20EA6E0050EE260150B1
:10C30E00ED22D950080FE66E000EDA20E66E26D822
:10C31E0048EC62F0E552E552E552E552080EDBCFED
:10C32E0000F0090EDBCF01F00A0EDBCF02F00B0E90
:10C33E00DBCF03F000C038F001C039F002C03AF094
:10C34E0003C03BF00C0EE15C02E2E16AE552E16EE5
:10C35E00E552E5CFDAFFE7CFD9FF1200D9CFE6FFDE
:10C36E00DACFE6FF1200D9CFE6FFDACFE6FFE1CF54
:10C37E00D9FFE2CFDAFFE652006801687F0E026E47
:10C38E00036AD950FA0FE96EFF0EDA20EA6EEE500C
:10C39E000016EE500116EE500216EE5003166AD835
:10C3AE0000C0EEFF01C0EEFF02C0EEFF03C0EEFFC5
:10C3BE00FD0EDB50800B02E0010E01D0000EE66E8A
:10C3CE0059D8060EE926000EEA22E552E750EF6E26
:10C3DE00FC0EDBCF00F0FD0EDBCF01F0D890003667
:10C3EE000136FC0E00C0DBFFFD0E01C0DBFFDB5093
:10C3FE00E66E40D8040EE926000EEA22E552E7501A
:10C40E00EE6EED6AFD0EDB50006E016AFF0E001837
:10C41E0018E1015016E12ED8EECF00F0EECF01F06C
:10C42E00EECF02F0EFCF03F0005001100210031018
:10C43E0006E0210E0701F16FF26B800E0BD0040E99
:10C44E0009D0FD0EDB5008E115D8EE6AEE6AEE6AF1
:10C45E00EE6A010EDF6E06D0020EDF6E0BD8EE52C4
:10C46E00EE52EE8EDF50E552E552E5CFDAFFE7CF22
:10C47E00D9FF1200F80EDBCFE9FFF90EDBCFEAFF92
:10C48E001200D9CFE6FFDACFE6FFE1CFD9FFE2CF38
:10C49E00DAFF5BD8013411E20050FE08000E0154A1
:10C4AE000CE276D805E06CD8800EEE6EEE6847D0C2
:10C4BE0067D8800EEE6E7F0E0ED047D8D890015002
:10C4CE0004E6010E005C000E01580BE261D805E097
:10C4DE0057D8EE6A800EEE6E32D052D8EE6AEE6A01
:10C4EE002ED047D8EECF00F0EECF01F0EECF02F017
:10C4FE00EFCF03F032D800C0EEFF01C0EEFF02C056
:10C50E00EEFF03C0EEFF21D80050010B05E025D849
:10C51E00020E3AD8EF8E04D020D8020E35D8EF9EF8
:10C52E0014D8D8900132003218D8030E2DD800C07E
:10C53E00EFFF1AD804E011D8030E26D8EF8EE5527D
:10C54E00E5CFDAFFE7CFD9FF120013D8040E1CD8BF
:10C55E00EECF00F0EFCF01F01200FA0EDBCFE9FFC5
:10C56E00FB0EDBCFEAFF120004D8060E0DD8EF50FB
:10C57E001200FC0EDBCFE9FFFD0EDBCFEAFF12004F
:10C58E00ECDFEE6AEE6A1200E926000EEA221200D5
:10C59E00220E0701F16FF26BBBEF62F02A0EF66E00
:10C5AE00100EF76E000EF86E07010900F550EA6FD7
:10C5BE000900F550EB6F03E1EA6701D03DD00900A9
:10C5CE00F550E56F0900F550E66F0900F550E76F7D
:10C5DE0009000900F550E96E0900F550EA6E0900F0
:10C5EE0009000900F550E86F0900F550E96F0900E0
:10C5FE000900F6CFECF7F7CFEDF7F8CFEEF7E5C77A
:10C60E00F6FFE6C7F7FFE7C7F8FF0701E85302E1B9
:10C61E00E95307E00900F550EE6EE807F8E2E90786
:10C62E00F9D7ECC7F6FFEDC7F7FFEEC7F8FF070126
:10C63E00EA07000EEB5BBFD71200FE0EE3CFE9FF59
:10C64E00FF0EE3CFEAFFE9CFF3FFEACFF4FFFB0ED5
:10C65E00E35003E1FC0EE35009E0FB0EE30602E2B9
:10C66E00FC0EE306FD0EE350EE6EF1D71200FE0E49
:10C67E00E3CFE9FFFF0EE3CFEAFFF36AF46AEE526F
:10C68E0003E0F34AF42AFBD71200FF0EE3CFF8FFC4
:10C69E00E552FF0EE3CFF7FFE552FF0EE3CFF6FFB5
:10C6AE00E552E66AE66AE66A0900F55209E0FD0E11
:10C6BE00E32A05E1FE0EE32A02E1FF0EE32AF4D798
:10C6CE00FD0EE3CF39F0FE0EE3CF3AF0FF0EE3CFCF
:10C6DE003BF01200D9CFE6FFDACFE6FFE1CFD9FF6C
:10C6EE00E2CFDAFFE652E652E652E652D950FB0F9F
:10C6FE00006EFF0EDA20016E00C0DEFFDD6EDECFB3
:10C70E00E6FFDDCFE6FFFB0EDBCFE6FFFC0EDBCF59
:10C71E00E6FFFD0EDBCFE6FFF3C7E6FFF4C7E6FF4D
:10C72E0028EC4FF0006E070EE15C02E2E16AE55282
:10C73E00E16E0050020EF3CFDBFF030EF4CFDBFFF2
:10C74E00020EDBCF00F0030EDBCF01F000C0F3FFD3
:10C75E0001C0F4FF040EE15C02E2E16AE552E16E13
:10C76E00E552E5CFDAFFE7CFD9FF12001201000242
:10C77E0002000040D80492FD82010102000109026C
:10C78E004300020100C03209040000010202010050
:10C79E0005240010010424020205240600010524CC
:10C7AE000100010705810308000209040100020AC5
:10C7BE00000000070502024000000705820240004B
:10C7CE00000403090418035300630068006D006140
:10C7DE00006C007A00480061007500730016034576
:10C7EE0000690042006F00740042006F0061007229
:0BC7FE000064008CC7CFC7D3C7EBC797
:10C80A00D9CFE6FFDACFE6FFE1CFD9FFE2CFDAFFF1
:10C81A00FB0EDBCF00F0FC0EDBCF01F00001800E37
:10C82A0001141AE1FB0EDBCFE9FFFC0EDBCFEAFFB6
:10C83A00EECFF3FFEDCFF4FFEE2A000EEF22F3CF97
:10C84A00E9FFF4CFEAFFFD0EDBCFEFFFEF50016AFD
:10C85A00F36E01C0F4FF10D0FB0EDB50FE0806E1B8
:10C86A00FD0EDBCFE6FF18EC65F005D0FD0EDBCF41
:10C87A00E6FF6FEC3BF0E552E552E5CFDAFFE7CF92
:10C88A00D9FF120038503D02F3CF34F0F4CF35F01F
:10C89A003E02F3503526000EF420366E38503F0221
:10C8AA00F3503626000EF420376E38504002F3500B
:10C8BA00372639503D02F3503526F4503622000E01
:10C8CA00372239503E02F3503626F4503722395077
:10C8DA003F02F35037263A503D02F3503626F450C1
:10C8EA0037223A503E02F35037263B503D02F3506E
:10C8FA0037261200FF0EE124E96EFF0EE220EA6EEF
:10C90A00EDCFF4FFEFCFF3FFF46607D0600EF364C8
:10C91A0004D07B0EF36001D0F39A1200F36AF46A32
:10C92A00FF0EE124E96EFF0EE220EA6EED6607D003
:10C93A002F0EEF6404D03A0EEF6001D0F32A1200F2
:10C94A00376A366A356A346A200EE76ED890383606
:10C95A0039363A363B3634363536363637363D5042
:10C96A00345C3E5035583F5036584050375809E3EA
:10C97A003D50345E3E50355A3F50365A4050375A31
:10C98A00382AE72EE4D712004F4B0D0A000D0A0091
:10C99A004542427631335F616E645F61626F7665EC
:10C9AA00204542204669726D77617265205665722C
:0DC9BA0073696F6E20322E342E360D0A0088
:10C9C800376A366A100EE76ED8903A363B363636F6
:10C9D80037363F50365C4050375805E33F50365E97
:10C9E8004050375A3A2AE72EF0D71200C00EF36E9D
:10C9F80000EE00F00E0E01D81200EA6002D0EE6AD6
:10CA0800FCD7F350E9601200EE6AFCD71DEE00F087
:10CA18002DEE00F0F86A439CD5EC62F03AEC65F034
:10CA28007AEC60F0FBD71200FF0EE350ADBA04D0E9
:10CA3800B06AAC8EAD8A949CADA2FED7AE6EF36E92
:10CA4800F46A1200F36AF46AF32A0F0B05E0D8902F
:10CA5800F336F436E804FBE1120030313233343572
:0BCA6800363738396162636465660090
:10CA74001200FEFF000000000000000001000000A2
:10CA840000000000000000000000000000000000A2
:10CA94000000000000000000000000000000000092
:10CAA4000000000000000000000000000000000082
:10CAB4000000000000000000000000000000000072
:10CAC4000000000000000000000000000000000062
:10CAD4000000000000000000000000000000000052
:10CAE40000920F920F920F930F930F930F930F9344
:10CAF4000F930F930F930F940F940F940F940F941D
:10CB04000F940F940F940F950F950F950F950F9504
:10CB14000F950F890F890F890F8A0F8A0F8A0F8A41
:10CB24000F8A0F8A0F8A0F8A0F8B0F8B0F8B0F8B35
:10CB34000F8B0F8B0F8B0F8B0F8C0F8C0F8C0F8C1D
:10CB44000F8C0F8C0F00010500010203040506077A
:0ECB540000010203040506070203040506079C
:08FFF800ACF70AFF63F801F009
:00000001FF
